:020000040800F2
:10000000F0FF0010E570050829FC0408B1F50108AF
:1000100085710508857105088571050800000000D7
:100020000000000000000000000000002DFC04089B
:1000300031FC04080000000035FC040865BB010821
:1000400085710508857105088571050885710508A4
:10005000857105088571050859A101087DA1010870
:10006000B9A10108F5A1010831A20108CDBE00081F
:10007000E1BE0008F5BE000809BF00081DBF00086A
:1000800031BF000845BF0008857105088571050866
:100090008571050885710508857105086DA201083F
:1000A000F9F1010859F1010809F2010849F10108C3
:1000B00081F1010891F10108A1F10108B5B2000830
:1000C00079B70008BDB200087DB700088571050842
:1000D0008571050865B5010855B6010845B70108E1
:1000E000A9A20108857105082163050819F2010814
:1000F000D1F1010829F20108C1F1010859BF000836
:100100008571050885710508B1F10108857105083B
:1001100035B8010825B901088571050885710508FC
:100120006DBF000881BF000895BF0008A9BF000887
:10013000BDBF000885710508857105088571050832
:1001400085710508857105088571050839FC040865
:10015000D1BF0008E5BF0008F9BF000815BA0108C3
:10016000C5B2000881B700088571050885710508CA
:100170008571050885710508857105088571050873
:08018000857105088571050871
:0828000000C00F0800001008E1
:1080000082B01E4B002201920193019B1C4A043353
:108010000193019B1968936803F00C03042B06D0AD
:10802000082B08D0174B184A1A6002B07047154B3E
:10803000196002B070475368506813F4800F00F065
:108040003F00536812D1C3F388130F49B1FBF0F11D
:1080500001FB03F30A4A0B495268C2F301420132A1
:108060005200B3FBF2F30B6002B07047C3F3881306
:10807000B1FBF0F101FB03F3ECE700BF5028004037
:1080800000380240E81800200024F400074BD0F824
:10809000E4105B68D0F8F0205B1A9A42B8BFC0F8D1
:1080A000F030012380F81C3100207047001000E000
:1080B000B84B00EB800103EBC10170B54A68526810
:1080C000B2F814E01EF0010F4FEA800C6ED15FFA97
:1080D0008EF4A60742D5BFF35F8F91F82040012CA4
:1080E000E5B200F0D180118BBFF35F8F0CEB000184
:1080F00003EBC10191F82040022C00F0E7800CEB6B
:10810000000103EBC10191F82040032C07D191F845
:10811000221021B193F87D10002940F0E78091886A
:1081200089B241F48061918093F97C100CEB000ED0
:1081300003EBCE0E9EF820E00EF1010E8E450CD121
:10814000002183F87D1093F87E10002940F0B7805D
:10815000604403EBC00300225A7770BD65075DD40D
:1081600014F0400400F0CB80148A93F97C508E6A9E
:10817000E4B274555FFA85FE0EF1010464B291F821
:10818000206083F87C40E51CAE42214600F025814A
:108190000CEB000503EBC50595F82050AC42C5D1AA
:1081A0000EF1020149B283F87C10BFE7B2F800E09B
:1081B0002EF4006E4FEA0E4E4FEA1E4EA2F800E07B
:1081C0001488A4B244F48064148091F822400025FD
:1081D00083F87C50002C48D093F87D40002C41D08F
:1081E000012183F87D100CEB000103EBC10191F834
:1081F0002010022904D1118889B241F40061118054
:108200000CEB000103EBC101897F41F001011182F8
:10821000604403EBC00393F8203070BD91F8224016
:10822000012583F87E50002C70D093F87D40002CFF
:1082300071D10CEB000103EBC10191F82110002971
:1082400000F0AA80118889B241F40071118093F87E
:108250007C1001314CB283F87C401188CE05FCD4EF
:10826000214663E7C97FFF29BAD00CEB000103EB7D
:10827000C1018C7F04F0FE041482CA7FFF2AC7D09C
:10828000FF2283F87C20C3E791F8221000293FF4F5
:108290002AAF93F87D1000293FF425AF118821F40F
:1082A00080610904090C1180BFF35F8F118B118865
:1082B00083F87E5089B241F4007111802FE79188D4
:1082C00021F440710904090C918041E791F82210D2
:1082D00000293FF414AF93F87D1000293FF40FAF4D
:1082E000118821F480610904090C1180918821F41E
:1082F00080610904090C918093F97C1016E71FFA3C
:108300008EF52D062DD493F97C100FE793F87D1090
:1083100000298ED096E791F82040022C148846D987
:1083200024F480642404240C1480158A8E6A93F942
:108330007C40EDB235558E6A118889B241F40071E6
:108340001180E4B2158A611C49B2EDB2755491886E
:10835000023489B264B241F4806183F87C40918038
:108360007BE793F97C506E1C3ED04C6A665D1682AA
:108370006C1C91F8205064B2A54283F87C402146E1
:108380007FF4D4AE948824F480642404240C948074
:10839000CCE600BFE8180020118893F97C4089B230
:1083A00041F480711180012183F87D1055E7A4B25A
:1083B00044F400741480158A8E6A93F97C40EDB2FF
:1083C0003555E4B28E6A158A611C49B20334EDB2A8
:1083D00064B2755483F87C403FE7958825F4806546
:1083E0002D042D0C9580D3E683F87C40CC7F14823D
:1083F00091F8224024B991F8201000297FF408AFA9
:10840000918821F480610904090C918000E700BF84
:1084100030B5EAB18E464FEA014C034600F1C00583
:10842000002419689A6841EA0C0142EA0E029A6037
:10843000C3E900140C33AB42F3D1D0F8C030C0F81C
:10844000C44043EA0E03C0F8C030C0F8C84030BD95
:108450004FEA014E8C46E0E783691969B3F80CC016
:108460000A6830B49C6822F0010224680A60A2897C
:1084700092B222EA0C02A281027D04681F2A06D968
:108480006568203A08209040284245D0FEE72568DC
:10849000082090402842F9D1202000FA02F2A26080
:1084A000264A1278002A35D01A7E012A39D0D3F80C
:1084B000F4200132C3F8F420EFF31181502282F34B
:1084C000128858685C6C026822EA04029C6C2243A1
:1084D000C9B2026081F31188D3E90C401A69996826
:1084E0001D6C096814605061D3E90E4054609060BF
:1084F0000024B3F8A800D5604C62C862106801245B
:10850000204310601C7683F8F1408A899B891343CD
:108510009BB28B8130BC7047202000FA02F2E260EF
:10852000BEE7002283F8F120D3F8F8000A68013092
:1085300022F00102C3F8F8000A60EBE70400001023
:1085400010B40C4C6368002B11DD002004F1080C02
:108550000146DCF8A03003F1C00259600C339342AD
:10856000FBD16368013083420CF5807CF1DC5DF85F
:10857000044B704704000010F0B5494C04EB401C5C
:108580009CF8242402B9F0BD464B4FF08C0E0EFB34
:10859000003E93F8E06493F8E1249EF882708CF832
:1085A0000A7496424FF0000C4FEA40158EF882C0D4
:1085B0000ED002EB420C03EBCC0C57009CF8E4C449
:1085C0000CF1FF3EBEF1010F5CD9BCF1030F53D09B
:1085D0006019A0F80814EFF31182902383F3128836
:1085E00090F80A34B0F8081443EA41030021D2B2EB
:1085F0009BB280F80A1482F311881A09217882EA62
:1086000013225A40D9B1D0F82044D0F80C14D4F831
:10861000A040D2431B019BB202F00F020120884010
:10862000134304F1C0015A0013F4004F93B202D176
:108630006268024362600C348C42F4D1F0BDD0F821
:108640002014D0F80C04D1F8A0401B0100F1100157
:108650009BB202F00F0201208840134304F1C001D5
:108660005A0013F4004F93B202D162680243626071
:108670000C34A142F4D1F0BD02F1010C0CF0030C5A
:10868000B445A5D03A4403EBC202131893F8F11491
:1086900000299DD06319012283F80A2498E700BFBE
:1086A00004000010E8180020704700BF024B03EBE5
:1086B000401090F825047047040000104368B0F89B
:1086C000502010B41A83EFF31182502383F31288E1
:1086D0004168446C0B6823EA0403C46C2343D2B2A0
:1086E0000B6082F31188D0E9074182680369126840
:1086F0001C605961D0E909415C60C46A9960B0F8B6
:108700006010DC600023D1625DF8044B0376704793
:10871000037D1F2B30B54FF02002046816D9A3F15A
:1087200020056168AA400A420FD00C4A002182F855
:10873000441541680A681F2B22F001020A604FF0BD
:10874000200206D9203B9A40E26030BD21689A4061
:10875000E9E702FA03F3A360F7E700BFE818002097
:108760004FF40063838170473D4B9FED3E4A93F881
:10877000491593F8480593F84A2593F84BC5090223
:1087800001EB00410A44090248BF02F17F4207EEB3
:10879000902AB3F9642593F84C0593F84D1506EE2D
:1087A000102AB3F96025F8EEE77A06EE902A67EE14
:1087B000847AB3F96225B8EEC66AF8EEE66A00027A
:1087C000E7EE866A00EB0C40014406EE102AB3F98E
:1087D0005E2505EE102AD3F85825000207EE102A70
:1087E000B3F95C2548BF01F17F41F8EEC75A04EEAA
:1087F000902A07EE101AD3F85425B8EEC66AB8EEE0
:10880000C55AE6EEA75A012006EE902AB8EEC77ABE
:10881000A7EE865AB3F95225B3F9503527EE047AFC
:10882000F8EEE44AB8EEE66A06EE902AA7EE246A6D
:10883000E5EE075AF8EEE66A05EE103A26EE877A7C
:10884000B8EEC55AF6EE004AF0EE466AE7EEA56AC3
:10885000054BA5EE247AC3ED066A83ED077A7047CF
:10886000E818002008218436381E002030B10A4B59
:10887000D3ED067AFDEEE77AC0ED007A51B1064BF2
:108880009FED067AD3ED077A67EE877AFDEEE77AF9
:10889000C1ED007A704700BF381E00200000C842BA
:1088A000704700BF0120704701207047704700BF2C
:1088B000024B002083F87005704700BFE8180020C5
:1088C00038B590F82820012A04464FF0000307D05D
:1088D000427F5AB103F00100607780F0010038BD9B
:1088E000406A0268117B69B9637F0BB9012038BD0A
:1088F000094D0A49022305F2745211F001F995F865
:108900007535E7E7516A19B1884201D0002038BDBA
:10891000136A002BE8D0F9E7E8180020880100204E
:1089200038B590F82810427F012904461DD022BB9B
:10893000012038BD596A09B1884217D11B6AABB909
:10894000002AF5D00E4D0F49022305F2745211F0A2
:10895000D7F895F8753503F0010363771A46002BB5
:10896000E6D094F828100129F7D1606A0368197BD2
:108970000029DFD1002ADBD0E4E70023EBE700BFCA
:10898000E818002088010020012343770020704769
:10899000D0E90B2108B583690B4483610AB108460D
:1089A0009047002008BD00BF436A1B681B6A5B68D4
:1089B0005B78024613F0010008BF5077704700BF94
:1089C000C2628161704700BF704700BF04307047CA
:1089D0000C4B93F87C25D3F878150244D2B283F877
:1089E0007C2593F87C2508441206C3F8780505D544
:1089F00093F87C2582F0800283F87C25024B0122CB
:108A00009A707047E8180020880100202DE9F0478F
:108A1000144FD7F88055ED0A1ED00026B04607F552
:108A2000B769D7F884351048D3F828A0C7F8B085BF
:108A3000AC19641010234A46E102D0470F280BDD21
:108A40000A4B03F1100C53F8041B013107D16345A5
:108A5000F9D12546B542E4DCE802BDE8F087661CA2
:108A6000F8E700BFE81800206C1E0020A01E0020C0
:108A70001C4BD3F8C815D3F8CC258A1A322A16D83D
:108A8000D3F8E0258A4200D37047D3F8D42522B327
:108A90001068928810B444693231224218BF428370
:108AA0005DF8044B08BF0283C3F8E015704793F8E4
:108AB000D025D3F8D41502F0010219B132B90A68F1
:108AC000898811830022C3F8E02570470A688988E5
:108AD00051830022C3F8E02570473231C3F8E01516
:108AE000704700BFE8180020122301480B80704730
:108AF0008C010020042301480B807047A001002056
:108B00002048D0F8E837D0F8EC2730B59B184FF064
:108B10001A040C8001D11C4830BD1B4AD0F8EA175A
:108B20004FF0000E10467546B3F1204F4FEA137C0C
:108B30000CF130040EF1020E2ABF0CF1370C8470D8
:108B400080F802C0BEF1100FC5704FEA031300F1A8
:108B50000200E9D100200446B1F1204F4FEA117321
:108B600003F1300C00F102002ABF373382F812C043
:108B700093740828D4744FEA011102F10202EBD178
:108B8000014830BD00F0FF1FA4010020094A92F8FF
:108B9000D035D2F8D42503F001031AB123B91368F4
:108BA00092881A8300207047136892885A830020A5
:108BB000704700BFE81800204FF40070034B1060AE
:108BC000D3F8F0350B600020704700BFE818002094
:108BD0000020704701207047012070470020704737
:108BE000164BD0F8E0105A6810B50446D0F8D800FB
:108BF00071B1131A99420BDC94F8D030C4F8D82024
:108C0000012B10D0D4F8D4300133C4F8D43010BDC7
:108C1000D4F8E430C4F8D8200344C4F8DC3094F825
:108C2000D030012BEED104F1E801201D10F09EFEA2
:108C3000D4F8D4300133C4F8D43010BD001000E0B3
:108C400070B5214B214C94B0CDE90043022302932F
:108C50001F4B04930546231D012205930023CDE9F4
:108C60000632CDE90E33CDE910330B9313932B7FEE
:108C7000406A8DF80C20002B14BF052304230C93AD
:108C8000144B0993A4F108030A930E468DF8202093
:108C90008DF834208DF8482010F0BAFD2B7F8BB171
:108CA000330E04F8073C063C320C330A2270637022
:108CB000A670686A694610F059FE686A10F0A8FD4F
:108CC00014B070BD073CEFE7081F0020C80100206A
:108CD000A98900088989000810B5044694B050227B
:108CE000064968464FF07EFC606A694610F03EFE19
:108CF000606A10F08DFD14B010BD00BF50870508EC
:108D00002DE9F0410446406A1E460F46904610F099
:108D10007FFD237F002B40D02A4DA0690523C5F895
:108D20008030030E85F8493005F14A039870020C33
:108D3000000A58701A703B68C5F88C300020D8F8CB
:108D40000030C5F89430012E2363C5F8A4002CD060
:108D5000022E20D1D8F80420C5F89C00796885F847
:108D60009800C5F8A01013441749C5F8A8200120A1
:108D7000236385F8AC00C5F8B010144B617F606ABE
:108D800003F11402002914BF1946114610F0EEFD3C
:108D9000E36A93B1206BBDE8F0810A4DA06904231A
:108DA000C5F8803005F14903C0E7074B85F89860A6
:108DB000C5E92730C5F8A800DFE7606A10F028FD94
:108DC000E8E700BF8801002091890008D801002051
:108DD00000B583B081610192049A0093C2620123BD
:108DE0006A4601A9FFF78CFF03B05DF804FB00BFE2
:108DF000F0B5836993F8DC20012A8BB005462ED0AC
:108E0000023A012A36D893F84C21D3F89C101E4C14
:108E100062F07F030B708669D6F8A0305F1C0FCC20
:108E2000EC46ACE80F00D6F89C30CDE900370FCC0B
:108E3000ACE80F0094E803008CE80300694606F1F3
:108E4000100010F093FDAB691A69516A03F110002C
:108E500099B1884200D0FEE7116A0029FCD1D3F80D
:108E6000A0305A8852BAEA819A8852BA2A82DB889C
:108E70005BBA6B8201200BB0F0BD116A0029EED005
:108E8000116A0029F9D1EAE7A08705082DE9F04128
:108E900090F8DC30D0F8A060012B8AB0044653D0A3
:108EA00016D8D0F89C304FF0FF321A605A609A60A2
:108EB000DA60D0F8E0300522B3F57A7FC0F8F02010
:108EC00064D8032380F8DC3001200AB0BDE8F081CB
:108ED000023B012BF8D890F84D31D0F89C20424D40
:108EE00063F07F031370D0F8A03000F110085F1C0E
:108EF0000FCDEC46ACE80F00D4F89C30CDE900373C
:108F00000FCDACE80F0095E803008CE8030069463C
:108F1000404610F02BFD23695A6A12B190452ED0BD
:108F2000FEE71A6A002AFCD173885BBAA4F8D03035
:108F3000B3885BBAA4F8D230F38801205BBAA4F8F6
:108F4000D4300AB0BDE8F08190F84C2190F84D3152
:108F50009B1A5B100133DBB206EB430236F8133089
:108F60005BBAA0F8D03053885BBAA0F8D2309388AF
:108F70005BBAA0F8D43001200AB0BDE8F0811A6ACB
:108F8000002AD1D01A6A002AF9D1CDE703691A7BE9
:108F90002AB35B691BB390F8983003B390F84C3157
:108FA000D0F89C20C4F8A40063F07F03137090F8FD
:108FB0004C1190F84D31D0F8A0200C48C4F80401B1
:108FC0005B1A07330121C4F8FC30D4F89C3084F8D4
:108FD00000110A44C4E93D3284F8DC1074E702232E
:108FE00084F8DC3070E700BFA08705088D8000089A
:108FF0002DE9F041AB4C94F82236012B94B000F0EF
:109000009D81022B00F03D81002B00F05781A64D81
:1090100095F8C8305B060DF10E060DF10F0804A996
:1090200004F2246740F138814FF4F073A5F8CA3098
:109030000023CDE90833CDE90A3305930D930123CD
:1090400085F8CC308DF81C308DF83030974BC4F853
:10905000BC3603F10213C4F8C03603F10213C4F89E
:10906000C43603F10213C4F8C83603F10213C4F87E
:10907000CC3603F102138E48C4F8D03603F1021344
:10908000C4F8D43603F102130490C4F8D8369838E3
:1090900020230693019110F069FCD4F8243601993D
:1090A0005A6A002A2FD0BA4200D0FEE71A6A002A74
:1090B000FCD100238DF80E3005938DF81C300893F9
:1090C0000A930D9310931293012306930B938DF83B
:1090D00030308DF8443095F8C8308DF80F300022CC
:1090E000002374480191CDE90E230496CDF8248025
:1090F00010F03CFCD4F8243601995A6A002A37D083
:10910000BA4207D0FEE71A6A002AD2D01A6A002AA9
:10911000F9D1CEE71A6A002AFCD1002305938DF815
:109120001C3008930A930D93109312930123069316
:109130000B938DF830308DF8443094F8DC368DF890
:109140000F30022300228DF80E305A48019100237F
:10915000CDE90E230496CDF8248010F007FCD4F856
:10916000243601995A6A002A37D0BA4207D0FEE75E
:109170001A6A002AD1D01A6A002AF9D1CDE71A6AF0
:10918000002AFCD1002305938DF81C3008930A9324
:109190000D9310931293012306930B938DF83030A7
:1091A0008DF8443094F8DD368DF80F30032300221B
:1091B0008DF80E303F4801910023CDE90E2304962F
:1091C000CDF8248010F0D2FBD4F8243601995A6AE5
:1091D000002A3CD0BA4207D0FEE71A6A002AD1D052
:1091E0001A6A002AF9D1CDE71A6A002AFCD194F84C
:1091F000DE36002B53D0012B00F0B380032B14BFBD
:10920000C723F7238DF80F30002305938DF81C300A
:1092100008930A930D9310931293012300228DF863
:109220000E3006930B938DF830308DF84430214882
:1092300004960023CDE90E23CDF8248010F096FB90
:10924000D4F824365A6AAAB1BA4207D0FEE71A6A9D
:10925000002ACCD01A6A002AF9D1C8E71A6A002A73
:10926000FCD1B5F8CA201448002114B0BDE8F04183
:109270004FF01BBA1A6A002AF3D01A6A002AF9D1F1
:10928000EFE7094D082385F8C8300DF10E060DF102
:109290000F0804A904F224674FF4C373C6E64723FA
:1092A000B0E700BFE818002088010020100111017C
:1092B000A41F00200C1F0020C81F00200122A02195
:1092C0000DF10E0604F22467CDE90463CDE90833FD
:1092D0008DF80E10069204A98DF81C300B928DF8B3
:1092E00030208DF844200D930022109312930DF13D
:1092F0000F0800233846CDE90E230191CDF82880D0
:1093000010F034FBD4F8243601995A6A12B1BA42EB
:1093100020D0FEE71A6A002AFCD19DF80F30144DC8
:1093200003F00602022A03D003F00503012B1AD032
:10933000082385F8C8304FF4C37377E60C4D4823F3
:1093400085F8C8300DF10E060DF10F0804A904F2DE
:10935000246769E61A6A002ADFD01A6A002AF9D15E
:10936000DBE787234EE7482385F8C8305CE600BF7B
:1093700088010020F0B511F0010583B00AD190F802
:109380002860012E044607D0C368B3F1807F01D95D
:109390000123237703B0F0BD0A4B476AD3F8C00816
:1093A00010F044FAE368B880B3F1807FF2D9B721B6
:1093B0008DF80410267733462A46384601A910F066
:1093C0009FFBE7E7E81800202DE9F043044695B03D
:1093D000406A334D0E469146984610F019FA314BCB
:1093E0000193314B049305F1D8030093217F0223AD
:1093F000029305F1D002012300278DF80C3005926D
:109400000697002935D08DF834308DF84830CDE9F5
:109410000977330ECDE90E77CDE9107785F8D13095
:109420000523CDF82C908DF82070CDF8308013975F
:10943000D2350793330C1D4F2B70330A6B70AE700F
:10944000D7F8C008656A10F0F1F9637FA8802BBBDC
:1094500005A9284610F08AFA606A10F0D9F9D7F801
:10946000C80810F0E3F9636A9880404615B0BDE87B
:10947000F0838DF834308DF848300423CDE909119C
:10948000CDE90E11CDE91011CDF82C908DF82010FA
:10949000CDF830801391D1350793CBE76946D8E7F3
:1094A00088010020AC210020A9890008E8180020CC
:1094B0002DE9F04112F0A2FB1F4F204E05464FF060
:1094C00000087C68002C2ADD00231A4607EB0321E4
:1094D000013391F8F9109C4242EA0102F6D142EAC6
:1094E0000804E4B290467368C3F30803A3B9EFF32A
:1094F00011838BB914F0ACFB431BB3F5FA6F02DC9C
:10950000B8F1000FDDD124B10D4B93F8CC284F2AD0
:1095100009D02046BDE8F08112F042FBECE744465A
:109520004FF00008DFE7B3F8D4280132A3F8D428BD
:109530002046BDE8F08100BF0400001000ED00E00F
:10954000E81800202DE9F04FDFF8C89299F800A044
:1095500091B0BAF1000F03D1012011B0BDE8F08F36
:10956000A849D9F80835A84A0493D1F8C835CDF8E8
:1095700000A0A2FB0323A54A5B09A2FB032E4FEA2E
:10958000DE0E0EEB8E0EA3EB4E0E91F8E134182298
:1095900002FB031303F2F1430F930B4691F8D81823
:1095A000029193F8CC180391B3F9D6180B91D9F81E
:1095B00014150191B3F9D018B3F9D23806910022ED
:1095C000D9F810150D9309F214645FFA8EF317465B
:1095D0000C920891079304EB8E0E09F5816609F24F
:1095E0000C5B09920E920A920592049BBB4240F3D7
:1095F000E0807368B2694FEA830AD2E93A310AF12E
:10960000085A0AEB431A01F18060029B39380AEBD1
:1096100080100AEB8313984240F288811A68002A6E
:1096200000F070811A6C002A00F06E81D3F880205F
:10963000002A00F06B81D3F8C02003F58073002A64
:10964000E9D1039DA3EB0A0A4F2D4FEAAA12CAF3F0
:10965000871A00F03881984240F29F80891A452984
:109660004FF0000528BF452103EB8111984628469D
:10967000AC460DE01A6C002A40F0CE80D3F8802072
:10968000002A40F0F480D3F8C02003F580732AB993
:10969000994206D91A68002AECD04033994200F268
:1096A000BF806546112D40F25A81CCF11503002B85
:1096B000C0F25581AAF10A0A5FFA8AF2029206D034
:1096C00098400122CCF1140302FA03F318435049E5
:1096D000C0F3C43301EB83030D469A6F00F01F0300
:1096E00001EB83039B6F43EA0233C0F3441201EBA7
:1096F0008202C0F3842105EB8101926F896F43EAF6
:10970000021343EA012181EA112383EA131303F0D0
:109710000F030F2B40F0C980B1F5803F80F0C5806A
:10972000039B4F2B4FEA111100F0D580019BB1F53F
:10973000606F03F10103019300F0DA80ABF80C10C5
:1097400094F858300798834210D0DEF80820236838
:109750009B1A2360DEF8302063689B1A6360002345
:10976000CEF80830CEF8303084F858002368013342
:109770002360DEF808300133CEF808304FF6FF736F
:10978000994240F08F80636801336360DEF83030C7
:109790000133CEF83030009B05930137082F04F1D8
:1097A0005C040EF15C0E06F120060BF1140B7FF445
:1097B0001CAF059B1BB1134B029A83F8D8280A9B58
:1097C0001BB1104B0B9AA3F8D6280E9B1BB10D4B67
:1097D0000D9AA3F8D228099B1BB10A4B069AA3F84D
:1097E000D028059B13B1019BC9F814350C9B13B10C
:1097F000089BC9F810350123012089F8123611B0F1
:10980000BDE8F08FE81800201F85EB51CDCCCCCC03
:109810005087050804000010803399427FF641AF5D
:10982000A3EB08029211551C4F4A82FB0582A2EB62
:10983000E572012AB8BF0122904001259444013A03
:1098400005FA02F210431D462A6892B12A6C002ADA
:109850005ED0D5F88020002A5CD0D5F8C02005F570
:1098600080753AB1A942EFD898462B4610E7C0332D
:1098700014E74035A942F7D9EB1A9B115A1C3A4B11
:1098800083FB0283A3EBE273012BB8BF0123984053
:109890009C440122013B02FA03F318432B469846ED
:1098A0002B46F5E6009B059377E7039B4F2B33D0C0
:1098B000019B01330193089B01330893009B0C9398
:1098C0004FF6FF713CE70FFA8AF598420B953DD9A8
:1098D00000980A90C2E6069B01331BB20693019BD7
:1098E00001330193B1F5606F009B09937FF426AFBC
:1098F0000F9BDB5D0D2B7FF421AF6FF07F038BF8A7
:109900001E301DE740339CE680339AE6C03398E66C
:109910008035AFE7C035ADE7069B01331BB2069338
:10992000019B01330193009B0993C4E7039DA3EBC3
:109930000A0A4F2D4FEAAA12CAF3871A7FF48BAE98
:109940000FFA8AF30B93009B0A9301E0009B0A93A2
:109950000D9B01331BB20D93009B0E931DE7039BE0
:109960004F2B7FF41AAFF3E75655555510B5044603
:109970004EF0C0F981B22046BDE81040FEF7FCBDB4
:109980002DE9F0411E4B93F8E02493F8E1349A421C
:109990002FD11C4F7D68002D12DD3846002410F8B1
:1099A000086BA046013416B1037E012B1CD002695E
:1099B0001368AC4243F0010300F580701360F1D1ED
:1099C00012F01CF9D7F8F448002C0BDD0E4A02EB1C
:1099D000C404116893888889083203439BB2944277
:1099E0008B81F6D1BDE8F08180F8F080FEF766FE4D
:1099F000DDE74AF08DF90028CBD1BDE8F08100BF4A
:109A0000E818002004000010FC08001010B57D4C80
:109A100094F8E02494F8E1349A4240F099817A4B2A
:109A200093F81829002A00F0EC8093F81C39002BD9
:109A300040F0EC80D4F8DC18088820F080000004A6
:109A4000000C0880B4F8E008C862088880B240F0D2
:109A5000800008804B62B1F80CC0B4F8F00840EA0E
:109A60000C0080B2012A8881A4F8F03800F0C98087
:109A7000D4F8F418088820F080000004000C088056
:109A8000B4F8F808C862088880B240F08000088006
:109A90004B62B1F80CC0B4F8080940EA0C0080B27F
:109AA000022A8881A4F8083900F0AB80D4F80C1998
:109AB000088820F080000004000C0880B4F8100929
:109AC000C862088880B240F0800008804B62B1F81C
:109AD0000CC0B4F8200940EA0C0080B2032A888147
:109AE000A4F8203900F08D80D4F82419088820F0DB
:109AF00080000004000C0880B4F82809C8620888B7
:109B000080B240F0800008804B62B1F80CC0B4F81D
:109B1000380940EA0C0080B2042A8881A4F8383958
:109B20006FD0D4F83C19088820F080000004000CA5
:109B30000880B4F84009C862088880B240F080000C
:109B400008804B62B1F80CC0B4F8500940EA0C0030
:109B500080B2052A8881A4F8503952D0D4F854191B
:109B6000088820F080000004000C0880B4F8580930
:109B7000C862088880B240F0800008804B62B1F86B
:109B80000CC0B4F8680940EA0C0080B2062A88814B
:109B9000A4F8683935D0D4F86C19088820F0800012
:109BA0000004000C0880B4F87009C862088880B20C
:109BB00040F0800008804B62B1F80CC0B4F8800916
:109BC00040EA0C0080B2072A8881A4F8803918D0B6
:109BD000D4F88429B4F88809118821F08001090497
:109BE000090C1180D0621088B4F8981980B240F046
:109BF0008000108053629089014389B29181A4F85A
:109C0000983910BDE818002004000010D4F8E4389A
:109C1000B4F8E81859601968D4F8DC0841F001017B
:109C2000196040F20D33A0F84830818989B241F4BF
:109C30008071012A8181E4D0D4F8FC18B4F80009BD
:109C40004860086840F001000860D4F8F408A0F803
:109C50004830818989B241F48071022A8181D0D053
:109C6000D4F81419B4F818094860086840F00100E5
:109C70000860D4F80C09A0F84830818989B241F411
:109C80008071032A8181BCD0D4F82C19B4F8300932
:109C90004860086840F001000860D4F82409A0F882
:109CA0004830818989B241F48071042A8181A8D029
:109CB000D4F84419B4F848094860086840F0010035
:109CC0000860D4F83C09A0F84830818989B241F491
:109CD0008071052A818194D0D4F85C19B4F86009A8
:109CE0004860086840F001000860D4F85409A0F802
:109CF0004830818989B241F48071062A818180D0FF
:109D0000D4F87419B4F878094860086840F0010084
:109D10000860D4F86C09A0F84830818989B241F410
:109D20008071072A81813FF46CAFD4F88C19B4F8A4
:109D300090294A600868D4F8842940F0010008603E
:109D4000A2F8483093899BB243F48073938110BD8D
:109D500049F0DEFF00287FF462AE10BD70B5104EF2
:109D6000D6F80835002B19DD06F58164002505E0DD
:109D7000D6F80835AB4204F120040FDD237F01350E
:109D8000002BF5D0E0680028F2D0217D10F04EFCC9
:109D9000D6F80835AB4204F12004EFDC012070BD99
:109DA00004000010F8B5037D85691F2B04464CD9CB
:109DB0000168A3F120024E6820209040064233D073
:109DC00010239340C860CB604B68D340DE077BD440
:109DD000EFF31183502282F312882A6C1168C907AD
:109DE0005AD4516889B271B9D5E90960864250D018
:109DF000AF690744D7606CD9301A80B25060AE6248
:109E0000002185F86410116841F00101DBB2116096
:109E100083F3118895F86430002B44D1237D1F2BE8
:109E200027D92168A3F120024C6808209040044201
:109E300000D0C8604C68042000FA02F2224203D02D
:109E4000203B00FA03F3CB60F8BD026820201668BF
:109E50009840064219460ED01021994090609160BA
:109E60001168D940C807B3D5012101FA03F3936003
:109E7000AEE722681946106808238B40184200D0CC
:109E800093601068042303FA01F10142DCD0916071
:109E9000F8BD012285F86420DBB283F3118895F8C0
:109EA0006430002BBAD095F87C30002BB6D195F8F1
:109EB000710011F02FF8012385F87C300028ADD017
:109EC000202110F0B3FBA9E7012303FA02F2CA60D4
:109ED0007EE72E69301A80B25060A96290E700BF19
:109EE0002DE9F047037D02681F2B044608D950680E
:109EF000A3F120052021A940014206D1BDE8F08749
:109F00001068202199400142F8D0BB49BB4E4968F6
:109F1000C6F8201996F81C19D4F81890DFF8E482D6
:109F2000F1B98C2101FB0981D1F88800D1F80071C9
:109F300005683868B1F88CC020F001003860A98944
:109F400089B221EA0C01A9813178E9B91F2B40F2CD
:109F5000B580A3F1200120238B40D360BDE8F087BA
:109F60008C2101FB0981D1F8881048690D680168CE
:109F700021F001010160A98921F480710904090C13
:109F8000A98131780029E1D04FF08C0A0AFB098AB7
:109F9000DAF80071384644F0F1FDD6F8283901228C
:109FA0008AF8D420002B00F0F5802A888C2303FB4C
:109FB000098392B242F080022A80B3F8F4204FF075
:109FC000FF31E962002A7FD12A8CB3F8F610B3F88A
:109FD000F800B3F8FCC022F001021204120C2A842B
:109FE000B3F8FA202B8B23F0F3031B0440EA0C1088
:109FF0001B0C0343288C9BB22B8383B223F00A03F0
:10A000000B4343F001032B842B8B23F00C031B0425
:10A010001B0C2B832B8B9BB21A432A838C2303FBB1
:10A0200009830022D3F8AC00C3F8A420D3F8982009
:10A0300039680243D3F8B0000243D3F8B4000243B6
:10A04000D3F8B8000243D3F8BC000243D3F8C000F1
:10A050000243D3F8CC000243D3F8D000024368484F
:10A06000084002433A60D3E931207969024321F084
:10A0700007010A437A61D3F8A8207A60D3F89C20BC
:10A08000BA60D3F8A020FA60D3F8002116215160FD
:10A09000116841F001011160D3F88820B3F88C30C9
:10A0A000126891890B439BB2534993814B68C6F860
:10A0B0002439237D22681F2B3FF64BAF202101FA64
:10A0C00003F39360BDE8F087042A33D0082A2A8C72
:10A0D00065D022F48052B3F8FC10B3F8F800B3F85E
:10A0E000F6C01204120C2A84090341EA0020A98B4D
:10A0F000B5F820E0B3F8FA2045F6FF7303EA0E0343
:10A1000043EA0C3340F6FF4C0CEA01019BB20143D9
:10A1100043F4805389B2A9832B84AB8B23F440632F
:10A120001B041B0CAB83AB8B9BB243EA02239BB299
:10A13000AB8373E7298CB3F8F820B3F8FC00B3F8CD
:10A14000F6C021F010010904090C29841202B3F8A9
:10A15000FA1042EA0032288B2B8C9BB223F0A0032A
:10A1600043EA0C1340F6FF4C0CEA00009BB202439A
:10A1700043F0100392B22A832B842B8B23F4406389
:10A180001B041B0C2B832B8B9BB243EA01239BB23A
:10A190002B8343E711F032FDC6F8280905E722F4C6
:10A1A00080721204120CB3F8F600B3F8F810B3F88A
:10A1B000FCC02A84B3F8FA20AB8B23F0F3031B0412
:10A1C00041EA0C111B0C0B4399B22B8CA9839BB257
:10A1D00023F4206343EA00239BB243F480732B846F
:10A1E000AB8B23F00C031B041B0CAB83AB8B9BB220
:10A1F0001A43AA8312E700BF001000E00400001019
:10A200003F801CF0E81800202DE9F04FDFF80CB17A
:10A210009BF8004087B024B90124204607B0BDE870
:10A22000F08F3B4ED6F8C85511F0E8FC9BF860392A
:10A230000390002B00F0DE82364AA2FB0532364B3B
:10A240005209A3FB0213DB0803EB8303A2EB4303D6
:10A25000DAB204920BF2146202EB830300930BF266
:10A260000C53019206F1E00402930027DBF8283931
:10A27000039AD31A04D454F8082C9342C0F26A8289
:10A28000234A54F858AC256ADAF800608C2303FBA3
:10A29000072393F8D430002B40F09681284644F0F1
:10A2A0006DFC1B4A8C2303FB0723002283F8D42078
:10A2B0009AF805100C2914D8DFE811F07801130082
:10A2C0001300130071011300130013007F0113002A
:10A2D000130013000D00B38B23F400631B041B0C4D
:10A2E000B3832246304615F033F89AF805300C2B2C
:10A2F0001ED8DFE813F04B011D001D001D004201B8
:10A300001D001D001D0039011D001D001D00150050
:10A31000E81800201F85EB51CDCCCCCC04000010F8
:10A32000B38B23F400631B041B0C43F40063B3835F
:10A33000019B54F8342C54F8101C5C330193009B9F
:10A340005C330093029B1433029354F8483C43F06F
:10A350004003134354F8302C134354F82C2C13436C
:10A3600054F8282C134354F8242C134354F8202C6D
:10A370001343402244F83C2C54F8142C13432A680D
:10A3800022F07E6222F45F3222F470720B43134398
:10A390002B6054E907316A690B4322F0070213432B
:10A3A0006B6154F8383C6B6054F8443CAB6054F833
:10A3B000403CEB602B6843F010032B609BF8603946
:10A3C00001379F4204F18C04FFF650AF01220021B7
:10A3D0008BF81226CBF82819002B3FF41DAF9D48AF
:10A3E00090F89010890700F1A081D0F888100868D3
:10A3F00049798A40018C92B289B221EA0201018432
:10A40000018C89B20A43012B02843FF405AF9149C4
:10A4100091F81C21970700F1A281D1F8142110684E
:10A420005479018C012289B2A24092B221EA020140
:10A430000184018C89B20A43022B02843FF4ECAE02
:10A44000844991F8A821960700F1A281D1F8A021B2
:10A4500010685479018C012289B2A24092B221EA9B
:10A4600002010184018C89B20A43032B02843FF468
:10A47000D3AE784991F83422950700F19281D1F852
:10A480002C2210685479018C012289B2A24092B228
:10A4900021EA02010184018C89B20A43042B02845F
:10A4A0003FF4BAAE6B4991F8C022940700F1828163
:10A4B000D1F8B82210685479018C012289B2A240E7
:10A4C00092B221EA02010184018C89B20A43052B70
:10A4D00002843FF4A1AE5F4991F84C23900700F14C
:10A4E0007281D1F8442310685479018C012289B219
:10A4F000A24092B221EA02010184018C89B20A438E
:10A50000062B02843FF488AE524991F8D823920773
:10A5100000F16281D1F8D02310685479018C0122B6
:10A5200089B2A24092B221EA02010184018C89B26F
:10A530000A43082B02847FF46FAE464A92F86434D3
:10A540009B0740F15281D2F85C24042311685079B2
:10A550000A8C83409BB292B222EA03020A840A8CDC
:10A5600092B213430B8457E6B38B23F008031B040A
:10A570001B0C43F00803B383DAE6338B23F4006348
:10A580001B041B0C43F400633383D1E6338B23F0AD
:10A5900008031B041B0C43F008033383C8E6338B0A
:10A5A00023F400631B041B0C33839AE6338B23F0E4
:10A5B00008031B041B0C338393E6B38B23F00803BF
:10A5C0001B041B0CB3838CE66B6834F8542C1FFA05
:10A5D00083F8B389C8F116089BB223EA0203B8F1E5
:10A5E000070FB3817FF65AAEDBF814350133CBF891
:10A5F0001435A36A05939E4600225EF804CB012120
:10A60000914660461DE0DEF800C0B9F1140FACEBD6
:10A61000000321DC13F1080048BF03F11700031108
:10A6200009EB2019604603F1FF3C013102FA03F304
:10A63000012202FA0CF2884542EA03020EF1040EEE
:10A640000AD38845DFD8C9F11503DEF800004FF0C2
:10A650001509E8E7E8180020B9F1150F5CD1684842
:10A66000C2F38423C2F3441100EB830300EB8101A6
:10A67000D3F8F830D1F8F8101B0243EA011302F0C6
:10A680001F0100EB8101C2F3C43200EB8202D1F85A
:10A69000F810D2F8F8200B4343EA023383EA13227E
:10A6A00082EA121202F00F020F2A35D1C3F30F1300
:10A6B0004FF6FF7293422FD0B3F5606F58D0029AD5
:10A6C00093810198049990F858208A4210D0009AFA
:10A6D00091680268521A00990260096B4268521A26
:10A6E0000099426000228A600A63049980F8581039
:10A6F000019900980A6801320A608268013282601A
:10A700004FF6FF7293427FF4C9AD4B6801334B6043
:10A71000036B01330363C1E5DBF810350133CBF87C
:10A7200010356FB14FF6FF73CBE7364AD2F8882069
:10A7300010685479018C0422A24089B292B25CE67E
:10A740000599314858224DF04DFFDAF800604FF678
:10A75000FF73B6E70024204607B0BDE8F08F294A12
:10A76000D2F8142110685479018C042289B25BE676
:10A77000244991F8E12402EB420201EBC2023A447F
:10A7800092F8F1240D2A9AD1029980228A7798E7CB
:10A790001C4AD2F8A02110685479018C042289B295
:10A7A0005BE6184AD2F82C2210685479018C0422F6
:10A7B00089B26BE6134AD2F8B82210685479018C3A
:10A7C000042289B27BE60F4AD2F8442310685479F8
:10A7D000018C042289B28BE60A4AD2F8D023106891
:10A7E0005479018C042289B29BE6064BD3F85C2491
:10A7F0000123ABE601228BF81226CBF828390CE5B1
:10A8000050870508E8180020BC050010F8B590F83E
:10A8100071301C09013C052C0FD8184E06EB440280
:10A820000546B2F8780103F00F0340FA03F2D207AD
:10A8300003D595F87C70012F01D00120F8BD07FAEF
:10A8400003F3013B184034444CF078FA94F8842127
:10A850000B4C104454F8302004EBC0041069A3885A
:10A860001840EBD0EB6E002285F87C20204693F850
:10A870002120022110F0BAF83846F8BD50870508AB
:10A880008422002038B500224E2105460FF060F9E1
:10A890001524962013F0ECFBF52128460FF08EF9D5
:10A8A000422807D0472807D0013C14F0FF04F0D11C
:10A8B000204638BD0C24FBE70D24F9E72DE9F743CA
:10A8C000064600F1100490480EF0B0FFB08296F8F2
:10A8D000210144F23B33A6F84C31A0B30709013FF4
:10A8E000052F00F00F0000F2E680DFF8348208EB5D
:10A8F0004703B3F8782142FA00F515F001050FD0AF
:10A90000012303FA00F00138104047444CF016FAD6
:10A9100097F884317D4D184405EBC0052623EB8064
:10A9200031467B4B41F80C3F284649F01FFD55B19D
:10A93000AB88B3FA83F24FF00043D34003D075499C
:10A940000A6813430B6042F21F53A6F84C310022F1
:10A95000762120460FF0FCF800224E2120460FF011
:10A96000F7F896F8D8906C4BB9F10C0F93F89D3C22
:10A9700040F0A380012B00F0B080022B15BF06250C
:10A9800003254FF4DC774FF4786714BF4FF01508B8
:10A990004FF03F080122762120460FF0D9F84246B9
:10A9A0000C2120460FF0D4F807F0FC020D212046C0
:10A9B0000FF0CEF82A0142EA17220E2120460FF0AE
:10A9C000C7F8B9F10C0F14BF4FF006084FF0150887
:10A9D0004FF002024FF07601204615BF24274FF4B6
:10A9E000DC770A2506250FF0B3F84FEA4802032169
:10A9F00020460FF0ADF807F0BC02042120460FF00E
:10AA0000A7F82A0142EA1722052120460FF0A0F8F4
:10AA10000022762120460FF09BF8FF22522120468B
:10AA20000FF096F80322142120460FF091F800222F
:10AA3000632120460FF08CF80822652120460FF094
:10AA400087F8E42120460FF0B9F800F0EF0040F05D
:10AA50006002642120460FF07BF80F224E21204631
:10AA60000FF076F8012013F003FB96F8DB30002B93
:10AA700045D096F82031013343F00103B3FA83F354
:10AA8000C3F11F03032B3ADC244AD25C02F00F020D
:10AA90004F21204601920FF05BF80F2013F0E8FAE7
:10AAA0002046019A50210FF053F80F2003B0BDE863
:10AAB000F04313F0DDBA002532E7022B13D0032B4D
:10AAC00017D0012B15BF0A2508252427902714BF6E
:10AAD0004FF006084FF00C085CE704254FF4C06700
:10AAE0004FF0270856E706254FF4DC774FF015089E
:10AAF00050E704254FF4AC674FF025084AE70023E0
:10AB000086F8DB300622C1E700366E018422002081
:10AB1000E18B0008003C0140E818002048FF0508D0
:10AB2000508705082DE9F047089F88461546002103
:10AB3000202204461E464DF0B8FD4FB13B68E3812C
:10AB40001B0C23827B687A89E3821B0C628223833D
:10AB500040464BF045FCEB0619D4431EB8B108EB58
:10AB6000000701E0013B12D317F801CDBCF12E0F15
:10AB7000F8D1C01A421E032AA8BF0322082B03F1F2
:10AB8000010AA8BF08239146C2441A4606E00828D5
:10AB90000246C246A8BF08224FF000094FF02033FA
:10ABA00041462360636004F1080720464DF01AFD1A
:10ABB000174B23815146BB704A4638464DF012FD73
:10ABC000611EE31D11F801CFACF1610EBEF1190F4A
:10ABD0009CBFACF1200C81F800C08B42F2D138460A
:10ABE00004F10B0110F8013BA3F16102192A9CBF8B
:10ABF000203B00F8013C8842F4D118232373330C26
:10AC0000A382E572099B6683E361BDE8F08700BF1C
:10AC1000202020000A4608B5054920B9054844F01F
:10AC200069FA034808BD044844F064FA004808BDC6
:10AC3000A82500201CFE050844FE050810B5044C9C
:10AC400004480A46214644F055FA204610BD00BF8C
:10AC5000A82500206CFE050810B5044C04480A46DF
:10AC6000214644F047FA204610BD00BFA825002029
:10AC700080FE050810B5044C04480A46214644F0FD
:10AC800039FA204610BD00BFA82500208CFE05081B
:10AC90002DE9F04FDFF88894D9F8C805C9F8CC053C
:10ACA00087B0002B00F0DA8001F5FE781344DFF85E
:10ACB00074B40393164601F12007C24621E0002E2A
:10ACC00064D0D9F8FC35B34200F0CC80D9F8F8351F
:10ACD000B34200F0FF80D9F80036D9F80416B34229
:10ACE0004BD8B14200F29981711A204647F088FC96
:10ACF000039B01369E4207F500770AF5007A00F0C3
:10AD0000AD80D9F80856B542A7F12004D7D8751BF5
:10AD1000D9F8188605F00702EB080492D8F830201D
:10AD20000233934203D3D8F8382093420BD94146DB
:10AD30001846059347F034FC059B8046002800F038
:10AD40008C81C9F8180698F80420002A40F0348154
:10AD5000D8F82850002D00F07981D8F830209B1ABF
:10AD6000049A02EBC303D8F80C20204602EB4322DE
:10AD70004FF400714346A847BAE7B142B4D9204620
:10AD80004FF4007200214DF090FCB1E74FF40072D7
:10AD9000314620464DF089FC802387F89E310C23F4
:10ADA00087F8A231D9F8F835D44AD9F8F015C4F8A3
:10ADB000C6319342C4F8CA1100F33481D04AD14C51
:10ADC00082FB03021A44D817C0EB621284FB0254C0
:10ADD000CD4D85FB03C5C0EB2530C2EB821587F84E
:10ADE000A1015B1B801020F03F000133034314449A
:10ADF00087F8A031D317C3EBE4142244BF4B87F884
:10AE00009F214A1E9A4200F31981BD4BBD4883FB26
:10AE100002311144D317C3EB611180FB0140BA4CDE
:10AE200084FB0254C3EB2433C1EB811487F8A531B2
:10AE3000121B9B1023F03F0301321343084487F891
:10AE4000A431CB17C3EBE010014487F8A3115523BD
:10AE500087F8DE31AA2387F8DF3149E7002007B001
:10AE6000BDE8F08F4FF0FF3384F8EC3184F8ED311A
:10AE700084F8EE3184F8EF31D9F81036C4F8E831AF
:10AE80005223237063706123A37084F8E731412358
:10AE90000025E37084F8E631722384F8E43184F805
:10AEA000E5314FF4F0722946A7F11C004DF0FDFB8F
:10AEB0005523C7F8D051C7F8D451C7F8D85184F8F2
:10AEC000FE316FF0550384F8FC5184F8FD5184F88D
:10AED000FF310DE700214FF4007220464DF0E5FBF5
:10AEE0008A4A03CA47F81D0CEB2007F8200C5820AB
:10AEF00007F81F0C902047F8191C07F81E0C0023B8
:10AF000002220821F820E372227307F8131CA273AF
:10AF1000E37307F8102C07F80B0CD9F8F80584F840
:10AF20002C20D9F8F0256376121A2262D9F800068F
:10AF3000D9F80426E376121A3F2020764FF0FF302E
:10AF4000A0763E20207701206377A377E37784F80B
:10AF50002D3084F82E3084F82F30626284F830006F
:10AF600084F8313087F82610802187F820102921B5
:10AF700087F82210942187F823100E2187F82410D7
:10AF80000D21634A87F82510552187F8DE11AA2183
:10AF900087F8DF1103CA5F4BC7F82700C7F82B10EB
:10AFA00003CB1388A7F82F309378C7F83200C7F87F
:10AFB000361087F831309BE64FF4007200212046AE
:10AFC0004DF073FB049B002B4ED1D8F84030002B82
:10AFD00000F0AA80049AD8F830304F49CDE9002219
:10AFE00020461122FFF79EFDD8F840301A6C002A47
:10AFF00000F0AD80049A1B6BCDE900224749112275
:10B000003846FFF78FFDD8F8448007F120044FF44D
:10B01000E075B8F1000F3FD16AE6F11A204647F01B
:10B02000EFFA65E6FF2387F89F3187F8A13187F8AB
:10B03000A031324B4A1E9A427FF7E7AEFF2387F8D2
:10B04000A33187F8A53187F8A43100E729462046C7
:10B050004FF400724DF029FB4AE6A7F1240343F8B0
:10B0600004BF9A45FBD143E6D8F84030049AD8F89B
:10B070004480002B0CBF01230223C3EB021543467F
:10B08000002B3FF435AE013D9B6CF9D198464FF44F
:10B090000075002B3FF42CAE254420342346203588
:10B0A0004446049698460EE05CF81C1B236BCDF8D2
:10B0B00000C000260196FFF735FDA46C08F12008BA
:10B0C000CCB1A84517D02379A44604F11C0E112257
:10B0D000A8F12000002BE7D162792669236B216853
:10B0E00042F02102CDE900E6FFF71CFDA46C08F157
:10B0F0002008002CE5D1049EFAE500BFFF03FB0009
:10B10000832008828180808097554541A4FE0508F0
:10B11000B0FE0508BCFE05089CFE0508A0FE05085B
:10B12000E8180020DEADBEEF049BD9F8F415CDE998
:10B13000003320460822FFF7F5FCD8F84480B8F128
:10B14000000F3FF4D5AD3C464FF4F075A4E7049BE7
:10B15000CDE9003352E700BFBFF34F8F0549064BDF
:10B16000CA6802F4E0621343CB60BFF34F8F00BFA5
:10B17000FDE700BF00ED00E00400FA051648174A9D
:10B18000174938B5174C184D121A4DF02BFAD4F850
:10B190008820164B164842F47002C4F888201A68BA
:10B1A000002142F001021A6099601A6822F084724C
:10B1B00022F480321A6058601A6822F480221A60E1
:10B1C0000C4AD960521B28460B494DF00BFAA5607A
:10B1D000BDE83840FCF714BF000000100400001068
:10B1E00089A8060800ED00E00000002000380240B9
:10B1F000103000248801002000000008F8B5CB784A
:10B2000013B900252846F8BD00F110070C46064684
:10B21000897838460EF040FB05460028F1D0E078EA
:10B220000FF078FEB06123780133DBB210B1C37147
:10B230002223837109210FF055F8B0690EF026FB27
:10B240000C4AD2F8C835632BFBD90B480EF0EEFA46
:10B25000B0823846FFF716FB074620B9E0780FF0BA
:10B26000B9FE3D46CEE7306986F8D8704AF07AFEDE
:10B27000C8E700BFE818002040420F0043680B4AAF
:10B2800023F0407323F4807343F480734360836836
:10B290001A4042F002028260C36A0139CAB223F442
:10B2A000700141EA0251C162704700BFFDF7FFC063
:10B2B000704700BF0020FCF7FBBE00BF0120FCF779
:10B2C000F7BE00BF0220FCF7F3BE00BF431C00F036
:10B2D00038812DE9F04FDFF898A300EB80030AEBEB
:10B2E000C30287B0D2F80480810005460191DB00DB
:10B2F000B8F1000F04D0D468002C4CD0A17911B162
:10B3000007B0BDE8F08FD2F81090B9F1000F00F04F
:10B31000478199F80620002AF2D118330AF1040671
:10B32000F018D8F80470F250691CC0E90122152306
:10B33000C260C9B2A3711623E17189F8063089F899
:10B34000071098F8180048F07BFDBB88A28823F40A
:10B3500040731B041B0CBB8023681A83D9F8003090
:10B36000B9F804201A83112120460EF0BBFF1121E9
:10B3700048460EF0B7FF09264FF0330B24B1226880
:10B38000A188106901422DD1BBF1010B00F0D380DF
:10B3900048F090FFF2E7D2F81090B9F1000F00F0FA
:10B3A000E88099F80620002AAAD118330AF104018E
:10B3B000CA18D8F80470CC50C2E901441623D460EE
:10B3C00089F806306B1C89F8073098F8180048F0A7
:10B3D00037FDBB8823F440731B041B0CBB80BDE707
:10B3E0002268A188518348F009FF2368A2881A8344
:10B3F00048F004FF013EBFD1002C00F0EF8023682D
:10B40000A2885A8348F0FAFEB9F1000F00F00B81D0
:10B41000D9F80030B9F804205A8348F0EFFE2368C9
:10B42000A2881A8348F0EAFED9F80030B9F804205F
:10B430001A83019B20465C190AEBC404A37D227D7C
:10B44000002B14BF322112210EF006F8A37D627D7D
:10B45000002B14BF3221122148460DF0FDFF7E4B18
:10B460009F4200F0CA807D4B9F4200F0D1807C4B10
:10B470009F4200F0E080019B2B440AEBC30A4FF48B
:10B480007A73BAF8184003FB04F4BB8823F44073C2
:10B490001B041B0CBB803B889BB243F001033B8029
:10B4A000BD8802A843F01CFB25F03F0504986D4BB6
:10B4B0002D04A3FB00232D0C45EA9345BD803A885B
:10B4C00022F001021204120C3A80674A990C94424D
:10B4D0000B4637DC6200B0FBF2F292B20133042A71
:10B4E00038BF04223B84BA833B889BB243F00103FC
:10B4F0003B803B8823F4816323F002031B041B0C75
:10B500004FF4804143F480633B8039813B8823F0D2
:10B5100080031B041B0C00223B8098F81A00114684
:10B5200047F0E4FA002298F81900114607B0BDE888
:10B53000F04F47F0DBBA002C7FF452AF48F05EFECC
:10B5400056E7704704EB4404B0FBF4F082B2C0F35A
:10B550000B0008B942F001024FF4967301FB03F3AC
:10B560004249A1FB03139B09013342F400423B848F
:10B57000B9E718330AF10401CA18D8F8047041F881
:10B580000390C2E90199C2F80C9098F8180048F0AD
:10B5900057FCBB8823F440731B041B0CBB80E2E602
:10B5A00018330AF10401CA18D8F8047041F803905E
:10B5B000C2E901991523C2F80C90A3716B1CE371C9
:10B5C00098F8180048F03CFCBB88A28823F440732C
:10B5D0001B041B0CBB8023681A83C4E648F00EFED4
:10B5E000B9F1000F32D0D9F80030B9F804205A83ED
:10B5F00048F004FE48F002FE16E703F5F2331A6A3B
:10B6000042F400121A621A6A22F400121A6232E735
:10B6100003F5F0331A6A42F480021A621A6A22F4BD
:10B6200080021A6227E748F0E9FD2368A2881A839E
:10B6300048F0E4FDFDE603F5EE331A6A42F4000239
:10B640001A621A6A22F400021A6214E748F0D6FD60
:10B6500048F0D4FDEDE600BF005400400058004023
:10B66000005C004083DE1B43A0860100D34D6210C6
:10B67000E81800202DE9F843074610F091FADFF8AA
:10B680004C8007EB8709044608EBC90542F20F76A8
:10B6900004E010F085FA031BB3420ADC6B7F002B39
:10B6A000F7D108EBC90898F81C0080F00100BDE84C
:10B6B000F883B8F8C03D013338469BB2A8F8C03DC6
:10B6C000FFF704FE0020BDE8F88300BFE818002063
:10B6D00070B5284D00EB800305EBC30384B05A68B6
:10B6E0005468A28A92B20392039A12F4706F1CBF3C
:10B6F00001221A77039B13F4E06F4FEA80060CD106
:10B70000A38A304423F4706305EBC0051B041B0CB3
:10B710000022A3826A7704B070BD238BA38823F430
:10B7200080631B041B0CA380039B9A05E8D4238829
:10B730009B05E5D42388D9050FD52388DA05FCD4E9
:10B7400023889BB243F40073238023889B05FCD499
:10B750000190FFF7BBFD0198D2E723889BB243F429
:10B7600000732380A38823F440731B041B0CA38065
:10B77000C6E700BFE81800200020A9E70120A7E7DE
:10B780000220A5E72DE9F84F304F00EB800407EBCE
:10B79000C404D4F80880B8F1000F04D09A46637F3F
:10B7A00003F0FF0923B14FF000094846BDE8F88FC8
:10B7B0000E469346054610F0F3F90A9B7600F6B262
:10B7C000C4E909330123A67784F81FB084F82190D7
:10B7D00084F8223084F820A0637784F81C90B8F8AD
:10B7E00004209105064622D4B8F80030DA0512D4B8
:10B7F00042F20F7404E010F0D3F9831BA3421ADC69
:10B80000B8F800309B05F6D4B8F800309BB243F48A
:10B810008073A8F80030B8F804309BB24FF00109EB
:10B8200043F44073A8F804304846BDE8F88F9946C1
:10B830004846BDE8F88FB7F8C03D01339BB22846B3
:10B84000A7F8C03DFFF742FDAFE700BFE8180020B2
:10B8500010B503681C78012C82B00AD0022C05D1E7
:10B860005A6A0AB1904201D11B6A03B3012002B0A7
:10B8700010BD93F904C012490CEB8C0301EBC30318
:10B880005B7F03F0FF0213B1002002B010BDBCF1DA
:10B89000FF3FEBD0BCF1020F10DC01F5A963017989
:10B8A000009360460623FFF76DFF2046DFE7054A59
:10B8B000062380210EF090F80120D8E72046D6E735
:10B8C000E8180020301E0020F8B5774C04EB001675
:10B8D000D6F8C43D002B00F094800546070196F889
:10B8E000CC0D48F0ADFA96F8CC3D590903F01F0293
:10B8F00003294FF0010303FA02F300F098800429B2
:10B9000000F0858002297DD0E319013593F8C80D38
:10B910000FF000FBEDB2064610B112238371C57122
:10B92000E31993F8C90D0FF0F5FA10B11323C5719F
:10B930008371E31993F8CA0D0FF0ECFA10B11423D8
:10B94000C57183713C444A2194F8CB2D30460DF0EB
:10B9500083FD94F8C90D0FF0DDFA94F8CB2D2A2160
:10B960000DF07AFD94F8CA0D0FF0D4FA94F8CB2DAF
:10B970000A210DF071FDD4F8C42D4C4B9A425BD0D6
:10B980004B4B9A4248D04B4B9A4260D04A4B9A421A
:10B9900068D04A4B9A4270D0494B9A4278D0494974
:10B9A0009088B1F8DE40B1F8DC30B1F8E6502343BE
:10B9B000B1F8E0402343B1F8E24020F00300234314
:10B9C000B1F8E4400004000C2343B1F8E840908053
:10B9D0002B4310882343B1F8EA40B1F8EC1000F48F
:10B9E0004150234303439BB21380938B23F40063A2
:10B9F0001B041B0C9383118213889BB243F04003FA
:10BA00001380F8BD304A516A0B4353627CE72E4ADB
:10BA100011690B43136177E703F50033196A41F4A9
:10BA200080411962196A21F480411962B7E7264AF8
:10BA3000116A0B43136267E703F58433596A41F4D3
:10BA400080515962596A21F480515962A7E703F580
:10BA5000FE33196A41F400411962196A21F4004168
:10BA600019629CE703F58233596A41F40051596227
:10BA7000596A21F40051596291E703F56843596A04
:10BA800041F480115962596A21F48011596286E7A4
:10BA900003F56443596A41F400115962596A21F46B
:10BAA000001159627BE700BFE81800200030014018
:10BAB00000380040003C004000340140005001408C
:10BAC00000540140880100200038024010B404698D
:10BAD0008269E468416814604024D46044690023AA
:10BAE0000C31C2E90433C2E90633C2E90833C2E9C2
:10BAF0000A33C2E90C3393609363516084B1C26925
:10BB0000E0689363C2E90233C2E90433C2E9063351
:10BB1000C2E90833C2E90A33C2E90C33C2E90001C1
:10BB20005DF8044B704700BF436800221A60037D34
:10BB30001F2B08D9203B2022016802FA03F343F0AF
:10BB40001803CB6070472022016802FA03F343F028
:10BB500018038B60704700BF0268136A11B1D9697E
:10BB600001B3143330B49C681D689169DDB14FF4A2
:10BB7000806088618D60104640690C6180B15968B1
:10BB8000D369C9B10A464FF480619A609961224332
:10BB900012F0010F14BF00224FF400521A621C6110
:10BBA00030BC704770478D61054D4FF0FF0C05F8B4
:10BBB000EECF00688D60DFE7024A9A609961E6E7A0
:10BBC00088010020DC2600200168F8B5D1E90423B3
:10BBD00004465568002B49D09861107D5E681F2887
:10BBE00031D81768202202FA00F040F01800B8603F
:10BBF0001A7D1F2A32D91868203A202303FA02F24C
:10BC000042F01802C26000232B60336033688969F8
:10BC100043F010033360284643F046F8236830466B
:10BC2000D96943F041F82B68226843F001032B6087
:10BC30003368526843F00103336093889BB243F04A
:10BC400003039380F8BD17682038202202FA00F021
:10BC500040F01800F8601A7D1F2ACCD818682023FD
:10BC600003FA02F242F018028260CCE7137D906181
:10BC70001F2B1CD81068202202FA03F343F018038C
:10BC8000836000232B602B68896943F010032B60CD
:10BC9000284643F009F82B68226843F001035268F4
:10BCA0002B6093889BB243F002039380F8BD106829
:10BCB000203B202202FA03F343F01803C360E0E7BD
:10BCC0002DE9F843DFF800927D4F0646356896F877
:10BCD00088806B68B088012285F828201A8822F0B5
:10BCE00040021204120C1A802A89824223D0198839
:10BCF00021F0380109044B454FEA114100F0BC80A6
:10BD0000704A934200F0B8800246B2F5807FA8BF27
:10BD10004FF48072022AB8BF0222002A92FAA2F2DD
:10BD2000B2FA82F208BF4FF0FF32013A41EAC20292
:10BD300092B21A802881317BAA7A8A420CD01A8862
:10BD400022F003021204120C1A801A8892B20029FF
:10BD500000F08F801A80A9721A8892B242F04002D5
:10BD60001A802A6A9168002900F0A0804FF0000C28
:10BD70001432E64652F8100C8E4400EA070120B156
:10BD8000B1F1805F23D0696909B352F8140C143201
:10BD900000EA070110B1B1F1805F18D052F80C1C15
:10BDA0000CF1010C0029E5D12A7B82B1B8F1000F1A
:10BDB0000DD0BCF1010F6CD8BEF1070F69D80CEBA8
:10BDC0008C0189002A6A11440A7B002A61D02A6A00
:10BDD0009268002A52D000220AB1127B22B1B268C6
:10BDE00012B1116892884A832A6A14682A6A5168D3
:10BDF0002A6A9268501E9AB12CB3224612F801CBDF
:10BE000014461A899207FCD5A3F80CC01A89D207E8
:10BE1000FCD59A8992B209B101F8012B0138EBD215
:10BE20002B6A1B7BF3B92B6A1B6993B12B6AD6F87B
:10BE300094001B699847012808D0022809D10023E3
:10BE40002B62BDE8F8834FF0FF0CDAE72B6A143B56
:10BE50002B622A6A2B6A14332B622B6A9B686BB1A4
:10BE60006B68B9E7B368002BDDD01A689B88138331
:10BE7000D9E742F003026DE7420846E72B6A1B68E8
:10BE8000DBB12B6AD3E900622A620022C3E90022F7
:10BE90001CE700213046FFF75FFEB36813B11A6854
:10BEA0009B8853833046BDE8F8438DE62A7B002A01
:10BEB0008DD0B8F1000F85D189E72B62C1E700BFB3
:10BEC0000000FFFF003C0040003800400348D0F86D
:10BED00000310BB1F0301847704700BF88010020D7
:10BEE0000348D0F8243113B100F58A701847704721
:10BEF000880100200348D0F8483113B100F59C7048
:10BF000018477047880100200348D0F86C3113B1FE
:10BF100000F5AE7018477047880100200348D0F83C
:10BF2000903113B100F5C0701847704788010020A8
:10BF30000348D0F8B43113B100F5D27018477047F8
:10BF4000880100200348D0F8D83113B100F5E4701F
:10BF500018477047880100200348D0F8FC3113B11E
:10BF600000F5F67018477047880100200348D0F8A4
:10BF7000203213B100F50470184770478801002083
:10BF80000348D0F8443213B100F50D7018477047DC
:10BF9000880100200348D0F8683213B100F516700C
:10BFA00018477047880100200348D0F88C3213B13D
:10BFB00000F51F7018477047880100200348D0F82B
:10BFC000B03213B100F5287018477047880100207F
:10BFD0000348D0F8D43213B100F5317018477047D8
:10BFE000880100200348D0F8F83213B100F53A7008
:10BFF00018477047880100200348D0F81C3313B15C
:10C0000000F543701847704788010020094B0A4A21
:10C01000013800EBC00003EB8000116BD0F8F0306A
:10C02000064883420CBF4FF400134FF480030B43C8
:10C03000136370478801002000380240006002400E
:10C0400070B501383C4C3D4D00EBC00C04EB8C0C42
:10C050009646DCF8F0603A4AAE420CBF4FF4001549
:10C060004FF48005166B35431563CCF80011CCF8FE
:10C0700008313449DCF8F4308B424FEAC0023ED03C
:10C0800001F580618B423AD0A1F57A718B4247D09D
:10C0900001F580618B4243D0A1F57A718B4241D08A
:10C0A00001F580618B423DD0A1F57A718B4235D08C
:10C0B00001F580618B4231D0A1F57A718B4233D08A
:10C0C00001F580618B422FD0A1F57A718B422DD082
:10C0D00001F580618B4229D0A1F57A718B4227D07E
:10C0E00001F580618B4223D0A1F57A718B4221D07A
:10C0F000154D01F580618B4218BF002500E0134DFE
:10C10000104404EB8003CEF38711C3F8105193F869
:10C110000501BDE87040002246F0E8BC0C4DEFE799
:10C120000C4DEDE70C4DEBE70C4DE9E70C4DE7E767
:10C130000C4DE5E7044DE3E7880100200060024074
:10C14000003802401060024000800028208000106B
:10C15000008000180088001000802010208000203F
:10C1600000880020008020202DE9F04FA24BDFF84E
:10C17000A89293F80A3EA14F8DB0CDE90139013B59
:10C18000DBB200939E4B0025A3F2D466DFF88CB29D
:10C19000DFF88CA25B46D3469A464FEA9A23A3F572
:10C1A0008013522B4CD8334493F88C310D2B47D845
:10C1B000FC56019B012B40F0FE80012C35D14FF045
:10C1C00000084146204612F065FC12F003FD03789A
:10C1D00013B1542B40F0098108F104081FFA88F8C4
:10C1E000B8F1100FEDD14FF0000E8DB3494600208D
:10C1F0000CE0334493F88C310D2B0ED8FB56A34240
:10C200000ED00130A84201F580711EDA8A681368E9
:10C210009B0AA3F58013522BEBD90023A342F0D144
:10C2200053799BF805209A42EBD1754B9B454BD037
:10C230005BF820AF4FEA9A23A3F58013522BB2D9B3
:10C24000009B012BF1D90024B9E7BEF1000FECD11E
:10C2500058460DF02DFFC3B2022B9BF805C000F22B
:10C260003C83431C5BB203EB43034FEA830E654BF5
:10C27000654903F5727004E0834200F02E8353F8A1
:10C280002C1F5145F8D11A796245F5D153F80E406B
:10C29000002CF1D05D4800234268A24203F1010363
:10C2A00000F08680102B00F12400F5D14FF0FF3311
:10C2B000574A03EBC30302EB830393F80C31002BC3
:10C2C000B3D1029BC3F808B0029B013503F580731C
:10C2D000042D02937FF45AAFDFF848A10AF29C5371
:10C2E0004FF0010800934B4BD3F8082508F1FF33BA
:10C2F0009A425ADDDAF80C50002D00F0EA822968E3
:10C30000AE8801F13F41B6FA86F601F57E01C6F12D
:10C310001F06890A3F4B5F68002F40F38780002388
:10C3200002E00133BB427FD01C0259F804208A424C
:10C33000F7D14C44CAF80460CAF818405FFA88F391
:10C3400015B1EB710323AB71636CE16C72000320D8
:10C35000904003436364012303FA02F20A43E26458
:10C360002C4A127872B3226DB3401A43226515B17C
:10C370002A68A9881183D4F8A00099B20122FCF799
:10C3800047F82046FCF79AF9009A012308F10108C2
:10C390008AF81C308AF81D305374B8F1090F02F185
:10C3A00018030AF1200A00939DD10DB0BDE8F08F6B
:10C3B000DBB2013B7CE7022B7FF401AF082C3FF49A
:10C3C000FEAE32E7226D06F110018B401343236568
:10C3D00015B12B68AA885A830121B140D4F8A00076
:10C3E00089B20022FCF714F8CBE74FF0010E002DC4
:10C3F0007FF4FCAE19E700BFE818002050FF0508E5
:10C40000248E0508308905080000014078020020CC
:10C4100088010020040000100C00001000040140FE
:10C42000248D05080C040010032B61DCA64B03EBE4
:10C4300007233A0218690192002800F043829960AC
:10C440000131CAB283F8052102929F4AD0F800B0A8
:10C4500001375760542283F8042144790DF028FEF7
:10C460009A4AC3B292F81FCE9AF810200392022B78
:10C4700000F23382471C7FB207EB4707944A954985
:10C48000BF00002305E00133172B00F0268252F88D
:10C490002C1F8B45F7D11179A142F4D1D159002934
:10C4A000F1D02C2200EB400002FB03F38A4A03EB9D
:10C4B000800313440198D3F8F021834B0344C3E96C
:10C4C0000612864B00221F4618464368994220D028
:10C4D0000132102A00F12400F7D1814B93F8E820B3
:10C4E00052B9542283F8E820029A83F8E92003E045
:10C4F000764A032382F81E3E73487A497A4A7B4B78
:10C50000C0F88C19C0F88429C0F894390DB0BDE882
:10C51000F08F531CDBB2724A0597013B03EBC30358
:10C5200002EB830393F80C210492002AE4D1019FCB
:10C53000029A83F80D21FA116D4802EB2722542448
:10C5400002EB021200EB82028C2183F80C41694855
:10C550002C683B1201FB03F300EB43005A4B3B44B6
:10C56000C3E93C01C3F8A8203322DC60C3F8AC2047
:10C57000614B9B4509EB070418D0564B9B4515D0E2
:10C5800003F580439B4511D003F580639B450DD097
:10C5900003F580639B4509D04C4B1A68BCF1060F2C
:10C5A0004FEA520207D15549554B0EE0474BBCF1BB
:10C5B000060F1A68F7D0534B53485449BCF1070F84
:10C5C00008BF1946524B08BF0346B2FBF3F33E4F78
:10C5D000B2FBF1F201995846013B07EB010B9BB20C
:10C5E000013AABF8B020ABF868305431A3650023B2
:10C5F0004944A4F85C30636542F0CCFCDBF810B031
:10C600004449DBF80000028892B242F080020280C6
:10C610000023ADF82030038807914FF48072022187
:10C6200023F00103CDE90A121B044FF00A0C1B0C86
:10C63000CDF824C003809BF8051007AA12F088FEED
:10C640009BF80400002840F025811F4B019A059FAC
:10C650009A1800231069D2F818C001680A8892B2AB
:10C6600042F001020A807A68944503F1010300F068
:10C670000D81102B07F12407F5D14FF0FF33184A35
:10C68000254FDFF89CC003EBC30302EB8303234A6F
:10C69000D3F8F030BB420CBF4FF400134FF48003CB
:10C6A000176B3B43136343790C2B9CBF0A4A02EB85
:10C6B0004303019A98BFB3F8F476034B134488BF41
:10C6C00000279F82002334E004000010E8180020B7
:10C6D00030890508000001405087050878020020D5
:10C6E00088010020517001084D700108597001083F
:10C6F00008270020382A002000040140882A110061
:10C70000A0BB0D001055220040771B004495080087
:10C71000D0DD0600600001000060024000380240E9
:10C72000FC080010914200F0D2800133042B00F08D
:10C73000D7805CF83320002AF4D16B4A1046D2F837
:10C74000F4280132C0F8F42800EBC302DB00C2F881
:10C75000F818634404989A88644917439F80624A92
:10C76000019BD71823469022FFF76AFCB86902683C
:10C77000002342F010020260C4E92533A367C4F825
:10C780008830C4F89C30FA6962664FF400310422A4
:10C79000C4E923124FF4806B4021C4F87CB02167B8
:10C7A000D7F8AC106167F968019B1831A1664FF4A6
:10C7B0008051C4F88010D7F8A820E26603F1640124
:10C7C0004FF480424944C4F8842042F06DFAB869BD
:10C7D000019BD0F800E0C4F81CE0D0F814E0C4F8E5
:10C7E00020E0D0F804E0C4F824E003F1AC01D0F874
:10C7F00008E0C4F828E00023D0F80CE0C4F82CE0EE
:10C80000C4E93733C4F8B830C4F8C030C4F8D03005
:10C81000C4F8E43004224FF4403CFB69C4F8AC3067
:10C82000C4E935C2C4F8C4B0D7F8F430C4F8BC3099
:10C83000FB681033C4F8B0304FF40063C4F8C8305C
:10C84000D7F8F030C4F8B4304FF480434944C4F80A
:10C85000CC3042F029FABA691168216351696163E9
:10C860005168A1639168E163D1682164116841F066
:10C8700010011160039A8AF810205FFA88F3CAF851
:10C880000460CAF80C50CAF818405AE5DBB20493A9
:10C89000013BF4E60EF03EFB029038B19BF8082015
:10C8A00002210EF0A3F8029B5422DA80DBF800206C
:10C8B000B2F844306FEA43436FEA53439BB2A2F8A5
:10C8C0004430C2E60A4A022382F81E3E14E6DB0028
:10C8D0003FE74FF0FF3631461CE500235B68FFDE83
:10C8E00000239B88FFDE00BF04000010598400086D
:10C8F000E8180020084B10B5D3F8B83418440C469B
:10C90000007E0EF007FB18B1036882880CB11A8311
:10C9100010BD5A83FCE700BFE02900200B4B10B587
:10C92000D3F8B83403440446187E0EF0F3FA58B135
:10C930002E228271621CC27101210DF0D3FC2046AF
:10C940000021BDE81040D5E710BD00BFE029002060
:10C950002DE9F04F8DB00E469DF858400194039399
:10C960000546002800F0D080DFF8D0C10779002309
:10C970000CF2BC4402E0152B00F0C68003EB43012F
:10C980000133605CB842F6D161442F6891F9BE84EE
:10C9900095F805E05FFA88F3022B00F2B58008F104
:10C9A000010C4FFA8CFC0CEB4C0C604B4FEA8C0CDE
:10C9B000002105E00131172903F12C0300F0A480C8
:10C9C00018688742F6D118797045F3D153F80C40B6
:10C9D000002CEFD02C2303FB01F108EB4808544B4B
:10C9E000DFF85CB101EB88011944D1F8F03105930F
:10C9F0009BF81C390093002B40F08B804D4FD7F8EB
:10CA0000F430A34200F0E482D7F818319C4200F0E1
:10CA1000CF84D7F83C31A34200F0CC84D7F8603102
:10CA2000A34200F0C984D7F884319C4200F0C68448
:10CA3000D7F8A831A34200F06584D7F8CC31A342DF
:10CA400000F0BE84D7F8F0319C4200F0BB84D7F8E8
:10CA50001432A34200F0BB84D7F83832A34200F06E
:10CA6000C284D7F85C329C4200F0BB84D7F8803295
:10CA7000A34200F0BA84D7F8A4329C4200F0BF84ED
:10CA8000D7F8C832A34200F0C184D7F8EC32A342F1
:10CA900000F0BA84D7F81033A34208BF0F2300F088
:10CAA000988200234FF0FF3A0693009B002B49D059
:10CAB0000AEBCA0207EB82024FEACA03079392F815
:10CAC0000C31392B00F02983D5F800804FEA9822E9
:10CAD000A2F58012522A00F29C8215490A4492F86B
:10CAE0008C210D2A00F295821349895CCBB9079AF3
:10CAF000524407EB820282F80D11392182F80C11A1
:10CB0000069A72B1009333E0DFF834B09BF81C3919
:10CB10003BB1D5E9054305931CB1012300936DE7B3
:10CB200031B300200DB0BDE8F08F00BF308905089B
:10CB3000508705088801002050FF0508E0290020E3
:10CB4000040000100AEBCA0307EB83034FEACA0193
:10CB5000079193F80C110029E3D1013283F80D21DC
:10CB6000032283F80C21069B002BDAD0D5F8008035
:10CB7000DFF86C939BF8183906EB8602C2EBC20211
:10CB800031B20B919100089109F1800101EB820211
:10CB90000992ABB3D9F8DC28424500F01584012B8B
:10CBA0002ED0D9F8F428904500F01884022B27D015
:10CBB000D9F80C29424500F01A84032B20D0D9F86B
:10CBC0002429424500F01D84042B19D0D9F83C29B2
:10CBD000424500F01D84052B12D0D9F85429424556
:10CBE00000F01984062B0BD0D9F86C29424500F0CF
:10CBF0001684072B04D0D9F88429424500F0848399
:10CC000003EB430209EBC2020293C2F8DC885A1C10
:10CC1000D2B28BF818291346013B0299AB4A049310
:10CC20008C2303FB069301EB410102EBC10183F866
:10CC30009160C3F88850C3F8041195F804C04FEA16
:10CC40001C13013B052B0CF00F0C00F25183A04983
:10CC50000A9301EB4300B0F878E14EFA0CF010F0C3
:10CC6000010012D0012000FA0CFC0CF1FF3C0CEA90
:10CC70000E004AF063F896490A9B944A0B44C0326E
:10CC800093F88431184402EBC000019A9BF80030FD
:10CC900002F00101013113B182F0010301938C23F1
:10CCA00003FB0693490141F00A01C3F894102A7A64
:10CCB0000CF0D2FB049B029A934200F07382039B18
:10CCC000063BDBB20A93089A82496032531807EE9A
:10CCD000903A8C2306FB03F303F1680C0A468C445C
:10CCE00009EB030100206033A1F8E400C1F8E8007B
:10CCF000CCE901004FF0600C42F803C0019B13F037
:10CD00000202089200F07881DB0003F00803A1F82A
:10CD1000EE300423A1F8F200A1F8E4308C2303FBE9
:10CD200006930021C3F8E8104FF00A0C68799BF8CD
:10CD30001C19A3F8F6C04FF0010CC3F8F8C04FF06F
:10CD4000020CA3F8F400A3F8FCC0002900F0D08185
:10CD5000D3F804319C602368CDED017A23F0010300
:10CD60002360204641F00AFF009BDDED017A002B95
:10CD700000F0AC818C2303FB06939BF81C09002771
:10CD8000C3E92677C3E92877C3E92A77C3E92C7773
:10CD9000C3E92E77C3E93077C3E93277C3F8D0709F
:10CDA000002800F06F81039A2968082A029A01F18D
:10CDB0004C00494902EBC20ED3F8042101EB4E119D
:10CDC0001161AA69C3F89820C3E927014FF0400117
:10CDD000C3F8A4104FF0040E4FF00301C3E93377FA
:10CDE000C3E931E10CBF06211221C3F8AC70C3F8CE
:10CDF000BC70C3F8A8104FF480624FF48051C3E9AF
:10CE00002C214FF48041C3F8B8104FF400310A9A36
:10CE1000C3F8C0108C2303FB0693022AC3F8004119
:10CE200000F2E58003990829294901EB820108BF36
:10CE30005F27D1F880072949B1FBF0F101F1230107
:10CE4000C3F8D81018BF13278C2101FB0691204688
:10CE5000D1F80431D1F888A09F80CDED037A0191FB
:10CE6000DAF8007041F08AFE0199DDED037A0023C3
:10CE700081F8D4309AF805100C2914D8DFE811F0A5
:10CE8000CB00130013001300F40013001300130071
:10CE9000ED001300130013000D00BB8B23F400639F
:10CEA0001B041B0CBB8317EE902A384612F050FA75
:10CEB0009AF805300C2B1DD8DFE803F0C61C1C1CAB
:10CEC000BD1C1C1CB41C1C1C140000BFC421002071
:10CED0005087050868190020DC2E002000D01213AE
:10CEE000E8180020BB8B23F400631B041B0C43F4E5
:10CEF0000063BB83099920688C2202FB06924023C1
:10CF00004B62D2F8A410D2F898300B43D2F8AC1090
:10CF10000B43D2F8B0100B43D2F8B4100B43D2F845
:10CF2000B8100B43D2F8BC100B43D2F8C0100B431F
:10CF3000D2F8CC100B43D2F8D0100B4393490140E8
:10CF40000B439BF81C092360D2E9313167690B431D
:10CF500027F007073B436361D2F8A8306360D2F83B
:10CF60009C30A360D2F8A030E360236843F0100344
:10CF7000236090B3009B83B3B8F800309BB243F0BA
:10CF80000103A8F80030B8F82020089B697992B214
:10CF90005BB304238B409BB222EA0302A8F8202053
:10CFA000B8F8202092B21343A8F82030029A049BCC
:10CFB000934200F0D2809BF80030002B5BD18C2391
:10CFC00003FB0696012086F88F000DB0BDE8F08FB8
:10CFD0000023591C06919A4667E592F8913006980D
:10CFE0006B499022FFF72CF8C6E70123D2E78D2189
:10CFF000C3F8D810132727E75B0003F00203A1F85A
:10D00000EC300123A1F8E2304FF48073A1F8F03046
:10D0100084E600216AE53B8B23F008031B041B0C0C
:10D020003B8340E7BB8B23F008031B041B0C43F03E
:10D030000803BB835EE73B8B23F400631B041B0CDC
:10D0400043F400633B8355E73B8B23F008031B0449
:10D050001B0C43F008033B834CE7BB8B23F0080316
:10D060001B041B0CBB831EE73B8B23F400631B04D8
:10D070001B0C3B8317E72B686A7934334FF6FF713B
:10D0800099509CE7059AC3F898200B9A4149C3F838
:10D09000D00002EB820702EB470701EBC701C3F8A0
:10D0A0000811C3F8A010C3E932004021C3F8A4104E
:10D0B0000421C3F8C41029686F79C3F8AC00343177
:10D0C0003944C3F89C10C3F8BC0094E6079B32496E
:10D0D0003248534407EB8307D7F8F03083420CBF44
:10D0E0004FF400134FF48003086B03430B6341E6D6
:10D0F0000C2800F2FF802A4B03EB4000B0F8F41636
:10D10000C84300B28C2303FB0693A3F88C10D3F81A
:10D110000431998A084098821DE6D5F8008092F87B
:10D120000D114FEA9822A2F58012522A3FF6F8AC70
:10D130001B4800EB020C9CF88CC1BCF10D0F40F2B7
:10D14000DC804FF0000C61453FF412AD024492F8D0
:10D150008C210D2A7FF6C8ACE3E4B8F800309BB20E
:10D1600043F08003A8F80030B8F844306FEA434336
:10D170006FEA53439BB2A8F84430B8F800309BB232
:10D1800043F00103A8F8003015E700BF3F801CF012
:10D19000E19E0008DC3700200038024000600240B9
:10D1A00050870508AC4B984500F03D81B8F1804FA1
:10D1B00000F03D81A3F57C43984500F0368103F5EE
:10D1C0008063984500F0378103F58063984500F04F
:10D1D000308103F58063984500F0338103F5806367
:10D1E000984500F02C8103F57043984500F031819B
:10D1F00003F57053984500F02A8103F58063984544
:10D2000000F0238103F58063984500F01C81A3F5AD
:10D21000983398457BD003F58063984500F00D81E5
:10D2200003F58063984508BF0D2371D0B8F800302E
:10D2300023F001031B041B0CA8F80030D9F80030C0
:10D240005B0807EE903A039B063BDAB2022AF8EE3F
:10D25000677A0A9200F29980804BDFED816A03EBD6
:10D26000820303F5F06292ED007AB8EE477A87EE1A
:10D27000870A30EE260A4AF03DFD039B0138082B51
:10D2800082B214BF13215F217348B8F80030804583
:10D290009BB26FD000F5806080456BD0B8F1804FB5
:10D2A00068D0A0F58030804564D000F5806080456E
:10D2B00060D000F5806080455CD06A48804570D0C1
:10D2C00000F5806080456CD023F440739BB2A8F8D1
:10D2D0000030614BC8F82C109845A8F8282040F081
:10D2E00089800023A8F830300123A8F81430EAE43C
:10D2F0000020CAE44FF0FF3004E7DFF878E11EF9C0
:10D300000CC020E7052364E60722029284E40B2385
:10D31000524A02EBC303012193F8143703F01F02B2
:10D320005B09032B01FA02F253D0042B26D14E499C
:10D330000B6B13430B63B8F8003023F001031B049D
:10D340001B0CA8F80030494B984510D0A3F580631A
:10D3500098450CD003F58043984508D003F58063C9
:10D36000984504D003F5806398457FF467AFD9ED05
:10D37000007A68E723F070039BB29EE7022BDAD1B4
:10D3800039494B6C1A434A64D5E79FED397A9FEDD2
:10D39000340AA7EE870A4AF0ADFC013882B21321A5
:10D3A00072E7A8F80030C8F82C10A8F828209BE7EE
:10D3B00001230EE602230CE603230AE6042308E613
:10D3C000062306E6072304E60022029224E408234B
:10D3D000FFE525490B6C1A430A64ACE7012202926F
:10D3E0001AE40A23F5E50923F3E50B23F1E502220C
:10D3F000029211E41D4B98453FF473AF74E70C2380
:10D40000E7E50322029207E40E23E2E50D23E0E5BF
:10D410000422029200E405220292FFF7FDBB0622DD
:10D420000292FFF7F9BB002372E7022370E70123A2
:10D430006EE704236CE703236AE70C2368E70623FF
:10D4400066E7052364E70A2362E7092360E7082308
:10D450005EE707235CE700BF000001405087050836
:10D460000AD7233C0010004000380240000401406D
:10D47000FCF4B23450FF050838B5424C8C2303FB52
:10D48000004393F88F3003B938BD94F8E0C494F8A2
:10D49000E1349C450ED003EB430204EBC20292F848
:10D4A000E4E40EF1FF35012D4FEA430246D9BEF107
:10D4B000030F3ED08C2202FB0042A2F88010EFF353
:10D4C0001181902383F31288B2F8805092F8823051
:10D4D00043EA45030025C9B29BB282F8825081F32A
:10D4E000118829491A090D7882EA13225A4005B198
:10D4F000D2431B019BB202F00F021A4391F81C3970
:10D500005BBB8C2303FB0044D1F8643AD4F80801D8
:10D5100001219847D4F80411B4F88C508A8AD4F8C1
:10D5200000312A438A8258601A6842F001021A6068
:10D5300038BD5D1C05F003056545BBD0134404EB05
:10D54000C303034493F8F1140029B3D08C2303FBE5
:10D550000043012283F88220ACE78C2303FB0044C4
:10D56000D1F8645AD4F88830D4F804115B7908698A
:10D5700003F0FC0318440421A847D4F804318000C8
:10D58000988138BDE81800200400001030B504462A
:10D59000006EA268838923F400531B041B0C838153
:10D5A000637995B013F0040F4FF00001019214BF9E
:10D5B0004FF480520A46ADF808201A031B0203F408
:10D5C0008063ADF80C302379ADF80E1002F40052F0
:10D5D000ADF80A20DA0744BF0422ADF80E209B07FD
:10D5E000ADF8101005D5BDF80E3043F00803ADF8C6
:10D5F0000E3001A941F01CFD6279236ED50700F1C0
:10D600008B8012F0080F9A8A48D092B242F008023A
:10D610009A829A8992B242F400529A812279D00772
:10D6200032D5E06B002800F089800023E26D08937A
:10D63000CDE90C33CDE91033CDE912334FF48075C9
:10D640000A936369E1680E9506920793626C0592EE
:10D650004FF480634FF480350B9309910F9541F09F
:10D660008DFA05A9E06B41F01FFBE26B216E136898
:10D6700043F0010313608B8A9BB243F040038B821B
:10D68000536822799BB2636591070DD4226E93890A
:10D690009BB243F40053938115B030BD22F00802D1
:10D6A0001204120C9A82B4E7206C002852D023692D
:10D6B000A26D0993A36CCDE90532402300254FF4F8
:10D6C000803108934FF480630B930F91CDE90C5593
:10D6D000CDE91055CDE9125507950A950E9541F003
:10D6E0004DFA206C05A941F0DFFA236C226E5869CF
:10D6F00040F080005861186840F0160018605D60C6
:10D70000938A9BB243F0800302F10C0193820B6871
:10D7100043F040030B60BAE71E498B4224D0A1F5C9
:10D720004C418B421ED001F580618B421ED10220FC
:10D730000121FFF7DFF86279236E62E74FF6DF71B0
:10D740001980D96841F02001D960D96841F01001F1
:10D75000D96099E7226ED36843F0800302F10C018F
:10D76000D360D4E70120E3E70020E1E701F5806121
:10D770008B420AD001F580618B4208D001F544410B
:10D780008B427FF43EAF0520D2E70320D0E7042090
:10D79000CEE700BF001001402DE9F84F484C04EBE4
:10D7A0008004D4F8684A002C00F08180E56E002DDA
:10D7B00079D01F46EB6A6361AB6AA3616B8EE3604D
:10D7C0002B8E23616B6823663E4B23603E4BA1602A
:10D7D000A3660646204691460DF002FD94F87100BE
:10D7E0000DF098FB804695F8200094F870B0A246A2
:10D7F000002855D102233A0784F87C303BD419F035
:10D80000020F15D0B8F1000F12D00B2388F80630A4
:10D81000731C88F80730FB074BD494F871000DF0A7
:10D8200079FB012384F87C3010B120210CF0FEFE3E
:10D8300019F0010F04D1E26B9AB15046BDE8F88FA0
:10D8400058460DF067FB0028F5D00C220136C67152
:10D85000827195F8212022210BF0FEFDE26B002A57
:10D86000EBD195F8241095F82200890945F03EF98E
:10D870005046BDE8F88F0136F6B2B8F1000F04D07B
:10D880000B2388F8076088F8063017F0500F95F8DA
:10D890002120404614BF022112210BF0DDFDCAE712
:10D8A00046F0CEFAA6E7AA465046BDE8F88FA24653
:10D8B000C3E795F82120404622210BF0CDFDB7E7C4
:10D8C00004000010DC8E05080DA8000808B572B62B
:10D8D000FDF742FC00B583B00D4900220092009193
:10D8E000009B0C330093009B1B68012B02D003B0FC
:10D8F0005DF804FB01920191019B06490C330193F1
:10D90000019B1A600B6883F308884B689847FEE711
:10D91000502800400000FF1F30B5012085B041F0C5
:10D9200045FA7A4A936823F003039360936813F0EF
:10D930000C0FFBD113687549002858D143F001033F
:10D94000136041F288330A68950771D4013BFAD11C
:10D950006F4C704D6D4B704AEA60704A596FAA6007
:10D96000596B6F4821F080015963596F41F0807104
:10D970005967196B41F4CE0119635A6B5A639A6B5C
:10D980009A631A6C02431A64596C664A0A435A64D1
:10D99000684641F0A5F8009B6349644A6448A1FBCE
:10D9A00003139B0C44F8243CD5F8FC30002143F0D1
:10D9B0008073C5F8FC30C2F8B00F516013685D4841
:10D9C00043F00103136003685B4AA2FB03239B0936
:10D9D000013BB3F1807F08D24FF0E022F020536189
:10D9E000072385F823009161136105B030BD43F42E
:10D9F000803313600A68940341F2883304D4013BF6
:10DA0000A6D00A689403FAD5414C4C4A4C4BB0FB63
:10DA1000F3F3B0FBF2F0B3EB400F18BF18464FF42E
:10DA20008002B3FBF0F344F8282C44E90F0307E02D
:10DA3000374C0822022344E90F23002144F8281C14
:10DA4000022041F0B3F903280FD83E4B54F8381C9C
:10DA500003EBC0008588C288438844F8305CB3FB80
:10DA6000F1F344F82C2C44F8343C284B36491A6C1A
:10DA700042F080521A640A6842F440420A609A688E
:10DA80009A609A6842F400429A609A6842F4A052FE
:10DA90009A6054F8280C54F83C2C54F8341C024377
:10DAA00042EA811254E90C10490842EA0062013945
:10DAB00042EA01425A601A6842F080721A601A689B
:10DAC0009201FCD5214A40F205711160996821F05C
:10DAD00003019960996841F00201A2F580629960A2
:10DAE000936803F00C03082BFAD154F8380C18494A
:10DAF000D823B3FBF0F39B0143F000530120C2F89D
:10DB000084308866FAF77CFA23E700BF00380240C9
:10DB1000D83A002000ED00E00005FA0500000020E2
:10DB2000FFC9FE36335F070083DE1B43001000E0B1
:10DB300055CEACC5E8180020D34D621080841E007D
:10DB400040420F000C8F050800700040003C02406E
:10DB5000000047421D4B1E48196C1E4A10B441F08C
:10DB600080510124196404625321FF24CA205462A5
:10DB7000506251625B6FDB0085B017D416480423F6
:10DB8000002102910290029A1A440292029A0433EE
:10DB90001C2B1160F5D103910390039B0393039B0E
:10DBA0000E4A1A6005B05DF8044B70470A4B00221C
:10DBB00001920193019B0193019A084B12689A42CA
:10DBC000DCD105B05DF8044B704700BF003802405F
:10DBD00000000E4200280040502800403166654297
:10DBE00070B5444DC1F1030195F8CC2041EA8001A4
:10DBF000CBB29A428AB073D03F4C85F8CC3010211A
:10DC000084F8BC16122184F8C016132184F8C216B9
:10DC1000142184F8C416152184F8C616162184F838
:10DC2000C816172184F8CA16182184F8CC161921B1
:10DC300084F8CE161A2184F8D0161B2184F8D21647
:10DC40001C2184F8D4161D2184F8D6161E2111201B
:10DC500084F8D8161F2184F8BE0684F8BD3684F8EF
:10DC6000BF3684F8C13684F8C33684F8C53684F8E4
:10DC7000C73684F8C93684F8CB3684F8CD3684F8B4
:10DC8000CF3684F8D13684F8D33684F8D53684F884
:10DC9000D73684F8D93684F8DA1604F2246684F884
:10DCA000DB3604F2BC630022012500936946202381
:10DCB0003046CDE90123CDE90422CDE906220992BF
:10DCC0008DF80C508DF820500BF050FED4F824360F
:10DCD0005A6A12B1B24205D0FEE71A6A002AFCD194
:10DCE0000AB070BD1A6A002AFAD01A6A002AF9D15D
:10DCF000F6E700BF88010020E81800200A4BB3F8BF
:10DD0000CA1071B1094B0A4A01EB030C01E06345EB
:10DD100007D013F8010B12F8011B8842F7D000203E
:10DD200070470120704700BF88010020B83A0020EA
:10DD3000C81F00202DE9F041964D974ED5F8C845F3
:10DD400094B028B9D6F8303303F57A73A34254D28D
:10DD5000924FC6F8304300230122FF21CDE905325E
:10DD6000CDE90833CDE90A338DF80C100D9304A9E1
:10DD700003AB38468DF81C208DF8302004930191B8
:10DD80000BF0F4FDD5F8243601995A6A002A3BD0ED
:10DD9000BA4200D0FEE71A6A002AFCD10023CDE97E
:10DDA000083305938DF81C300D93109312930123C3
:10DDB00006930B938DF830308DF8443080238DF826
:10DDC0000E300DF10E0304930DF10F0300220A93A0
:10DDD00072480023CDE90E230BF0C8FDD5F8243698
:10DDE0005A6AC2B1BA421DD11A6A002AFCD19DF802
:10DDF0000F3096F8C8209A423ED195F8220690B18D
:10DE0000002014B0BDE8F0811A6A002AC6D01A6A50
:10DE1000002AF9D1C2E71A6A002AE8D01A6A002A51
:10DE2000F9D1E4E7FEE7DFF87881D8F8A033E31A08
:10DE3000B3F57A7FE5D90123584F06938DF81C304E
:10DE40008DF83030FF2304A9CDE90800CDE90A00A0
:10DE500005900D908DF80D3038460DF10D030493AB
:10DE600001910BF083FDD5F8243601995A6A002AF6
:10DE700032D0BA4206D0FEE7FBF7BAF8012014B060
:10DE8000BDE8F0811A6A002AFCD10023CDE90833ED
:10DE900005938DF81C300D93109312930123069374
:10DEA0000B938DF830308DF84430A0238DF80E3070
:10DEB0000DF10E0304930DF10F0300220A9337486E
:10DEC0000023CDE90E230BF051FDD5F824365A6A14
:10DED0006AB3BA4207D0FEE71A6A002AD5D01A6A96
:10DEE000002AF9D1D1E71A6A002AFCD195F8CC288A
:10DEF0009DF80F30172A0FD196F8C82002F0400283
:10DF0000002AA5F8D02803F00702A5F8D22814BFEC
:10DF100010220D22A5F8D62859070FD50023C8F8DE
:10DF2000A4330020C8F8A04314B0BDE8F0811A6AF9
:10DF3000002ADBD01A6A002AF9D1D7E703F00503DB
:10DF4000012B1CD0002BECD196F8C8305B06E8D52D
:10DF5000D8F8A433C3B1D5F8C825D31A642BE0D9B7
:10DF6000FBF746F895F8CC38172BDAD1B8F8A83378
:10DF700001339BB2A8F8A833A5F8D438D1E796F8B6
:10DF8000C8305A06E4D5CCE7D5F8C835C8F8A4336C
:10DF9000C7E700BFE8180020880100200C1F002000
:10DFA000D83A00202DE9F04FDFF8E4B19BF8AA330E
:10DFB00085B03BB1BBF8AC03003818BF012005B0F9
:10DFC000BDE8F08FDFF8CCA1DAF82436197B61B90F
:10DFD0000A220821CDE90021596A91B1684881429D
:10DFE0000FD0012005B0BDE8F08F9AF8AC160029DB
:10DFF00014BFF6220822019214BF14220A220092B2
:10E00000EAE71E6A002EECD19BF8AB135D4BDFF8FC
:10E010008881BBF8AC73C1EB011103EB411903F527
:10E0200074730393B8F8CA3007EB53070DF0E6FD9D
:10E03000BBF8AC33029001253446BB4257DA0DF0F1
:10E04000DDFD029BC01A009B834250DDBBF8AC3360
:10E050000AEB030009EB030E90F8E0C619F8030081
:10E06000844567D0FF285FD005B92EBB0AEB0301BA
:10E070009EF8016091F8E1168E4265D09BF8AA14D3
:10E080000BEB040641F0010186F8B113042186F878
:10E09000B013023401260BEB04014FF0050C81F89C
:10E0A000B0C34FEA132C81F8B1C34FF0060C04340F
:10E0B00081F8B33381F8B2C3611C0AEB030E0BEB9A
:10E0C000040C59448EF8E0064FF0070E8CF8B0E3CC
:10E0D000023481F8B0030025B8F8CA0001339BB2BE
:10E0E0009842ABF8AC3347D9019A9442A5DB002E95
:10E0F00038D02548002D3AD0631C0BEB04015B445B
:10E100009BF8AA54042681F8B063023483F8B05314
:10E11000C8F8340301231D491948C8F83C438AF85C
:10E1200070350BF023FC45E74FF0200209F803207F
:10E13000202099E7002DCFD196B1039A4FF60771B1
:10E14000115335460234C7E70BEB04019BF8AA6470
:10E1500081F8B163042681F8B063023400269AE79F
:10E160000125B9E7002C3FF425AF0748D0E74FF66B
:10E17000077303530234BFE70023ABF8AC33B6E7B1
:10E180000C1F0020B83A0020883E0020BC0400206C
:10E19000D83A0020E81800208801002008B50120A6
:10E1A000FFF7C8FDFFF7FEFE0028FBD108BD00BF4A
:10E1B00000B5114BA3F1200C93F8AB33C1EB011E5A
:10E1C0001178C3EB03130CEB431C91B11D2810D83D
:10E1D0004FEA4E0E431E73440CF11D00634470441D
:10E1E00001E0834205D003F8011F12F8011F002946
:10E1F000F7D15DF804FB00BFD83A00202DE9F04FBD
:10E20000A74CD4F824362DED028B5A6A93B0814680
:10E210000F46002A34D004F22468424500D0FEE7BD
:10E220001A6A002AFCD100239E4A8DF806308DF828
:10E23000073003938DF81430069308930B930E93D5
:10E240001093012382F8AA330493002209938DF8D6
:10E2500028308DF83C30944800230DF106050DF16F
:10E26000070602A9CDE90C23029507960BF07EFB69
:10E27000D4F824365A6A002A32D0424506D0FEE746
:10E280001A6A002AFCD1DFF82082CCE71A6A002A39
:10E29000FCD1002303938DF81430069308930B935D
:10E2A0000E9310930123049309938DF828308DF871
:10E2B0003C30092300228DF806307B488DF807900A
:10E2C000002302A9CDE90C23029507960BF04EFB23
:10E2D000D4F824365A6A002A39D0424507D0FEE7DE
:10E2E0001A6A002AD5D01A6A002AF9D1D1E71A6A27
:10E2F000002AFCD19FED688BDFF8ACA1013F4FF005
:10E30000000B4FF00A090023012202A95046CDE973
:10E310000832CDE90253CDE9063604928DF8143067
:10E320008DF828200B930E938DF83C2010938DEDE3
:10E330000C8B8DF806908DF807B00BF017FBD4F816
:10E3400024365A6A002A33D0424507D0FEE71A6ABB
:10E35000002ACFD01A6A002AF9D1CBE71A6A002A1C
:10E36000FCD10B238DF80630002317F8012F8DF810
:10E370001430CDE90253CDE9063608930B930E9382
:10E38000109302A9012350468DF8072004930993A6
:10E390008DF828308DF83C308DED0C8B0BF0E6FAC3
:10E3A000D4F824365A6A002A43D0424507D0FEE703
:10E3B0001A6A002AD5D01A6A002AF9D1D1E71A6A56
:10E3C000002AFCD1D4F8D43533B19A881B68596936
:10E3D0000A4214BF5A831A830BF1010BBBF1360FAB
:10E3E00091D1002303938DF81430069308930B9377
:10E3F0000E9310930123049309938DF828308DF820
:10E400003C3008238DF80630A02300228DF8073019
:10E4100025480295002302A9CDE90C2307960BF0AD
:10E42000A5FAD4F824365A6A002A3FD0424507D0CC
:10E43000FEE71A6A002AC5D01A6A002AF9D1C1E794
:10E440001A6A002AFCD1DFF86090A0274FF0000A7A
:10E450004FF0000B0023012202A94846CDE90253E8
:10E46000CDE90633CDE9086204928DF814308DF8B9
:10E4700028200B930E938DF83C201093CDE90CAB24
:10E480008DF806700BF072FAD4F824365A6A0AB383
:10E49000424512D0FEE700BF00000000000000006F
:10E4A000E8180020D83A00200C1F00201A6A002A21
:10E4B000C9D01A6A002AF9D1C5E71A6A002AFCD124
:10E4C0009DF807309B06C5D4012013B0BDEC028B2C
:10E4D000BDE8F08F1A6A002AF2D01A6A002AF9D130
:10E4E000EEE700BF0548D0F8843523B1DB6A13B1ED
:10E4F00000F2845018470248704700BFE818002017
:10E500002C8F050838B5184CD4F8AC341B8843B9A7
:10E51000164D002384F8B83485F87C35C5F8783575
:10E5200038BDD4F8B024002AF2DD012A09D0D4F88D
:10E53000B43459880D4DA4F8BA14012384F8BC34BE
:10E54000E7E7D4F8B4148A8849880132521A9A420B
:10E55000F0D1064DD5F8843500221B69C5F8B025E9
:10E5600005F284509847D4E7D83A0020E8180020F4
:10E570000748D0F880351BB1064B93F8BC340BB17B
:10E5800000207047D0F8843500F284505B6818474B
:10E59000E8180020D83A002030B4154A154D92F8FA
:10E5A0007C3505F598642344036095F8B8344460DD
:10E5B00092F87C05834292F87C0512D8834204D3FA
:10E5C000002030BCC1E90000704792F87C25002B88
:10E5D000C2F180020CBF0120022030BCC1E900233F
:10E5E00070471B1A0022012030BCC1E9003270477D
:10E5F000E8180020D83A00200E4B0F4A93F87C15FB
:10E6000092F8B80493F87C25904293F87C250CD8B6
:10E61000904238BF93F87C25D3F878353ABFC2F1E1
:10E6200080028018002018447047D3F87835801A8B
:10E6300018447047E8180020D83A002030B51C4C28
:10E640001C4D94F87C3594F87C1585B005F59862DE
:10E650001344029395F8B83403928B421DD894F872
:10E660007C25934211D294F87C150193C1F180016D
:10E670000091D3B9012208B93F2906D90023694680
:10E6800002A847F0FBFD95F8B83494F87C05C01A51
:10E69000B0FA80F0400905B030BD94F87C15002236
:10E6A000591A019200910122E5E719440222E2E79A
:10E6B000E8180020D83A00202DE9F043164685B02E
:10E6C000002935D0441E254D254F04EB01084FF09D
:10E6D000000901E0A0452BD095F8B80414F8013FDB
:10E6E000411C2844C9B280F8C0340B0648BF002042
:10E6F00097F87C3585F8B8144ABF0146084685F876
:10E70000B8948B4297F87C358ABFC3F18003C01A56
:10E71000C0183F28DED997F87C358B42DAD0114BF0
:10E720009B78002BD6D00020FFF788FFA045D3D1DF
:10E73000694602A8FFF730FF20B1DDE9003213443B
:10E740003F2B02D805B0BDE8F0830246334602A84D
:10E7500047F094FD05B0BDE8F08300BFD83A002033
:10E76000E81800208801002030B585B0694602A86D
:10E77000FFF712FF58B9094C04F28455D4F88435D8
:10E7800028465B6898470028F8D005B030BD02469F
:10E79000012302A847F072FDEDE700BFE818002052
:10E7A00070B5124E1546D6F880350A464119994281
:10E7B0000F4988BF1D1A91F8B81496F87C35994214
:10E7C00082B0044603D00192FFF7CEFF019AD6F83B
:10E7D000841508480023C6F8B0352B468D6A2146BB
:10E7E000AC4602B0BDE87040604700BFE8180020AA
:10E7F000D83A00206C1E00208C4613460146624623
:10E800001846CDE738B52448244C0023C4F8803599
:10E8100002461178022902F106022CD00133062BA0
:10E82000F7D11F4DD4F884350022C5F8B424F3B1D4
:10E83000DA6AE2B11B489047D5F8B434C5F8AC04A5
:10E84000A3B19A885B88D21A436802FB0333C4F8E9
:10E850008035FAF7DBF895F8B82494F87C359A42BD
:10E86000054601D0FFF780FFC4F8785538BD0E4B40
:10E87000C5F8AC3438BD0A4DD4F8842503EB430306
:10E8800000EB4303C5F8B43412B1D26A002AD1D1E7
:10E890000548C5F8AC04D4E718400020E81800206B
:10E8A000D83A00206C1E00202C8F050810B50A4CA9
:10E8B000D4F884355B6A13B104F284509847074A50
:10E8C000D4F87835D2F8AC245288013B1344524234
:10E8D0001340C4F8783510BDE8180020D83A00205D
:10E8E0002DE9F043DFF8E890374F93B0FFF70AFEC9
:10E8F000FFF788FF99F87C3597F8B8249A4201D041
:10E90000FFF732FFD9F880850025C9F87855B8F1AE
:10E91000000F11D02D4E6C462A463146204601F09C
:10E9200089FE204647F05CFD203501460122204645
:10E93000FFF7C2FEA845EFD899F87C3597F8B824C0
:10E940009A4201D0FFF710FFD7F8AC349B7B012B24
:10E9500033D099F87C3597F8B8249A4201D0FFF764
:10E9600003FF0027C9F87875B8F1000F28D0DFF849
:10E970005C903D466C462A46494609A801F05AFE7D
:10E9800021220021204649F090FE202221462846DF
:10E99000FFF706FF2022064609A92046154449F044
:10E9A000B0FE08B9202E00D00137A845E3D8B7FA49
:10E9B00087F0400913B0BDE8F083FFF777FFC8E7A1
:10E9C000012013B0BDE8F083D83A0020C8FE050846
:10E9D000E8180020032108B5054608463EF00EF968
:10E9E00072B6104B53E9022352EA03010AD1002404
:10E9F000214604203EF002F9214605203EF0FEF8B3
:10EA0000FCF7AAFB0848D0F8C84529B24EF66020AA
:10EA100000FB01F1A41843F100030C1943EBE17171
:10EA2000E7E700BF48400020E818002008B50021B3
:10EA300003203EF0E3F872B6FCF78EFB08B5184CE5
:10EA4000D4F8702594F876054AB11168938809695D
:10EA50000B40F8B9003B18BF0123002BF4D1142060
:10EA60000FF006FB00BFD4F8703563B11A689B88BD
:10EA7000116994F876250B4042B9003B18BF012379
:10EA80000BB1FFF7D3FFF9F7F3FFEBE7B3FA83F32B
:10EA90005B09F5E7B3FA83F35B09002BD4D1DEE71A
:10EAA000D83A002008B541F019FC1B200CF032FACE
:10EAB00008B12923C38041F027FC08B12923C38072
:10EAC000094B93F87D25012A01D0012008BD074894
:10EAD000C3F8800500F120014C3043F0E3FD044B06
:10EAE000002083F8230008BDD83A0020E404002069
:10EAF00000ED00E02DE9F04F41F694628BB000216B
:10EB0000BD4849F0D2FD042040F050F904460520EC
:10EB100040F04CF950EA040340F05C81B74B03939A
:10EB20004C220021B44849F0C0FD4C220021B248DB
:10EB300049F0BBFD039BB049D3F8F433B04A0A60F7
:10EB40000124C1E907334B620C7145F08DFCFFF7DE
:10EB500059FE002108460CF06FFAF9F757FFB0F1A3
:10EB6000000B40F30881A74BA74D0193A24BA74E82
:10EB70000024029403F14C092746A04605F2845A6A
:10EB800004E008F50068C34540F3AE80019AD2F86E
:10EB9000C835C2F8CC35F9F76BFF20225146404604
:10EBA000FFF7FEFD9A491222504649F0AAFD0028BF
:10EBB000E7D1B84522D00299964BCDF8149001EBDD
:10EBC000410203EB82004A1C93490292049001F037
:10EBD00031FDDDE90403D9F81C2043F84C0BC9E9E9
:10EBE00008228E4AC9F80C70C9F82820A8EB07073C
:10EBF0000122C9E90477C9F808209946039BD3F894
:10EC0000F433C9F81C3047461222A918335D91F835
:10EC10008415994202F101020BD00024202AF4D17C
:10EC20002037BB455146384654DBFFF7B9FD00227B
:10EC3000EBE70134152CF1D1D01979492022FFF7E7
:10EC4000AFFD00230A2209A97548CDF824A001F0E0
:10EC50009FFE04900998002301300A2209A9099017
:10EC600001F096FE07900998002301300A2209A9B5
:10EC7000099001F08DFE06900998002301300A22C8
:10EC800009A9099001F084FE0590099809A90130AD
:10EC900000230A22099001F07BFE07460998002311
:10ECA000013019460A22099001F072FE049989B1D7
:10ECB000DDE9063243EA4212059B7F0147EAC3239E
:10ECC000A1F2BC7143EA600342EA412243EA0243F3
:10ECD000C9F81C30029B642B00F0EC80474608F515
:10ECE0000068C3453FF752AF029A642A00F0E28001
:10ECF000B84500F0E380474C4749484E0C2303FBDE
:10ED00000244531C1A462046A8EB0705029301F063
:10ED100091FCD9F81C30C9F80040C9E90375C9E96C
:10ED200008330123C9F81450C9F82860C9F808301D
:10ED3000029B5D1C4C22304F02FB05F57B19002124
:10ED4000184649F0B2FC4C22002149F0AEFC039A6F
:10ED50003449D2F8F4237951029C4262C0E904BBE1
:10ED6000C0E9072201220234866282604FEA4B0327
:10ED7000B3F1805F1EDA4C221F4D02FB04F42B1905
:10ED80001846002149F091FC4C22002149F08DFCED
:10ED90000399CBF10062D1F8F413034652002248E4
:10EDA0002851C3E90422C3E9071102225A71012242
:10EDB00059629A60104A95682DB913791BB113688E
:10EDC000002B40F08980002108460BB0BDE8F04FD1
:10EDD0000CF032B94FF47A720023214647F05EFFFF
:10EDE000124B40F26D11A3FB00231B0C022440F2D6
:10EDF000B2720D4625E000BFE845002088010020E2
:10EE00004CFF0508E8180020D83A00200CFF050840
:10EE1000E8FE05087C400020FCFE0508F9E7000834
:10EE20005C40002024FF050834FF050807452EC27A
:10EE3000013212F00304A3EB01030CBF4FF4B771CE
:10EE400029469942F4DD7A49002C3FD00391039979
:10EE5000D1F8C4138B4272DB764D01245B1A55F84E
:10EE6000041F994204F10104F8DD013343EA44131D
:10EE7000A2F2BC7243EA42236F4A039DB0FBF2F157
:10EE800002FB11024FF461603C24B2FBF0F100FB85
:10EE900011221C20C5F8C803B2FBF4F004FB1022B9
:10EEA000521042EA401242EAC12242EA0343C5F844
:10EEB000F43335E66423614E029339E7029B012463
:10EEC0005D1C002B3FF452AF5C4E33E70C460391C0
:10EED0001D21C4F8C813BAE7C2E911551564D563FA
:10EEE00029462E46D46C02F14C0354B39C681E6430
:10EEF000481E8442C3E91166DE6312D0481C844276
:10EF000016D08C427FF45FAF084600283FF45BAF19
:10EF1000116CCC6B0134CC631964936401461A46BE
:10EF2000E0E700293FF44FAF884253F80C2CECD1B6
:10EF3000117900293FF447AF53641A64EEE70124C6
:10EF400093E73F490222264613E0CB6B0A635B013D
:10EF50001DBF03F6FF7702F1FF3303EB17331346B0
:10EF6000C1E90466C1E90D3351F84C0F5A1C013553
:10EF7000C8B10B79002BE8D10F690A63002F4AD181
:10EF80004F691046531E4863002F4DD007F6FF7798
:10EF900003EB1733201A8B63C41851F84C0F5A1C1B
:10EFA00001350028E5D127492748C1F81C563E22E3
:10EFB0000D46C1F8F8253F22013BC1F8FC2540224F
:10EFC000C1F800260191C1F80C36C1F810469A002C
:10EFD000990FC5F8F4054BB340F2FF10121841F138
:10EFE0000001520A42EAC152019C02F140010A4466
:10EFF00002EBC303C4F80826C4F80416134A1049E8
:10F00000C4F81416C4F818165802D90D42E90201C2
:10F01000C4F8F035D7E607F6FF77531E03EB173039
:10F020004F694863002FB1D11346B3E70122DBE7F4
:10F03000880100204C05002080510100F9E70008FC
:10F04000E8450020E818002040FF0508D81E0020F1
:10F0500000234FF6FF720121017243818381C38136
:10F0600002828274704700BF154BFF22F0B54FF04B
:10F07000000C4FF0FF3EC270027102724272427386
:10F08000827303F10C07764665466446624602EBDE
:10F09000820281189F4284544D7081F802C0CE7064
:10F0A00081F804E00BD093F90620DC791D7A93F8FF
:10F0B00009C093F90A6093F90BE00633E7E7F0BD66
:10F0C000688F050800230222037043708370C370A9
:10F0D00002717047002303704370704700230122C0
:10F0E000027043708370C370704700BF4FF4F072BA
:10F0F00002804FF4FA6240F22E4C0921028440F261
:10F1000026220023A0F81EC081704FF47A7C0E21C5
:10F1100082830222A0F822C0437140F2012C836056
:10F12000C36080F82410427440F2034140F205624B
:10F1300043820723A0F814C0C182028383767047FC
:10F140008388C3F30B039342A8BF134670B51A46D6
:10F150001D460C460646806849F044FA62199442FE
:10F16000B569074B08D0074814F8011B00FB03F3EF
:10F17000A24283EA0103F7D12B60012070BD00BFDA
:10F18000C59D1C81930100010023037043708370AF
:10F19000C37070470023037043708370C37070475F
:10F1A000002306214FF47A72C0E901230170037332
:10F1B000704700BF10B50023411CFF2200F8132048
:10F1C00001F813200133082BF8D10B4B4FF0FF311E
:10F1D00003F10F0400228C4605E093F904C093F973
:10F1E000051013F8032F00F812C000EB420E9C42EA
:10F1F0008EF80110F1D110BD7C8F0508704700BF5B
:10F200000A44914219D000B501F1FF3C02F1FF3EE2
:10F2100041F221011CF8012F082380EA022010F49A
:10F22000004F81EA40020ABF400090B280B2013B29
:10F23000F5D1E645EED15DF804FB7047704700BF9D
:10F24000D0ED007AD0ED016A30EE677AE6EE877A8B
:10F25000B0EE670AC0ED007A704700BFD0ED017ACA
:10F26000D0ED026A30EE677A90ED000AE6EE877A1A
:10F2700037EEC07AC0ED017AA6EE870A80ED000A6B
:10F28000704700BF90ED017AD0ED036AD0ED027AAD
:10F2900030EE470AA6EE807A90ED000A80ED017A02
:10F2A00037EE676AE6EE867A37EEC07AC0ED027A0C
:10F2B000A6EE870A80ED000A704700BFD0ED056A10
:10F2C000D0ED017A90ED007A90ED066AD0ED025A09
:10F2D00090ED035A80ED050A66EEA77AC0ED066A46
:10F2E000E7EE007A90ED077AE5EE867A90ED086A0F
:10F2F000D0ED045A80ED087AE5EE477AE5EEC67A5D
:10F30000B0EE670AC0ED077A704700BFD0ED057A0E
:10F3100090ED006A90ED067AD0ED035AE6EE007AA1
:10F3200090ED016AF0EE406AA6EE267AB0EE670A2A
:10F33000D0ED047A90ED026A67EEC07AA5EEC07A4D
:10F34000E6EE267A80ED057AC0ED067A704700BFBA
:10F350002DE9F047089F3C460E4614F8011B002B90
:10F36000054614BF4FF030094FF0200941B3002A81
:10F370002CDD234600E0B2B113F8010B9046013AB0
:10F380000028F8D1A8F102086AB1C24649462846C9
:10F39000B0475346002B0AF1FF3AF7DC397828EAE8
:10F3A000E872013249B1D71B2846B047E01914F87A
:10F3B000011B0029F8D1BDE8F0871046BDE8F087B1
:10F3C000002A02F1FF38E0DC0846F4E70022EAE711
:10F3D00003685A1C02601970704700BF024B18681E
:10F3E00003681B68184700BF706A0020884210B588
:10F3F0004FF001043ED301FB04F4B0FBF4FC8C4558
:10F40000F9D2CCB122BB08E0A14203F801EBB4FB76
:10F41000F1F211D8B0FBF2FC1446BCF1090F0CF16B
:10F42000570E0CF1300204FB1C00EDDCA14203F886
:10F43000012BB4FBF1F2EDD900221A7010BDA142EC
:10F4400003F801EBB4FBF1F2F6D8B0FBF2FC144682
:10F45000BCF1090F0CF1370E0CF1300204FB1C005B
:10F46000EDDCA14203F8012BB4FBF1F2EDD900224F
:10F470001A7010BD8446002AEAD1CEE7002870B584
:10F4800003DA2D2301F8013B4042092886464FF05C
:10F49000010307DD03EB83035B00B0FBF3F2092AF2
:10F4A000F8D8EBB1104CBEFBF3FCA4FB0320C00862
:10F4B000BCF1090F0CF130060CF15705024607D8D4
:10F4C000092B01F8016B03FB1CEE09D90346EAE79F
:10F4D000092B01F8015B03FB1CEE01D91346E2E79F
:10F4E00000230B7070BD00BFCDCCCCCC0378202B9B
:10F4F000024600F10100F9D0092BF7D02D2B28D0BE
:10F500002B2B03BF5378B7EE000A0246B7EE000A72
:10F51000A3F13001C8B209289FED567A10D8F2EE57
:10F52000046A07EE901AF8EEE77A12F8013FE7EE68
:10F53000267AA3F13001C8B20928B0EE677AF0D973
:10F540002E2B5ED003F0DF03452B07D020EE070AF9
:10F5500070475378BFEE000A0246D9E710B45178DD
:10F560002D2978D02B296AD0A1F13003092B02F183
:10F5700001026BD80024002303EB830301EB430358
:10F5800012F8011FA1F130000928A3F13003F3D9CB
:10F59000B3F59A7F1A4628BF4FF49A72072B66D9A3
:10F5A000DFED356A1346F7EE007A083B072B67EE6E
:10F5B000A67AFAD802F00702DAB1F2EE046A012A5A
:10F5C00067EEA67A15D0022A67EEA67A11D0032A32
:10F5D00067EEA67A0DD0042A67EEA67A09D0053A1E
:10F5E00067EEA67A05D067EEA67A012A18BF67EE05
:10F5F000A67A6CB387EE277A5DF8044B20EE070AF3
:10F6000070475378A3F13001C8B2092802F1010212
:10F6100098D8F2EE046AF0EE665A07EE901AF8EE09
:10F62000E77A12F8013F87EEA66AA3F13001C8B26B
:10F63000092866EEA56A37EE067AEED982E7917858
:10F64000A1F13003092B02F1020293D9F7EE007AFF
:10F6500027EE277AD0E79178A1F13003092B02F148
:10F66000020288BFF7EE007AC4D8012483E7F7EEE0
:10F67000007AA1E70000000020BCBE4CF8B5164D92
:10F680006B78BE2B25D1022229464FF6FF70FFF77B
:10F69000B7FD124FAC1C22884AB1A618BE4218D240
:10F6A000052A16D92146FFF7ABFD3446F3E721467C
:10F6B0000222FFF7A5FD0222A118FFF7A1FD0634E3
:10F6C000074B641B9C8041F60F53C31A58425841A4
:10F6D000F8BD0020FCE700BF0040000800800008E3
:10F6E000706A0020F0B5067906F0E003402B03D1E4
:10F6F00044794FF0FF3506E0602B4FF00104F8D15C
:10F70000457904FA05F50023012006F00706A34217
:10F7100000D1F0BD042E0FD8DFE806F00308101D5D
:10F72000240048B1C85CD75C78400FE020B1C856CF
:10F73000D756C71B784278410133E8E70028FBD051
:10F7400031F8130032F81370784080B228420CBFB1
:10F7500001200020F0E70028EED031F9130032F943
:10F760001370E6E70028E7D051F8230052F8237021
:10F77000DAE7037903F01803102B1CD004D82BB15F
:10F78000082B06D000207047182BFBD1B0F80B00D7
:10F7900070470F4BB0F80B0093F90030591C06BFAF
:10F7A0000C4B1B7ADBB203EB8303C3EB031300EBBD
:10F7B000430080B27047064BB0F80B0093F901305C
:10F7C0005A1C06BF034B5B7ADBB200EB4310F0E739
:10F7D000A4050020706A0020114B002130B50160A3
:10F7E000818003F10C054FF448748E460A4602EB03
:10F7F000420200EB420C00F812E08CF80110DA78BB
:10F800008CF80220AB42ACF8044007D093F90620F4
:10F8100093F807E0197A5C890633E8E730BD00BF4A
:10F82000908F050801394B0003F00802930001F0A6
:10F830000301A3EB9203C1EB0111C3EB0313C1EB73
:10F84000011100229B008900026081804380704783
:10F8500000B589B000220DF1100C0492ADF814200F
:10F8600003469CE803004FF40070ADF81C101880AC
:10F87000BDF81C0098814FF4807E014640F20120C3
:10F880005A80A3F806E09A60D8811A82A3F814E09F
:10F89000C3F81620598309B05DF804FB144B1549D1
:10F8A00010B5044618681B79206284F824301522AC
:10F8B00004F1250048F039FF0F4B1A7E4FF0010E7E
:10F8C00084F83AE012B984F83B2010BD03F11C0C17
:10F8D000BCE80F0020606160A260E360BCE80F003C
:10F8E00084F83BE020616161A261E36110BD00BF6B
:10F8F00060FF050868FF0508706A002010B5002148
:10F900003822044648F0D1FE0B490C4A0C48C4E9A1
:10F9100004120C490C4AA262C4E90601012341F613
:10F920001E6CA373A4F826C084F821302146074832
:10F93000BDE810402FF072BB6400DC051A046C07B0
:10F940000019750343080E001E7D01017CFF0508A8
:10F95000B5EEC00ADFED347AF1EE10FACCBF30EE2E
:10F96000270A30EE670ADFED317A20EE270A70B5FC
:10F97000FDEEC07A86B017EE904A054684EAE47040
:10F98000002303A9A0EBE470CDE90033029341F01A
:10F99000B7F8002CACBF20232D2303A88DF800302E
:10F9A00046F01EFD01286E4628D0022832D00328DA
:10F9B0001CD003A9304648F080FE304646F010FDCA
:10F9C0000338C4B222463146284648F00BFE0023D5
:10F9D0002B55284646F004FD2E232B5401303119B7
:10F9E000284448F086FE284606B070BD302303A99F
:10F9F00030468DF8013048F060FEDEE743F2300219
:10FA0000302303A93046ADF801208DF8033048F0CB
:10FA100054FED2E743F2300303A93046ADF801307B
:10FA200048F04BFEC9E700BF6F12033A00007A446A
:10FA300009F0CEBE13B568B14C1E14F8011F21B9F0
:10FA400002B0BDE8104009F0D7BE019009F0C0FE39
:10FA50000198F2E702B010BD08B5202148F03CFE45
:10FA6000034620B11A78202A00F10100F8D0184688
:10FA700008BDF8B5D0B1104B0138C70003EBC0008A
:10FA8000CA4390F8406090F8415002F0010282EAC7
:10FA90000604A5420AD0C06B28B105688088B2422E
:10FAA00014BF288368833B4483F84140CB0701D4CB
:10FAB000FDF70CFFF8BD00BF706A00202DE9F3418F
:10FAC000124D134F002305F85C3F044600EB8106FE
:10FAD000B44203D10F4802B0BDE8F0813946284650
:10FAE00048F0EBFD2146684648F003FE4FF0000861
:10FAF0002021684648F0F0FD28B96946284648F0BC
:10FB0000DCFD0434E4E780F80080F1E7706A00204F
:10FB1000DD400608CC6A0020024BD3F8800037F0A5
:10FB2000C9BE00BF706A00202DE9FF471E46C368AA
:10FB3000BDF83070DDF8348004468946924643B300
:10FB4000CBB20D2B9ABF1A4AD5560025BAF1FF3F0A
:10FB500021D02368174A3146CDE9005A3846C047BC
:10FB6000524620795FFA89F109F0D4FE024600B1CD
:10FB70000288D3B20393C2F30323120BCDE90052E0
:10FB800002930D4A236831463846C04704B0BDE8A9
:10FB9000F0874D1CDAE77B06F8D42368074A0C95FA
:10FBA00031463846C44604B0BDE8F047604700BF60
:10FBB00050FF0508C83F0608D53F0608F93F06086C
:10FBC0002DE9F041154686B06A1C8846BDF83060C4
:10FBD0000D9F194623D0030900F00F044033CDE9EF
:10FBE0000045164A05933046B847A8B198F8051065
:10FBF000D8F800002A460AF0EFF968B102880178C7
:10FC00000391C2F30321120BCDE900420291059B3F
:10FC10000B4A00213046B84706B0BDE8F0817306B4
:10FC2000FAD40309074A00F00F000C904033304625
:10FC3000BC4606B0BDE8F041604700BF084006087A
:10FC40001A400608434006082DE9F04188B01E46D8
:10FC500003090E9F9046403300F00F0451B3079301
:10FC60000EF0BAFE027A079BCDE900420546164A1D
:10FC700041463046B847D0B128680EF099FFE9797F
:10FC80006A79DFF854C02D7A079B009411F0020FB7
:10FC90004FEA92020D4902F1010208BF6146CDE927
:10FCA0000102CDE903150A4A00213046B84708B0E1
:10FCB000BDE8F081074A0E9441463046BC4608B084
:10FCC000BDE8F041604700BF57400608A54106085F
:10FCD000694006088B400608964B0608084B094900
:10FCE0008B4202460AD2184602E01C30884205D2F6
:10FCF0000388C3F30B039A42F7D170470020704783
:10FD0000708706086C8F0608F8B50546B0F809003C
:10FD1000084EFFF7E3FF96F8847004462846FFF785
:10FD200028FD2FB196F8853013B9E3681844F8BD63
:10FD3000A368FBE7706A002038B505460C46FFF75C
:10FD4000E3FF2B7903F0E002602A03F0070329D1D7
:10FD5000022BDAB20ED0042A18D03AB96A790123FC
:10FD60009340DBB2027814B11343037038BD22EA2A
:10FD70000303FAE76A79012393409BB2028814B126
:10FD800013430380F2E722EA0303FAE76A790123C7
:10FD900003FA02F2036814B113430360E6E723EAAF
:10FDA0000203FAE7042BE1D8DFE803F003030505BB
:10FDB00007000470DAE70480D8E70460D6E700BFE4
:10FDC00070B585880B460446C5F30B052A4600210D
:10FDD000184648F06AFC6169084A9142034602D31A
:10FDE000074A914205D319B1BDE87040184608474B
:10FDF00070BD2A46BDE8704048F0F4BB6C8F060821
:10FE00002D91060838B5064C064DAC4206D2A168C5
:10FE100020461C34FFF7D4FFAC42F8D338BD00BFF6
:10FE2000708706086C8F06084840082310F0800F82
:10FE300082EA40010ABF4000C8B2C0B2013BF5D11E
:10FE4000704700BF30B505688D4219D901F1FF3EFA
:10FE50006C1E00231EF801CF082183EA0C0313F067
:10FE6000800F82EA430C0ABF5B005FFA8CF3DBB2BF
:10FE70000139F4D17445EDD16A1C02602B7030BD9C
:10FE800000236A1C02602B7030BD00BF07EE901A81
:10FE9000B8EE677ADFED7C7A27EE000A60EE277A0B
:10FEA000BDEEE77A17EE103A2033402B00F2DB80EC
:10FEB0009FED767AB4EEC70AF1EE10FAB0EE677AEB
:10FEC0000CDDDFED735A9FED736AF0EE476AF4EED6
:10FED000C66AF1EE10FA37EE657AF6DCDFED6E6A8F
:10FEE000B4EEE67AF1EE10FA0CD5DFED695A9FED2B
:10FEF0006B6AF0EE476AF4EEC66AF1EE10FA37EE7E
:10FF0000257AF6D4DFED666AB4EEE67AF1EE10FA01
:10FF100000F39D80DFED636AB4EEE67AF1EE10FA4D
:10FF200044BFDFED5D6A36EEC77A27EE075ADFED94
:10FF30005E5A9FED5E6ADFED5E6ADFED5E4AA5EE1A
:10FF4000256A27EE054AE5EE066AF7EE005AA4EEAA
:10FF5000267AF0EE656AE7EE646AE7EE245A86EEEA
:10FF6000A54A9FED4F7A77EE877ABDEEE77A17EED6
:10FF7000103A2033402B6FD89FED4F7AB4EEC70A6A
:10FF8000F1EE10FA0CDD9FED426ADFED426AB0EE51
:10FF9000677AB4EEE67AF1EE10FA77EEC67AF6DC1E
:10FFA0009FED3D7AF4EEC77AF1EE10FA0CD59FED95
:10FFB000386ADFED3A6AB0EE677AB4EEE67AF1EECF
:10FFC00010FA77EE867AF6D49FED357AF4EEC77A9A
:10FFD000F1EE10FA4CDD9FED397A77EE677A67EE35
:10FFE000A74A9FED317A9FED315ADFED316AA4EED9
:10FFF000875A67EEA43AE4EE856AB7EE006AE3EE4C
:020000040801F1
:10000000A67AB6EE007A36EE676AB8EE005A67EE68
:10001000857A26EE077AB7EE005AC5EE256A0023E8
:10002000836143610362C36180ED044A26EE877AEF
:1000300026EE866A66EEA77A80ED095A80ED007A90
:1000400080ED016A80ED027AC0ED037A7047DFED42
:100050001B6A36EEC77A68E7DFED197AB6EE007AEA
:10006000B7EE006AD7E7B7EE004AF0EE445A78E7F9
:100070009FED0C7AF4EEC77AF1EE10FA44BF9FEDD3
:10008000067A77EE677AAAE727D4D2360024F448B6
:10009000DB0FC940E4CB1641DB0F49C0E4CB16C1EE
:1000A000DB0FC93FDB0FC9BF92E741B99730083C6E
:1000B00015A82ABEF304353F00247448DB0F4940DD
:1000C00000000000DFED277AB4EEE70AF1EE10FA47
:1000D0000CDDDFED256A9FED257AF0EE407AF4EE37
:1000E000C77AF1EE10FA30EE660AF6DCDFED207A20
:1000F000B4EEE70AF1EE10FA0CD5DFED1B6A9FEDC6
:100100001D7AF0EE407AF4EEC77AF1EE10FA30EE96
:10011000260AF6D4DFED187AB4EEE70AF1EE10FA0B
:1001200014DDDFED107A37EEC00A60EE006A9FED55
:10013000136A9FED137ADFED137AA6EE867A20EE2E
:10014000266AE6EE877AA6EE270A7047DFED0E7A7A
:10015000B4EEE70AF1EE10FA44BFDFED057A37EEB0
:10016000C00AE2E7DB0F4940DB0FC940E4CB164190
:10017000DB0F49C0E4CB16C1DB0FC93F92E741B9A1
:100180009730083C15A82ABEDB0FC9BFF0EEC07A35
:10019000B0EEE07AB4EEE77AF1EE10FAB4BFB0EE6A
:1001A000676AB0EE476AB5EE406AF1EE10FA46D0E3
:1001B000B4EEE77AF1EE10FA8CBFF0EE675AF0EE8B
:1001C000475AC5EE866ADFED1F2ADFED1F3ADFEDE5
:1001D0001F4A9FED1F5A9FED1F3A9FED1F4ADFED0B
:1001E0001F5AE6EEE23AA6EE834AE6EEA34AB7EEDF
:1001F000006AA6EEA45AA6EE846AE6EE855AC5EE1B
:10020000866AB4EEE77AF1EE10FA48BFDFED147AB1
:10021000F5EEC00A48BF77EEE66AF1EE10FA48BF85
:10022000DFED107AB5EEC00A48BF77EEE66AF1EE70
:1002300010FA48BFF1EE666AB0EE660A7047DFED6D
:10024000076ADEE739094E3DE3B59E3E88FA163E61
:1002500045FE7F3F99FB243F69A2163EA7DFA834E5
:10026000DB0FC93FDB0F494090ED005A9FED4C0A70
:1002700035EE000A08B5FDEEC07A17EE903A20334D
:10028000402B7BD8FFF71EFFF0EE403AFDEEC57A1B
:1002900017EE903A2033402B7FD8B0EE450AFFF797
:1002A00011FFB0EE405AD0ED014A9FED3D0A34EE09
:1002B000800AFDEEC07A17EE903A2033402B69D8C1
:1002C000FFF700FFF0EE405AFDEEE47A17EE903AA9
:1002D0002033402B5BD8B0EE640AFFF7F3FEF0EE5C
:1002E000404A90ED023A9FED2E0A33EE000AFDEEF1
:1002F000C07A17EE903A2033402B45D8FFF7E2FE44
:10030000B0EE404AFDEEC37A17EE903A2033402B10
:1003100037D8B0EE430AFFF7D5FEF0EE407A24EE70
:10032000233A27EEA36A24EE057A67EE856AB0EEDB
:10033000462AF0EE432AA7EE242AE6EEE42AA6EEA9
:10034000247AE3EE646A24EE254A65EEE77A25EE28
:10035000655A65EEA35A81ED004AC1ED017AC1EDFF
:10036000024A81ED032AC1ED042A81ED055AC1ED4F
:10037000066A81ED077AC1ED085A08BDDFED093A3A
:1003800084E7DFED087ACAE79FED064ABAE7DFEDBA
:10039000054AA6E7DFED035A96E79FED025A82E78A
:1003A000DB0FC93F000000002DE9F04389B0541C69
:1003B00003941478002C00F0078100250746884636
:1003C0001E46A94609E021463846C047039A013532
:1003D000531C03931478002C3DD0252CF3D1931C8F
:1003E000CDE903395078302800F09480A0F1300333
:1003F000DBB2092B4FF0000440F297806C2838D014
:10040000782822D857282AD9A0F15803202B1CD8A5
:10041000DFE803F0B41B1B1B1B1B1B1B1B1B1B95CB
:100420009D1B1B1B1B1B1B1B1B1BAF1B1B1B1B1110
:100430001BA71B1BB40056F8043B049A009300232F
:1004400041463846FEF784FF0544039A531C039344
:100450001478002CC1D1284609B0BDE8F0830028EB
:10046000F9D02528F1D125213846C0470135039A16
:10047000AEE7039B5A1C039219787829A8D857290C
:1004800058D9A1F15803202BA2D801A050F823F08D
:1004900095050108D1030108D1030108D103010822
:1004A000D1030108D1030108D1030108D1030108D8
:1004B000D1030108D1030108D10301083F05010858
:1004C000AD050108D1030108D1030108D1030108DA
:1004D000D1030108D1030108D1030108D1030108A8
:1004E000D1030108D103010875050108D1030108F2
:1004F000D1030108D1030108D10301083704010821
:10050000D1030108B9050108D1030108D10301088D
:1005100095050108D31C03939078A0F13003DBB25A
:10052000092B4FF001043FF669AF04AA03A942F07A
:1005300003FB63E700298ED0252994D048E756F8BD
:10054000041B3846C9B2C0470135039A40E756F844
:10055000040B05A9FEF792FF05AB0093049A23460E
:100560006EE756F8040B05AB00220A21FEF73EFFAA
:10057000F2E7039A56F8043B1D6029E7A0F1580200
:10058000B2FA82F256F8040B520905AB1021FEF7BD
:100590002DFFE1E7A1F15802B2FA82F256F8040BFE
:1005A000520905AB1021FEF721FFD5E756F8040BE1
:1005B00005A9FEF763FFCFE756F8040B05AB002251
:1005C0000A21FEF713FFC7E7254644E773B5144C2D
:1005D00001920646D4F888000D46C0B11149FFF7D4
:1005E00029FAD4F888003146FFF724FA0E49D4F8E6
:1005F0008800FFF71FFA0D49019BD4F888002A46AE
:10060000FFF7D2FE0A49D4F88800FFF713FA94F8EE
:100610008C3013B1012384F88D3002B070BD00BF5F
:10062000706A00209D4006081E48060831FA00083E
:100630007D4A06080EB400B584B005AB019053F8AE
:10064000042B0649039301A8FFF7AEFE019B00228D
:100650001A7004B05DF804EB03B07047D1F30008E2
:100660002DE9F043002483B006460480214630463D
:10067000013436F0A5FB082CF8D10023DFF86880A0
:1006800086F8EA30C6F8EC30C6F8F030C6F8F43038
:10069000C6F8F8301F46FC3699463A46414601A84E
:1006A000FFF7C8FF3546032401AA12F8013B6BB1DE
:1006B000013C05F8013BF8D10137082F85F800907F
:1006C00006F10406E9D103B0BDE8F08328462246CE
:1006D00020212544013747F0E8FF082F85F80090D6
:1006E00006F10406D9D1EEE788FF0508F7B5114EEB
:1006F00007463046002300F88E3F0C460E4B0F494C
:10070000002F08BF1946154647F0D7FF0C4F04EBE2
:1007100045058E36AC4202D10A4803B0F0BD3946D9
:1007200034F8022B6846FFF785FF6946304647F0EC
:10073000C4FFEFE7706A0020B3400608AA4006082D
:10074000BC400608FE6A0020F7B50C4E0C4F002393
:1007500006F8BF3F044600EB4105AC4202D1094810
:1007600003B0F0BD394634F8022B6846FFF762FF4C
:100770006946304647F0A1FFEFE700BF706A0020EE
:100780004F4106082F6B0020F8B5084F4E1E054656
:1007900001F11F0416F8012F28463946FFF74AFFDA
:1007A000A64205F10205F5D1F8BD00BFC14006081B
:1007B0000246531C084605D1034B1A681B790A6090
:1007C0000B717047014935E70340060850410608A0
:1007D00010B5013114460EF0FFF828B9054B1A6820
:1007E0001B792260237110BD027A03492046BDE8BF
:1007F00010401FE7034006086440060803685A1CBF
:10080000026019700368090A5A1C02601970704767
:1008100002681146531C036011F802CB0160D31C1F
:100820005178036093781B0443EA0123111D016092
:10083000D07843EA0C0343EA00607047A0F130032C
:10084000092B07D920F02000413819288CBF00203F
:100850000120704701207047303809288CBF0020E4
:1008600001207047413819288CBF002001207047B3
:10087000613819288CBF002001207047202805D03E
:10088000093804288CBF00200120704701207047E0
:10089000A0F14103192B98BF20307047A0F16103EC
:1008A000192B98BF2038704710B500F1004402465C
:1008B000013C04E0B3EB0E0015D1A24214D012F8B3
:1008C000013BA3F14100192811F8010BA0F1410CE3
:1008D00098BF2033BCF1190F00F1200EEAD91B1A82
:1008E00004D10028E9D110BD002010BD184610BD6C
:1008F00002B310B58446841804E0B3EB0E0014D1A3
:10090000A44513D01CF8013B11F8010BA3F14102DF
:10091000192AA0F1410298BF2033192A00F1200EB4
:10092000EBD91B1A04D10028EAD110BD002010BD5C
:10093000184610BD1046704770B5044608460D466F
:1009400045F04EFD064602E014F8013F43B1204653
:1009500032462946FFF7CCFF0028F5D1204670BD6E
:100960001C46204670BD38B507490546FFF7E4FF31
:100970000649041E284618BF0124FFF7DDFF08B111
:1009800044F00204204638BDC64006086A560608F0
:100990002DE9F041044686469EF800C0BCF1200FC8
:1009A0007046ACF109050EF1010EF5D0042DF3D916
:1009B000BCF12B0F5BD0BCF12D0F3BD1102A4FF0B7
:1009C000010600F1010E58D19EF800C0BCF1300FB5
:1009D0005FD04FF010086FF070450F2742460EF1C0
:1009E000010E00200DE0ACF1300C5FFA8CFC944558
:1009F0000FDA854274462DD32AD008FB00C01EF8BA
:100A000001CBBCF1390FEED94CF0200CBCF1600FDA
:100A10000BD801B10C600EB323B1B0F1004F28BF69
:100A20004FF000404042BDE8F081ACF1570C5FFA56
:100A30008CFCDCE7102A864649D04FF0FF35B5FB29
:100A4000F2F502FB05F7FF43FFB290460026C6E72A
:100A50006745D2D21E404FF0FF30D0E7002BE2D0E6
:100A60006FF00043984228BF1846BDE8F081102A75
:100A70004FF0000600F1010EA6D04FF0FF35B5FB98
:100A8000F2F502FB05F7FF4390F801C0FFB2904674
:100A9000A5E79EF801C0ACF1410019280EF1010450
:100AA000624601D80CF12002782A4FF0100805D0D8
:100AB000A6466FF070450F27424690E79EF802C0A9
:100AC0006FF070450EF1020E0F27424687E70026B1
:100AD0007AE700BF01230A22002159E770B50D46CD
:100AE0001446FEF7B9FF0646A0B1FFF7F3FF40F644
:100AF00034039842A8BF1846B0F5617FB8BF4FF4E1
:100B00006170A0F561731920B3FBF0F32B702378AB
:100B1000013323703046FEF79FFF0646A0B1FFF772
:100B2000D9FF40F634039842A8BF1846B0F5617F5C
:100B3000B8BF4FF46170A0F561731920B3FBF0F3F7
:100B40006B70237801332370304670BD2DE9F0417E
:100B500017461E4605464FF47A7200233846314642
:100B600046F09CF84349444A014482FB0143C817BC
:100B70000B44C0EB631382FB03021A44D8173F4CAB
:100B8000C0EB621284FB02044FEAE27C3C48CCEBEF
:100B9000A40C80FB0C404FEAEC74C4EBE010C3EBF8
:100BA0000314A1EB8401A971C2EB0211A3EB810331
:100BB0006B710CEB4C03A2EBC30240F2B55303FB89
:100BC00010CCBCF5896F2A714FEA800044DA40F2FC
:100BD000DA239C4547DCBCF5B77FB4BF0022012275
:100BE000284B02EB420103EBC1034FEA4208B3F882
:100BF000523091B2244C08EB020E04EBCE041634B2
:100C00004FF00B0E01E034F8023D63451FDDBEF1ED
:100C1000010EF8D11B4B424403EBC2024FF0010E10
:100C2000938F85F802E000F5FA600CF1010C08449E
:100C3000ACEB030C288085F803C04FF47A720023D4
:100C40003846314646F02AF82A81BDE8F0810EF197
:100C5000010E5FFA8EFEE4E7032140F296530A4646
:100C60004FF00608C6E7022140F229430A464FF03A
:100C70000408BFE780BC92C789888888ABAAAA2AE3
:100C800073B06D16688F0508A48F050808B50C4B66
:100C9000D3E9002352EA030C09D1002340F20112E8
:100CA00042808380837103800381184608BD054913
:100CB00009688A1843F10003FFF748FF012008BDC7
:100CC00040400020B01E002090422DE9F0410B462C
:100CD000044615460AD2B0FBF5F6134A05FB164446
:100CE0001846135D00F8013BBDE8F081B0FBF2F659
:100CF0009642B6FBF2F706D20B4A05FB1767D15DA9
:100D000003F8011BEAE7BA42B7FBF2F807D9064A33
:100D100005FB187812F8081003F8011BEDE74046B0
:100D2000FFF7D2FF0346F2E790FF0508724B9A885F
:100D3000B3F808C058899989B2F57A7F88BF4FF413
:100D40007A7210B588BF9A80DA88B2F57A7F84BF4C
:100D50004FF47A72DA80BCF57A7F84BF4FF47A7CE4
:100D6000A3F808C0B0F57A7F88BF0020DA8988BF71
:100D70005881B1F57A7F84BF4FF47A719981B2F5C9
:100D80007A7F84BF0022DA8184459CBF00201881CD
:100D9000914298BF0022598B98BF9A819A8B9142B9
:100DA00084BF00225A83554B1A8882B0002A47D04C
:100DB000534CA179A37800296ED1062B97BF5148D7
:100DC0009FED510A00EB830090ED270A207998BB34
:100DD0004E4B93F8C00307EE902A07EE100AF8EE88
:100DE000E77AF8EEC76A86EEA77A00296AD1B4EEF0
:100DF000C07AF1EE10FA24D567EE807ABCEEE77A7D
:100E00008DED017A9DF8041007EE101AB8EEC77A3E
:100E1000F4EEC77AF1EE10FAC4BF0131C9B200296D
:100E200068D01029A8BF1021C9B281420A4638BF34
:100E3000024683F8C02304E0042B4BD8002B4CD18E
:100E4000324B334A5179022904BF002151715A7A39
:100E5000032A12D82F4901EB42111A7AC3F8C8139A
:100E6000032A12D82C4902EB8202C2EB021201EBD8
:100E70004202C3F8CC2302B010BD00225A721A7A83
:100E80002449C3F8C813032AECD9234AC3F8CC2356
:100E90000021197202B010BD072B8ED123790621D3
:100EA000A170002BCCD1194B9FED1C0A93F8C00305
:100EB00007EE902A07EE100AF8EEE77AF8EEC76A16
:100EC00086EEA77A30EE000AB4EEC07AF1EE10FAA0
:100ED000B7D591E7053B032BB2D9F7EE007A87EE41
:100EE000800A46F007FF2288084B904228BF104630
:100EF0002080A6E7012197E784250020840A0010BE
:100F0000E0260020688F05086F120338706A002001
:100F100050400020586B0020D86B002017B7D13804
:100F20002DE9F04F9B4E85B096F8D033A3F1170210
:100F3000022A00AF00F29582974BBB60DFF8608217
:100F400096F8E013DFF870B2944D08F16C0944464E
:100F50004FF0000A2FE00AF1010A5FFA8AFA43080B
:100F6000820802F0333203F077331344C20802F0F0
:100F70001132C31A9B1A03EB131303F00F33ABFBAD
:100F800003E2D209C2EB02229A1A830301D5012A95
:100F900019D0012A0BD9082A15D8BCF1000F01D0AD
:100FA000284204D1F96044F037FBF96858B10C3499
:100FB0004C4500F04F82206810F0010CCBD194F921
:100FC0000430142BCBD176480FF0AEF90024022068
:100FD00086F8804411F014FE96F88434022B00F059
:100FE000D482002800F028836E4B96F80DA503F5F7
:100FF000167B4FF47A7E4FF0000C5A88B2F57A7F58
:10100000B3F8462088BFA3F802E0B2F57A7F9A8849
:1010100088BFA3F846E0B2F57A7FDA8888BFA3F8E4
:1010200004E09988B2F57A7F84BF0022A3F806C055
:101030009142B3F85A10B3F85C2098BFA3F804C0EB
:10104000914293F86B2088BFA3F85AC0013A632AF3
:1010500084BF642283F86B2093F86C200132D2B2F3
:10106000092A88BF83F86CC003F166001946002284
:101070008D7A10F8014B0132A54238BF00F801CC3F
:10108000032A01F10601F3D1BAF1010F18BF83F869
:1010900084C096335B45B0D1434B9B78042B00F062
:1010A000A8823BB9404A1388B3F5F07F84BF4FF460
:1010B000F0731380FFF73AFE96F82715092902D03E
:1010C000002940F0E48196F83515092902D000295D
:1010D00040F0D981B6F84225B6F840351343B6F84A
:1010E000442513431BB213B10123A6F84635D6F8A5
:1010F000FC342E4A1A40002A00F0B482DA0700F1CC
:101100002B825D0440F1C7812949D6F800250B40A8
:101110000A40C6F8FC34C6F8002513F4004200F07B
:10112000FE81002286F8E72386F8F723D90440F1F0
:10113000008296F85335DFF87CB0022B04BF012300
:1011400086F853350BF178045B4602E006339C4287
:101150000CD01A78072AF9D19978DA78914202D31B
:101160005A79002AF2D0072024F0F2FA00234FF433
:10117000806086F8803411F043FD002800F04F8233
:101180000C4DAA469AF8051019B39AF80000F0B170
:101190005B4616E0706A0020688F0508BC020200FA
:1011A000806E0020D86B0020E0260020096000023D
:1011B000F6DFFFFDC86F0020818080800633A342E8
:1011C00007D01A788A42F9D15A79002AF6D024F049
:1011D000BFFA0AF1060AA245D4D1BA4B93F802B07D
:1011E000BBF1080F00F0C681B749D6F8FC34D6F839
:1011F00000250B40C6F8FC3496F80D35A3F1010329
:10120000B3FA83F35B0986F8D03596F80E35A3F16F
:101210000103B3FA83F35B0986F8D435B6F8E835F1
:101220001140C2F3C032C6F8001586F8D225002B53
:1012300040F0C981D6F8EC3513F07F4F1CBF002376
:10124000C6F8EC35D6F8F43523F4007323F0020326
:1012500013B10023C6F8F43596F8F035013B042BA2
:1012600084BF012386F8F035ABF1050B974BBBF13A
:10127000030F93F8901540F2498111B30023FB60EE
:10128000904B7C606FF00702A2EB030A544603F117
:10129000080B8A4604E004EB0B03534580F0FF8003
:1012A0001BF8010B0028F6D00DF0BEFB0028F2D091
:1012B000C3799B07EFD5FA687C680123002A40F0C8
:1012C000F480804B9B7913B17E4A00239371B6F86A
:1012D000FE3513F00C0F03D1C3F30313022B03D914
:1012E0004FF42063A6F8FE35B6F8003613F00C0F65
:1012F00003D1C3F30313022B03D940F60123A6F84D
:10130000003696F8793696F86D269A4296F86C363D
:1013100005D9002286F86D2653B1A6F8702696F8F6
:1013200078269A4204D2002386F86C36A6F87036E6
:1013300096F8623796F86E266548FC609A4288BF38
:101340000023BC6888BF86F86E3600F1800B10F869
:10135000043C03EB4303234493F890A193F891E1F9
:1013600093F892C1C31E1A785245A8BF524603F89B
:10137000012B59799A787145A8BF71466245A8BF7B
:101380006246984259719A70EDD120305845DED1AD
:10139000D6F80824FC68002A00F01F814FF0000CEA
:1013A000012002E00635A54211D02B78282BF9D177
:1013B0006B7800FA03F11142F4D00433063500FAD9
:1013C00003F3A54222EA03024FF0010CEDD1BCF178
:1013D000000F01D0C6F808243E4C04F1080523464E
:1013E00013F8012B072A00F283809D42F8D1EA46C8
:1013F00088B0EB462022FF21584647F056F9354A7F
:1014000012F8013B5BF82310013178D195424BF87B
:101410002330F5D1B6F80625B6F804359A42D546FC
:1014200002D32D4BC6F80435FF232C4986F8943798
:1014300098F90430142B05D0D8F8002031EA0202C4
:1014400000F0D18008F10C08C845F1D11437BD4631
:10145000BDE8F08F0AF1FF3ABAF1020F7FF6B6ADA0
:10146000B1E51F4ABA6002EBC30393F8B820002A23
:101470003FF464ADD3F8BC30002B7FF45FAD17238D
:1014800086F8D0335AE51748FEF7CCF922E616481D
:10149000FEF7C8F917E61C0767D5144935E6FA6860
:1014A0007C680023002A3FF40CAF06494A7C002ADE
:1014B0007FF40DAF4A79012A3FF403AF002B7FF48C
:1014C00000AF04E7E0260020DEDDCDFD840A001039
:1014D0005E6B0020F3260020AE014A0101000200ED
:1014E000688F0508A66F0020986F0020FE9FFFFD03
:1014F000EA4688B02022FF21684647F0D6F800234C
:1015000004F8013B0133082BFAD183E75B4A00233F
:101510001371002900F09D800123FB60B0E696F86E
:10152000E71300293FF402AED90486F8F7233FF50C
:1015300000AE1A067FF5FDAD96F8D013182906D82F
:101540004F4B01228A401340002B7FF4F2ADDFF8AD
:1015500040B10BF1780409E64A49D6F800250B4062
:101560000A40C6F8FC34C6F8002598047FF5D5ADCE
:101570004549CAE51A469B79002B3FF435AE537CAA
:10158000012B04BF022353742EE600283FF42CAD38
:101590003E4B96F88D1490F904504FF0FF0C03F178
:1015A0006C0093F90820AA4204D1013983F808C0DD
:1015B000C9B201240C338342F3D1002C3FF414ADA3
:1015C00086F88D1410E596F8E4050DF02DFA002844
:1015D0007FF430AEA6F8E8052CE6282024F0B8F811
:1015E000D6F80824DAE6143786F89437BD46BDE805
:1015F000F08FD6F8FC34214A23F48053C6F8FC342B
:10160000D6F8003523F48053C6F80035538CB3F573
:101610007A7FBFF44FAD4FF47A7353844AE5D6F81E
:10162000FC3423F00063C6F8FC34D6F8003523F010
:101630000063C6F80035A3E5D6F8FC24D6F80035DB
:1016400022F0800223F08003C6F8FC24C6F800359F
:10165000CAE4537C002B7FF43AAE5379012B7FF41C
:1016600036AE2EE6D6F8002543F0080342F0080215
:10167000C6F8FC34C6F8002540E500BFE02600208F
:1016800000410001F79FFFFDF6BFFFFD006F002046
:10169000C86F00202DE9F04F754F764BD7F8A4277F
:1016A00002F2DC52C7F8A427734A934283B080F059
:1016B000DB8003F11C059B46704B714E4FF0010A15
:1016C00003F102086D4B5A88002A00F0B68008EB3F
:1016D0000203B34280F0B180444608E01A881C46F9
:1016E0001344002A00F0A980B34280F0A680052AA6
:1016F00040F2A38035F81C2C6188C2F30B029142A2
:10170000ECD162799207E9D1238855F8141C94F83A
:10171000049001935846FEF753FB35F81C2CB9EBA7
:10172000123F00F092804FF0000A35F8181C55F86F
:10173000140CC1F30B0140F0EDFB55F8043C1860AC
:101740004D4B0BF11C0B9B4505F11C05BAD3D7F88B
:10175000FC34C7F80035FFF7E3FB3B7A494D797A53
:10176000494C03EB8303C3EB0313A5F1800202EBA7
:10177000411205EB4303C7E9F22323F087FA4FF048
:10178000FF33D7F8CC03636029F000FC24F034F871
:1017900005F57C7305F58D6102E006338B425ED062
:1017A0001A78002AF9D19D78D878854202D35879E1
:1017B0000028F2D097F85035227203EB830303EB35
:1017C00083039B00C72BD8BFC823C7F89C37B7F843
:1017D00054352E49642202FB03F3C72BD8BFC8231C
:1017E0000022C7F8A037C7F8B837294BC7F8A42795
:1017F000C7F8A827C7F8AC27C7F8B027C7F8B42799
:10180000A7F8BC2787F8BE27C1F804372DF0A4FC41
:10181000B7F8C00797F8C21725F030FF36F0D8F8B0
:1018200017F0D8FE1B4A1268C7F8A42701235046B8
:1018300087F8BD3703B0BDE8F08F55F8141C584643
:10184000FEF7BEFA4FF0000A6FE7019BA11D9A1F39
:101850005846FDF775FC00287FF467AF63E7FA7D13
:10186000003A18BF0122A5E74FF0010A6FE700BF59
:10187000706A0020708706086C8F06080040000818
:1018800000800008D86B0020A4050020840A001006
:10189000B06F0020B01E00201C4B0122032870B541
:1018A0001B4D83F80C2706461ED9711CC9B249008E
:1018B0004029184A28BF4021002302244FF0140E6B
:1018C000D454023302EB030C99420CF801ECF7D824
:1018D000FF2E08BF02212944FF2381F8C437BDE849
:1018E00070400E2016F028BA00EB800005F5B473A6
:1018F000C0EB001003EB4000C5F8CC032E7229F0BA
:1019000045FB26F09FF926F073FACEE7840A001013
:10191000706A002034720020054BD3F8082801219A
:1019200042F4001283F80518C3F80828704700BF76
:10193000706A0020F8B50468C4F30D0406460F462B
:101940000CB335683F683DF0DDF9092840F0878029
:10195000444C236923F440732361236943F40073E7
:101960002361236943F0010323612F603DF0CAF92D
:101970002369092823F00103236170D133680433FC
:101980003360002034E0384B384A93422AD302F5C2
:101990008042934225D302F58042934229D3344AB0
:1019A000934228D902F58032934226D902F50032BB
:1019B000934224D902F50032934222D902F5003233
:1019C000934220D902F5003293421ED902F58022BB
:1019D00093421CD9B3F1016F1BD341F059FE44F07F
:1019E000F7FC08243DF08EF9092814D04FF0FF30A1
:1019F000F8BD1024F6E71824F4E72024F2E72824A1
:101A0000F0E73024EEE73824ECE74024EAE7482406
:101A1000E8E75824E6E7134D2B6923F440732B6164
:101A20002B6943F400732B612B6923F0F8032B61BE
:101A30002B691C4344F002042C612B6943F480336E
:101A40002B613DF05FF92B6923F002032B612B69B9
:101A5000092823F0F8032B613FF473AFC6E76FF05A
:101A60000100C5E7003C02400040000800400008BB
:101A7000FFFF00082DE9F041574F3B78AF2B8AB0AC
:101A80006FD1FDF7FBFD80F00104E4B2534B544DE0
:101A9000B3F89F31534EADF8003004F00104B54265
:101AA00061D3002C00F096801022002106A846F099
:101AB000FCFD4D4B0497DB1B05934C4B1A69002A28
:101AC00004DA4B4A5A6002F188325A6001228DF8DA
:101AD0002420F322DA606946022204A80025089532
:101AE00044F054FA022269464FF6FF70FDF788FB76
:101AF0003B4F0446B74243D3022201A904A8002564
:101B0000ADF8045044F042FA022201A92046FDF744
:101B100077FB40BAC043ADF80800022204A802A92E
:101B200044F034FA079868B106ABC0F104022946C4
:101B3000184446F0BAFD089818B906A904A8FFF79A
:101B4000F9FE08909DF82430089823B1274A1369BC
:101B500043F000431361B0FA80F040090AB0BDE8D9
:101B6000F081012492E7A988A868C1F30B0140F035
:101B7000D1F9AB691B681C35834218BF01248EE77D
:101B8000B7F804808DF80D50C8F30B0808F1060370
:101B9000ADF808303B88C3F30B02ADF80A201B0BED
:101BA000062202A904A88DF80C3044F0EFF90622B1
:101BB00002A92046FDF724FBB9680446424604A862
:101BC00044F0E4F9B96820464246FDF719FB1C379A
:101BD00004468FE70120C1E700400008688F050830
:101BE000708706086C8F060800800008003C0240E1
:101BF0002301674510B5194CFFF792F9D4F8A437C3
:101C0000012203F2DC53C4F8A43784F80C28FFF750
:101C100031FF10B9FFF72EFF50B1114B1B78AF2BDE
:101C200002D1FDF72BFD58B941F032FD44F0D0FB55
:101C3000FFF720FF0028F0D141F02AFD44F0C8FB57
:101C4000084A0023116884F80C380122C4F8A4174C
:101C500084F8BD2784F80D3810BD00BF706A0020DD
:101C600000400008B01E002010B50B4A0B4C0223A8
:101C70000121A37582F80C17FFF7BCFFFFF70AFDDF
:101C800041F20242FF23A4F8C42784F8C6370E208D
:101C9000BDE8104016F050B8840A0010706A0020A9
:101CA00090F88630DFED6A5A03EE903A90F88A3069
:101CB00006EE103A90F8883004EE103A90F8893029
:101CC000F8EEE33A04EE903A90F88C3063EEA57AA1
:101CD000B8EEC66A03EE903A26EE256AB8EEC44A1C
:101CE000F8EEE44AF8EEE33A26EE276A24EE254AB7
:101CF00064EEA54A63EEA53AF0B5564D24EE064AC9
:101D000064EEA74A63EEA73A00210626F7EE002A02
:101D1000A5F10C0C00F1660E06FB01F2B7EE005ABD
:101D2000AC1890F885700244F0EE456A15E0012980
:101D300004F1060402F10602EED190F8873007EEB6
:101D4000903A90F88F3006EE903AF8EEE77AF8EE97
:101D5000E66A27EEA55A66EEA56A237807EE103AE2
:101D600066EE867AB8EEC77A27EE277AFDEEC77A56
:101D700017EE903AFA2BA8BFFA2323EAE373137203
:101D8000637807EE103A66EE847AB8EEC77A27EEEB
:101D9000277AFDEEC77A17EE903AFA2BA8BFFA23FE
:101DA00023EAE37353725CF8213007EE903A002B7C
:101DB000F8EEE77A49DDA37807EE103AB8EE477AF5
:101DC00090F88B3037EE677A03EE103A87EE272AC9
:101DD000B8EEC33AB0EE627A23EE253AA2EE037A69
:101DE00064EEA77A66EEA36A67EE857A27EE877AB5
:101DF000FDEEE77ABDEEC77A17EE103AFA2BA8BFD0
:101E0000FA2323EAE373937217EE903AFA2BA8BFF2
:101E1000FA2323EAE3730EF80130A38807EE903A21
:101E2000F8EEE77A013167EEA67AFDEEE77A17EE73
:101E3000903AB3F57A7FA8BF4FF47A7323EAE3733D
:101E40008F429381BFF673AFF0BDB7EE007AC7E75C
:101E50000AD7233C4493050890F88D306BB3B0F853
:101E60005A308BB190F88E2002EB82036421C3EBD1
:101E70000313B3FBF1F3A0F85A30962312FB03F3DC
:101E8000B3FBF1F3A0F85C3043884BB190F88E308F
:101E900003EB8303C3EB03136422B3FBF2F343802E
:101EA000B0F846304BB190F88E30962213FB02F317
:101EB0006422B3FBF2F3A0F84630704790F821306B
:101EC0004BB3438B83B190F82230FA2213FB02F21A
:101ED00003EB8303B3F57A7FA8BF4FF47A736421D1
:101EE0008383B2FBF1F24283838843B190F82230BE
:101EF000FA2213FB02F36422B3FBF2F38380C3885C
:101F00004BB190F8223003EB8303B3F57A7FA8BF7F
:101F10004FF47A73C3807047034BD3F8440D08B174
:101F200007F06ABC704700BF706A002008B50B4616
:101F300005490246D1F8440D28B10449FEF734FAA8
:101F4000BDE80840E8E708BD706A002031FA0008E3
:101F5000024B0146D3F8440DFDF76CBD706A0020BA
:101F600008B504460848FFF7F3FFFFF7D5FF074B16
:101F7000D3F8800015F05EFE0CF020F8012C01D1A2
:101F800044F026FAFBF7A2FCCE400608706A002057
:101F90000048DDE7944B06080CB4C30607B500D52E
:101FA00061B9049805A90191FFF7C0FFFFF7F0FFA1
:101FB000012003B05DF804EB02B070470020F8E7A1
:101FC00008B5FFF7C5FFBDE80840E1E710B50446D6
:101FD0000348FFF7BDFF2046BDE81040F0E700BF13
:101FE000DA40060808B50948FFF7F0FFFFF794FF4D
:101FF000074B002483F8484DC3F8484E83F84C4EF5
:1020000025F096FF2046FFF7ABFF00BFDF40060834
:10201000706A0020034B0146D3F8440D08B107F065
:10202000D7BB7047706A00200CB407B510F02000D1
:102030000BD079B92320FFF7EDFF049805A9019192
:10204000FFF774FFFFF7A4FF012003B05DF804EB76
:1020500002B070470020F8E70FB407B504A951F8A3
:10206000040B0191FFF762FF03B05DF804EB04B0CD
:102070007047154B1B6870B52BB31448144EFFF70F
:102080009FFFFFF749FFFCF73DFA0025FCF770FAC8
:10209000044640B1132015F04FFEFFF779FFBDE86D
:1020A00070400C488CE73046FFF7D6FF782D06D8F5
:1020B0000135FFF731FF64200BF0DAFFE6E7FFF7A9
:1020C00067FF2546F5E770BD681E0020064106083B
:1020D0007E6C0608204106080FB407B504A951F824
:1020E000040B0191FFF722FFFFF752FF03B05DF8E9
:1020F00004EB04B070472DE9F041037903F0E002EE
:10210000402A4AD004D85AB1202A23D0BDE8F08111
:10211000602A45D0802AF9D18279417922480BE0A2
:1021200003F00703022B02D0042B08D06BB9B0F8E0
:102130000720B0F805101D48BDE8F041CCE7D0F805
:1021400005101B48BDE8F041C6E7B0F90720B0F91B
:102150000510F0E74679174D174805EBC605FFF760
:10216000F7FE95F8F47300240123A74202D8BDE8D6
:10217000F0410DE7D5F8F06356F824204FEA8408C3
:102180004AB113B90D48FFF7E3FE56F808100C48A2
:10219000FFF762FF00230134E7E741790948D1E7FF
:1021A000BDE8F041084897E7784106083C41060839
:1021B00026410608688F0508534106086441060851
:1021C000F3560608674106088F4106082DE9F043DB
:1021D00087B0FCF787F902698389018802928268D7
:1021E00001924288009242681B4EDFF880801B4FAC
:1021F000DFF87C9004461A48FFF76EFF002515B9FA
:102200004046FFF7DDFE3B689D4213DA3378154800
:10221000052B96BF09EB83030022D3F89825B388DA
:102220000093294673880135FFF756FF062D06F106
:102230000606E4D140F0A6FC81884388CB1A616889
:1022400003FB01110591FCF7D7F9059902460648F1
:1022500007B0BDE8F0433FE718400020883F00206A
:10226000A741060811420608204206080542060852
:10227000688F05080249034801F521610EC92BE763
:102280000070FF1F3D42060810B5752104462DF071
:1022900009FA01460948FFF71FFF1A2120462DF0D1
:1022A00001FA01460648FFF717FF1B2120462DF0D3
:1022B000F9F9BDE81040014602480DE75142060811
:1022C000644206087742060838B50B4DE87810F0EE
:1022D000FD0405D10948FFF7FFFE2046FFF7D4FFB4
:1022E000EB78013B012B06D80548FFF7F5FEBDE86A
:1022F00038400120C8E738BD842500208A420608FE
:10230000954206082DE9F04F764B77491A687748D1
:10231000774BB2FBF3F299B0FFF79EFE754BDFF8F7
:1023200044C20FCBDCF808400CAF87E80F00724BBB
:102330000793A608714B089316F00206C4F38104B4
:1023400018AB18BFDCF8045003EB840318BFC5F3C7
:10235000805553F8301C002E00F0C28018AB03EB00
:10236000850555F8442C664C6648674F674EDFF884
:10237000F881DFF8C091FFF76FFEB4F84E2E4FF4EE
:102380007A73B2FBF3F103FB11220A20B4F9503E39
:1023900092B2B2FBF0F25E48FFF79EFE5D4A5E49E4
:1023A0005E48FFF759FEFFF7F3FDA17D5C4A5D4BE8
:1023B0005D4807EB8101D31AD1F8C015A288FFF759
:1023C0008BFE5A48FFF7C4FD94F8521E5848FFF799
:1023D00043FE5848FFF7BCFD94F8531E5648FFF7DC
:1023E0003BFEFFF7D5FD5548FFF7B2FD00210A4639
:1023F000F37F0B4113F0010F01F1010508D012B179
:102400004846FFF7A5FD29464046FFF725FE012275
:10241000072D2946ECD14A4D95F86A1505F5EC7360
:1024200005F13C02012918BF134693F8DC30032B59
:1024300002D04448FFF710FE434B95F86A15A3F508
:10244000CE72012918BF134693F8DC30012B02D15C
:102450003E48FFF701FE3C4B95F86A15A3F5CE7296
:10246000012918BF13461B695B7B012B02D9384831
:10247000FFF7F2FDDFF8F480DFF8F4B0FFF788FD36
:10248000D4F8543E0393002608F1200958F8041BA1
:1024900000296FD0012303FA06FA039B1AEA030FFF
:1024A0001CD01AF01F0F19D02A4B59F82620985D1E
:1024B00052F8202036B12848CDE90412FFF748FD34
:1024C000DDE904125846FFF7C7FDBAF1020F05D146
:1024D00095F8311A11B12148FFF7BEFD0136D5E755
:1024E0001F4A40E7E8180020A0420608A542060857
:1024F00040420F0018950508C2420608C742060868
:10250000706A0020CC420608688F050884250020E8
:10251000D4420608F0FF001000080000F54206084B
:1025200000800008004000081943060848430608D8
:102530005A43060862430608644306086C430608CB
:10254000840A0010854306085C0C00108D430608C1
:1025500092430608C005002064410608A04306080F
:10256000964B0608003802407C430608349505085F
:102570009A430608FFF70CFD94F8A21CD4F8A42C8B
:102580004F48137A527A07EB8101D1F80016FFF712
:10259000A3FD4C494C48FFF75FFD4C494C48FFF701
:1025A0005BFDFFF7F5FC4B4B4B4819684FF47A7312
:1025B000B1FBF3F1FFF750FD09A8FEF767FB38B157
:1025C00009A910A843F010FE444810A9FFF744FDE4
:1025D000FFF7DEFCD4F8E02E002A5ED007EE902A4A
:1025E000DFED3F6AB8EEE77AC6EE877AFDEEE77A6E
:1025F00017EE903ADFF80881B8F8600458B107EE9A
:10260000900ADFED376AF8EEE77A86EEA77AFDEEFC
:10261000C77A17EE900AD4F8606E5EB107EE906A42
:10262000DFED2F6AF8EEE77A86EEA77AFDEEC77A3D
:1026300017EE906AB5F86C1A6429A8BF6421CDE939
:1026400000062848FFF748FD98F8623498F863249C
:10265000B8F86414244807EB8303D3F81436FFF763
:102660003BFD224B2248198889B2FFF735FDFBF765
:1026700039FF016921B182681E48120DFFF72CFD58
:102680001D481E4EFFF764FCD4F80848012534B9F4
:10269000FFF77EFC19B0BDE8F08F1346AAE794FA65
:1026A000A4F3B3FA83F305FA03F207EB830330468E
:1026B000D3F8281624EA0204FFF7CEFCE7E700BFB0
:1026C000A4430608B6430608D7430608E5430608B0
:1026D000EB430608B01E0020F14306080B44060831
:1026E000002474491E44060864440608A8260020F5
:1026F0008B4406089A440608B54406087048060844
:10270000687B00202DE9F04FDFF8788198F80B30D6
:1027100099B0002B00F098805148524EDFF868B114
:10272000DFF86891DFF868A1FFF74AFC00252F4623
:102730000BA9E8B217F098F99DF83430002B53D06C
:10274000139C54B107EE904A9FED470AF8EE677A62
:1027500080EE270A45F0CEFA04460B9A29465846E1
:10276000FFF77AFC109A002A70D002FB04F04FF4B5
:102770007A73B0FBF3F30993DDF848C0BCF1000FA6
:1027800066D00CFB04F142F21073B1FBF3F198F840
:102790000B30082D18BF7F18002B5BD017980790BF
:1027A00015980690169805900A2311984FF47A7E92
:1027B000B0FBFEFE0998CDF810E0B1FBF3FE03FB81
:1027C0001E11CDE902E10999B1FBF3F103FB110000
:1027D000CDE90010BCFBF3F321465046FFF77CFC2B
:1027E0000023C6E90D33B36201351C2D06F1400606
:1027F0009ED198F80B3023B31C4C1D48D4F870249C
:10280000D4F86C14D2084FF47A73B1FBF3F3D4F814
:102810007414FFF761FC0A221648B7FBF2F102FBC1
:102820001172FFF759FC144B1B78432B06D1D4F8D7
:102830007824D4F87C141148FFF74EFC0023C4F828
:10284000743419B0BDE8F08F0D4866E7099293E73C
:1028500061469CE721464846FFF73EFCC0E700BFC3
:10286000CB440608C87800208096184B687B00206F
:102870007245060892450608B4210020B6450608B0
:1028800029450608706A0020334506085158060895
:102890004245060838B52A48FFF75AFB294B93F8FA
:1028A000F933002B49D0284C2848FFF789FB94F8CE
:1028B000D43A2BB194F8DA3A13B194F8D53A43B933
:1028C000B4F8E05A2248FFF743FB2DBB2148FFF73D
:1028D00077FBB4F8D61A2048FFF7BEFB94F8D43A39
:1028E0002BB31E48FFF76CFBB4F8DC1A1C48FFF74B
:1028F000B3FB94F8DA3AE3B11848FFF761FBB4F898
:10290000D81A1848FFF7A8FB94F8D53A9BB113489A
:10291000BDE83840FFF754BB4FF47A72B5FBF2F1D3
:1029200002FB1152104892B2FFF7D6FBD1E70F48D5
:10293000D8E70E48E1E70D48EAE70D48E8E700BFB1
:10294000E0450608706A0020840A0010F645060873
:10295000FD450608184606082C4606084C4606089B
:102960005C460608764606082246060855460608CE
:10297000948406080EB403B503AA52F8041B01920E
:10298000FDF724FE064BD3F8442D22B90549D3F8B0
:102990008800FDF74FF802B05DF804EB03B0704714
:1029A000706A0020944B06082DE9F04715460A7915
:1029B00002F0E004402C81460F4698462DD1DFF806
:1029C00078815C4EDFF89491002415E03B7903F0A8
:1029D0000703013B032B03D8DFE803F01315181B93
:1029E000295D3046FFF738FB7B79013BA34202DDCE
:1029F0004846FFF7ADFA01347B79A342E6DCBDE837
:102A0000F0872957EDE735F81410EAE735F9141087
:102A1000E7E755F824104046E4E702F00702042AED
:102A20003ED8DFE802F0030C141619002E78602C53
:102A300044D02BD8002C4CD0202C61D0DFE795F966
:102A40000060602C3AD021D8002CF5D12EE02E88E1
:102A5000EDE7B5F90060F4E7D5F800A0202C564664
:102A60004ED011D8002CCAD151463348FFF7F4FAA2
:102A7000D7F805108A4553D8B8F1000FBFD02F48BA
:102A8000BDE8F047FFF7E8BA602C17D0802CB6D12C
:102A900029782B4B2B48002914BF29461946EFE70C
:102AA000202C2CD007D8002CA9D12646B7F90540F8
:102AB000B7F9075011E0602CE8D100267B7946FA7F
:102AC00003F3DB07BDE8F0474CBF1F481F48FFF783
:102AD000C3BAB7F80540B7F8075016483146FFF7B4
:102AE000BBFAB4421CDCB5421ADBB8F1000F86D049
:102AF0002A4621461648BDE8F047FFF7ADBA002642
:102B00007A79144B03EBC20393F8F423B24207DD46
:102B1000D3F8F03353F82600BDE8F047FFF718BAB2
:102B2000FFF736FA3A680C4933464846BDE8F047A5
:102B300020E700BF504106083941060896460608BE
:102B4000FA6C0608F3560608A441060894840608A1
:102B5000CE3F0608688F05089C46060862430608B3
:102B600013B50446084601920091FDF7CDF8DDE962
:102B700000130246204602B0BDE8104014E70EB430
:102B800003B503AA52F8041B0192FDF71FFD054B84
:102B90000549D3F88800FCF74DFF02B05DF804EB5F
:102BA00003B07047706A0020944B06080149024642
:102BB000E5E700BFB6460608F8B5064608460C46E7
:102BC000FDF788FF20210546204645F085FD044697
:102BD00018B93046BDE8F840E8E7114F114E3B7890
:102BE00032789A4201D0FBF7BFFD0F4B20461D60A3
:102BF00043F0F6FB012201462046FBF75DFD3B78E2
:102C000032789A4201D0FBF7AFFD204643F0E8FB53
:102C10002A460146BDE8F8400448FFF75DBA00BF08
:102C2000641E0020903F0020601E0020CD46060854
:102C30002DE9F041064688B008460D46FDF74AFFEB
:102C400020210446284645F047FD20B9304608B00B
:102C5000BDE8F041AAE7FDF73DFF224605460146E3
:102C60000F48FFF739FA85B1202D2A46694628BF5B
:102C700020222046FBF794FDE84606460027B7428F
:102C800008DBAD1B3444002EEDD1FFF781F908B00D
:102C9000BDE8F08118F8010BFFF7BCF90137EEE74A
:102CA000E346060810B504460748FFF789F9FBF725
:102CB00017FE20B1BDE810400448FFF781B9204657
:102CC0000349BDE810405AE7FB46060805470608D9
:102CD0000D4706082DE9F041144BD3F88C3988B024
:102CE0000446F3B11A6804A9D56A18466A46A8478B
:102CF000064688B1DFF8408004AC6D46002735F801
:102D0000022B34F8021B40460137FFF7E5F9BE42BB
:102D1000F5DC08B0BDE8F08105492046FFF72FFF3C
:102D2000F7E7044908B0BDE8F04128E7706A0020E1
:102D30002E470608464706081447060813B50446FA
:102D40000846019143F04CFB024670B1112804D1B2
:102D50000199094845F0D5FC38B1074B074A0849A5
:102D6000204602B0BDE8104009E70349054802B01B
:102D7000BDE81040FFF7B0B968FF05084D470608E9
:102D8000584706088247060813B5044608460191CD
:102D900043F026FB0199024668B1042803D1094893
:102DA00045F0AFFC38B1074B074A0849204602B04E
:102DB000BDE81040E3E60349054802B0BDE8104015
:102DC000FFF78AB960FF05089047060858470608CC
:102DD000A04706082DE9F04306469BB008460C467E
:102DE00043F0FEFA002705461C22394602A8019747
:102DF00045F05BFC25B3402D07D0394940232A46D6
:102E000030461BB0BDE8F043B9E60DF1040804F10B
:102E1000400902222146684645F087FC0023102223
:102E200009A968468DF80270FDF7B2FD099B0DF106
:102E30000202934222D10234A14508F8010BE8D1E5
:102E400000213D220AA8099145F02FFC002D3AD01F
:102E5000244C257ED5B1202204F11C0101A845F0A7
:102E6000FAFB98B104F11C0109A8FDF78DFC1E4A7C
:102E70001E4909AB3046FFF782FE04E01A781C4970
:102E80003046FFF77CFE1BB0BDE8F08394F8843039
:102E9000CBB9C5B901AD0FCD164C0FC495E80F00E5
:102EA00084E80F00144B012209A8A4F1100183F853
:102EB0008024FDF769FC1148FFF788F8104809A93C
:102EC000FFF70AF9DFE70C4B93F880341BB9054B89
:102ED0001B7E002BF2D0074909A8FDF755FCEDE752
:102EE000B3470608706A0020F147060858470608ED
:102EF000D54706088C6A0020687B0020FB4706083F
:102F00000A4806082DE9F74F834608460D4643F068
:102F100067FA3B4F0446D7F8FC94B8B939483A4DA4
:102F20003A4FFFF715F8012655F8041B49B106FA88
:102F300004F313EA090F02D03846FFF78DF8013485
:102F4000F2E703B0BDE8F04FFFF722B80246304980
:102F50002846FDF7CDFC78B92E482B4C2E4DFEF7B8
:102F6000F7FF54F8041B0029EBD00B78002BF8D0A6
:102F70002846FFF771F8F4E72B782D2B224B03BF7F
:102F8000013504F1FF344FF0010A4FF0000A00262A
:102F900053F8048BB8F1000F06D120492A46584651
:102FA00003B0BDE8F04FEAE52246414628460193CA
:102FB000FDF79EFC019B00BB0123B3409A0505D59C
:102FC000174803B0BDE8F04FFEF7FABFBAF1000FA3
:102FD0000DD029EA03031348C7F8FC34FEF7B8FF05
:102FE0000D48414603B0BDE8F04FFFF775B849EA18
:102FF00003030D48C7F8FC34F0E70136C8E700BF0B
:10300000706A002017480608F89505082148060848
:103010002E45060825480608704806083048060868
:10302000414806084D480608564806082DE9F74F5E
:10303000814608460E461746984643F0D1F90446A5
:10304000E8B93F483F4DFFF707F820460FF0E4FB93
:103050003B68184206D020460FF0F0FB0146284698
:10306000FEF7FAFF0134182CEFD13B6813B936484C
:10307000FEF76EFF03B0BDE8F04FFEF789BF0246D2
:1030800032493046FDF734FC0546A8B93048FEF712
:103090005FFF2C462F4D20460FF0BEFB10EA080FB5
:1030A00006D020460FF0CAFB01462846FEF7D4FFA3
:1030B0000134192CEFD1DDE733782D2B48F08073E4
:1030C00003BF013604F1FF34012500254FF0000A4B
:1030D000019350460FF0B2FB22468346014630462C
:1030E000FDF706FC00BB50460FF096FB019B034228
:1030F0001AD08DB1BAF1180F1CBF3B6840EA030823
:103100001548C7F80080FEF723FF1248594603B060
:10311000BDE8F04FFEF7E0BFBAF1180F1CBF3D68E5
:1031200085433D600D48EEE70AF1010ABAF1190F37
:10313000CFD10B493246484603B0BDE8F04F1EE5FB
:103140005E4806086F480608684806082E450608C7
:1031500025480608704806084D48060856480608DF
:1031600030480608014A40F202235FE764700020FD
:10317000014A6FF07F4359E75C70002070B5054647
:1031800008461646FDF7A6FC0D4B93F89025904295
:10319000044605D201460B48FEF79EFF204670BD4F
:1031A0002EB1FF2803D10848FEF796FFF6E707493E
:1031B000013A2846FFF7E3FC4FF0FF34EEE700BF8B
:1031C000840A0010744806088548060898480608CE
:1031D0002DE9F04F074691B08248834D0E46FEF729
:1031E0007BFF8249C5F884D4002385F88834062201
:1031F000012391F890153046402485F889440AF05F
:10320000A7FD0A200AF034FF95F888340C2BDAB2B7
:1032100040F2E4809DF80C50FE2D30D0FF2D0BBF06
:1032200015240F2401260026944240F0D780611E09
:10323000C9B2684639F0F2FC04F140030DEB030417
:1032400014F8413C834240F0C48006F1FF385FFA35
:1032500088F8B8F1010F9DF80D3012D903F01F075F
:1032600061375C096248FEF773FE022E6AD0013CAA
:10327000042C65D8DFE804F00B5E6064620002266F
:10328000D2E79DF80E709DF80F401D46EAE75948B9
:10329000DFF8BC91DFF8BCB1FEF792FE5648FEF7AE
:1032A00057FE6C464FF0000A14F8011B48460AF11D
:1032B000010AFEF7D1FEBAF10C0F49D1FEF768FE04
:1032C000022E4FD06422B5FBF2F102FB11524B48A3
:1032D0003B46D2B2C9B2FEF7FFFEB8F1010F71D87A
:1032E000474A484B9DF810104748484D002914BFE5
:1032F00011461946FEF7F0FE9DF81110444B454863
:10330000002914BF19462946FEF7E6FE022E59D1C0
:103310009DF812404048FEF71BFE4CB3FF2C37D0FF
:103320000A22B4FBF2F102FB11423C48D2B2FEF792
:10333000D3FE20E03A48ABE73A48A9E73A48A7E786
:103340003A48A5E700238DF83F300DF11F009FE7B5
:10335000374B03FB0AF2B2F1553FA5D85846FEF7AA
:10336000F7FDA1E733483A462946FEF7B5FEB7E731
:103370002846FEF725FE9DF813402F48FEF7E8FD8E
:1033800044B1FF2C21D02D482146FEF7A5FE04E0D4
:103390002B48EEE71D48FEF713FE1C4E284FDFF8C2
:1033A00070800DF11305002415F8013F7BB1FF2B50
:1033B0000CBF3A464246214622480134FEF78CFEB5
:1033C000042CF1D111B0BDE8F08F1D48E3E732467F
:1033D000F1E71D493846FFF7D2FBF3E71B48FEF73C
:1033E000EFFDEFE7DE480608687B0020840A001046
:1033F000EF480608FA480608284906083A49060828
:10340000BE480608C748060871490608CE4806089F
:103410003D560608884906088F490608A34906084C
:103420000149060809490608114906082049060805
:10343000ABAAAAAA56490608AB4906085041060895
:10344000D2480608BB490608C6490608D6490608F8
:10345000C1400608FA6C06082DE9F84FDFF8A8808D
:10346000DFF88890DFF8A4A007460C46204642F01B
:10347000B7FF064660B91D4B1D4893F8D0231D4B7E
:1034800003EB8203D3F80817BDE8F84FFEF724BE1C
:10349000024641462046FDF72BFA60B1DFF860B0E6
:1034A00000255BF8041BB1B9224638461249BDE835
:1034B000F84FFFF764BB1148114C124DFEF748FD61
:1034C00054F8041B19B12846FEF7C6FDF8E7BDE81D
:1034D000F84FFEF75DBD32462046FDF709FA01358B
:1034E0000028DED189F8D0535446BFE7706A002027
:1034F000DF490608688F0508304806082548060891
:1035000074960508704806082E450608964B06086E
:1035100038B50D4604461A4905222846FDF7E8F954
:1035200068B9184B93F88C2022B9012183F88C10CC
:1035300083F88D20BDE838401348FEF741BD13499C
:1035400003222846FDF7D4F9A0B90E4D95F88C302A
:1035500063B195F88D304BB10D492046FFF70FFB55
:10356000002385F88C3085F88D3038BD0948FEF78A
:1035700027FDF5E720460849BDE83840FFF7FFBAC8
:1035800084550608706A0020E9490608E6560608D0
:10359000FF490608364A06084A4A060808B503469F
:1035A00010462AB1DB0600D511B1FEF70FFD002051
:1035B00008BDF8B50D4E96F88430054693B9F8BDB0
:1035C00025B12388C3F30B039D4204D0D4E9020143
:1035D000A28845F007F81C34BC42F1D3002386F8DA
:1035E0008430ECE7024C034FF6E700BF706A00201E
:1035F000708706086C8F06080A4B93F8843010B564
:1036000004460BB905F07AFCFCF7FCFB44B1012041
:1036100005F010FC20B9BDE810400348FEF7D0BC0F
:1036200010BD00BF706A0020594A06082DE9F04F0E
:1036300085B0164601911A46824600213046FFF7B2
:10364000ADFF324C06F0100305464FF0000902931F
:10365000FEF762FC2379019A03F01803934203D02A
:10366000002A48D1182B46D1284B4FF00D0B0BFBED
:103670000933B3F80900FCF731FB80462046FCF71C
:1036800078F8D8E902210746024401442046FCF7B5
:1036900029F880F001012A460390C9B23046FFF7AD
:1036A0007DFFDDE90223054602B123BB174A0BFB70
:1036B00009FB52F80BB0B2060FD573B91448039347
:1036C0005946FEF7C9FCD8F80820039B3A44214626
:1036D0005046FFF769F9FEF75BFC0E485946FEF7C6
:1036E000BBFCD8F80C2000233A4421465046FFF793
:1036F0005BF9FEF74DFC09F10109B9F50E7F04F104
:103700000D04A5D105B0BDE8F08F00BF9CA505084C
:10371000814A0608824A06080149FFF730BA00BF0D
:103720008C4A06082DE9F043064687B008460C4649
:1037300042F056FE082843D1671E03AD07342946E0
:103740003A46A84612F8010FFDF7A8F8A24201F880
:10375000010BF7D10023DFF87C908DF8143017F8B7
:10376000010FFDF79BF8C1B205F8010B4846019126
:1037700044F0B2FF20B10199284644F0ADFF28B1D2
:103780003046FFF7C9FF07B0BDE8F083A742E6D196
:103790000F4940462BF042FC0D480E49082310F813
:1037A000012B11F8014B18326A44013B02F80C4C12
:1037B000F5D109488DF8143003A9FEF78DFCE2E736
:1037C0000028E9D0304607B0BDE8F043FFF7EEB976
:1037D000486E00204C1106089B4A060807B5009366
:1037E00013460A460249FFF7CAF903B05DF804FB25
:1037F000A24A060820B10078B0FA80F0400970476C
:10380000012070472DE9F34106460846FFF7F2FF15
:103810000D46074670B1002401A920463DF070F91D
:10382000013401463046FFF7EDFF122CF4D102B00F
:10383000BDE8F0810846FDF74DF9C4B2112C71D8EE
:10384000681CFCF709F93B4D8046E8B93A4B03EB9D
:10385000440393F88C148A1E51425141364B03EBBA
:10386000440393F88C24AA5C002954D093F88D3437
:10387000192040F2EE2100FB03133048214602B02C
:10388000BDE8F041FEF728BC0178284644F024FF4B
:1038900070B1032C94BF00220122294902EB42029D
:1038A000431B0A4452FA83F393F87877032F04D129
:1038B000304602B0BDE8F0412EE74046FCF7CCF8B8
:1038C00008B3022FF4D1FDF705F940F6CA0280B221
:1038D0009042194BA8BF104640F2EE22904203EBF3
:1038E0004403B8BF1046A0F2EE201922B0FBF2F05C
:1038F00083F88D04BB1E594259410F4B03EB44031F
:1039000083F88C74AAE7022FF4D1304602B0BDE8E8
:10391000F041FFF74BB90B48214602B0BDE8F0413A
:10392000FEF7DABB084911233A46304602B0BDE83B
:10393000F04153E748130608687B0020BB4A06089D
:10394000688F0508CB4A0608D84A06082DE9F04FCB
:10395000024691B00846FFF74DFF0B46044628B1DA
:10396000104611B0BDE8F04FFFF720B94FF0FF321D
:10397000CDE90820A74ADFF8E482D2F88020DFF8FA
:10398000E09292F83810DFF8DCA2CDE90C10CDE916
:103990000E02CDE90A00A04907AA184644F058FED5
:1039A00027460546049426464DB9089A0C9FBA420C
:1039B00062D19A48FEF790FB11B0BDE8F08F062F58
:1039C00012D8DFE807F0041E2328454C5100514669
:1039D0002846FCF7B1FF78B14FF480600FF032F960
:1039E00090F90430089301248B4907AA002044F081
:1039F0002FFE01370546D7E72846FDF76BF80890FC
:103A0000F2E72846FDF766F80990EDE72846FCF74F
:103A1000AAFF0A90E8E7284642F0E2FC4146024647
:103A200005902846FCF764FF18B3059A49462846D6
:103A3000FCF75EFF06460028D6D02846FDF74AF878
:103A400004280646D0D901467548FEF745FBB3E782
:103A50002846FDF73FF800230C900F93C4E7284653
:103A6000FDF738F80D90BFE72846FCF77CFF0E9075
:103A7000BAE701230493B7E7DFF8EC8151B243467C
:103A800013F9010B884208D00135092DF8D1002126
:103A900064480131FEF720FB8EE763480121FEF701
:103AA0001BFB7AB2002318F9011B8A4200F00D813A
:103AB0000133092BF7D13A460121E9E7A7F11402B6
:103AC00053425341059308AD002303F10108EB680D
:103AD000A3BB95F900B058460FF07CF8D5F804A0C8
:103AE00020B1D0F80090B9F1000F5ED1BAF1000F0B
:103AF00019D14FF461436B604FF0010AAB680BB909
:103B00000323AB600023D5F8049002932A7A194668
:103B1000CDE9009258461A4613F0F4FFE86028B940
:103B20004248414691E74FF0000AE7E74A464146DE
:103B3000BAF1000F37D03E48FEF78EFAB8F1020F07
:103B400005F110054FF00103BFD1059BDDF83C8066
:103B50000B9D53B13748FEF733FAD8F800301B6A93
:103B60001BB135492A4640469847049B002B4ED04E
:103B70003249334B142F18BF19463248FEF7ACFABE
:103B8000142F09D1049B03B936B12B68DB691BB133
:103B90002D49324628469847002C67D100224146DD
:103BA00028463CF061FF2948C6E7C5F80C90BAF1F9
:103BB000000F25D0264841465246FEF74DFA5146A1
:103BC000484603F055FAD5F808A0BAF1000F0FD017
:103BD00099F8042092450BD01E4853464146FEF703
:103BE0003BFAD9F800305FFA8AF19B69484698475A
:103BF000D9F82C30002BA1D00023C9F82C309DE738
:103C0000D9F8082014484146FEF726FADBE70C49AC
:103C1000B3E700BF706A0020DD400608164B0608B7
:103C2000FE4A06085A4C06082F4B06083B4B06086E
:103C3000574B06080E4C060871700108E04A06084A
:103C4000964B0608374C060873FA00087B4B0608AB
:103C5000974B0608E94B0608C44B0608F84A0608C5
:103C60006A480608ED4A06084492050807F01CFA5F
:103C700005200AF0FDF91A4FDFF86C9000264FF08E
:103C8000030A99F89035B34288D917F801BBBBF104
:103C9000000F15D058460AF0C7FE044680B15846BA
:103CA00007F038F908B1A0F806A00121049006F049
:103CB00019FBE379049813F0010F03D005F0E0FD40
:103CC0000136DEE705F0E2FDFAE706483A46022152
:103CD000FEF702FA099B002B3FF4F0AE0023F1E659
:103CE000E82600202F4B0608840A001010B5044671
:103CF00008460B46FFF77EFD28B9094903221846FE
:103D0000FCF7F6FD28B90748FEF760F90120FEF739
:103D100027F920460449BDE81040FEF730BF00BF38
:103D20006C4C0608704C06084A4A06082DE9F74F05
:103D300005460846FFF75EFD0B46044618B9334AB0
:103D400092F8B07427B9284603B0BDE8F04FE3E419
:103D50002F49DFF8C880DFF8C890DFF8C8A001AAB3
:103D6000184644F075FC264610B907F0ABF908E098
:103D700056B9012201462846FFF700FA421C0446C4
:103D80001BD103B0BDE8F08FFCF7A4FE2F288346BB
:103D900036D80FB107F088F9BBF1060F14D01D49D2
:103DA000012391F890155FFA8BF2E0B209F0D0FF91
:103DB00059464846FEF790F90027154901AA002008
:103DC000013644F045FCCFE7DAF800351B0113D586
:103DD000FF2C0FD0E1B22846FFF7FAF9E8E72846B2
:103DE000FFF7F6F901370B4B93F89025F9B28A42A9
:103DF000F5D8DDE70027F6E70748FEF7E1F8D7E753
:103E00002F2241462846FEF7BAFED6E7687B0020FF
:103E1000DD400608840A0010924C0608B24C0608E1
:103E2000A14C0608706A00202DE9F04F064685B0C7
:103E30000846FFF7DFFC0B46044628B1304605B0C4
:103E4000BDE8F04FFEF7B2BE3149DFF8D490DFF89D
:103E5000D4A0DFF8D4B003AA184644F0F9FB2746F3
:103E60000546A04665B92B4B3A46D3F88000A1B26F
:103E700041F0B9FC68BB28493046FEF780FE28E0D7
:103E8000B8F1000F06D0B8F1010F25D03046FEF78B
:103E90008DFE1EE0284642F0A3FA494602460190F4
:103EA0002846FCF725FD50B3019A51462846FCF7F9
:103EB0001FFD30B3019A59462846FCF719FD10B38F
:103EC000019A16492846FCF713FDF0B13046FFF77A
:103ED00023FC05B0BDE8F08FBB1E5A425A4129466B
:103EE0003046FFF74BF9421C0446F2D0084903AABA
:103EF000002044F0ADFB08F101080546B2E7474653
:103F0000F4E70127F2E70227F0E70327EEE700BF17
:103F1000DD400608706A0020DE4C0608DB4C06080F
:103F2000D24C0608D54C0608D84C06082DE9F743B4
:103F300080460846FFF75EFC0B46054628B1404622
:103F4000FEF734FE03B0BDE8F0832E49DFF8B490ED
:103F500001AA184644F07CFB2F4604462E467CB945
:103F6000022DECD1A7F57A73B3F57A7F21D92649D2
:103F70004FF4FA634FF47A724046FFF72FFCE1E703
:103F80004DB1012D10D001AA4946002044F060FB3C
:103F900001350446E3E7012221464046FFF7EEF8EB
:103FA000431C0646EFD1CDE72046FCF793FD0746BC
:103FB000E9E7164DD5F8103AB8B25B689847FF2E7E
:103FC000BCEEC00A124B0BD195F89025F8EE407A62
:103FD000A24212DC10EE101A0E48FEF77DF8B1E78F
:103FE000F8EE407A03EB860310EE102A0A48C3ED80
:103FF000007A3146FEF770F8A4E7E3EC017A013469
:10400000E6E700BFDD400608EC4D0608840A001014
:104010001C800020094D0608FC4C0608F8B5074630
:104020000846FFF7E7FBC8B11F4B5E6A0136304612
:104030000EF004FC34460546F0B90134192CA8BF33
:10404000002420460EF0FAFB0546A8B9B442F4D18C
:1040500038461649BDE8F840FEF791BD0846FCF722
:1040600039FD04460EF0EAFB054628B92146104802
:10407000BDE8F840FEF730B80B4B5C6213F026FE4B
:104080000C482A462146FEF727F8182C09D80A487A
:104090000C2101FB040090F88007BDE8F84013F004
:1040A0004BBE0020F9E700BFA4050020184D06080C
:1040B0002C4D0608424D0608688F050838B5124D8C
:1040C00004460846FFF796FB60B1104B104893F981
:1040D00000104B1C0ABF0F4BC9B2197ABDE838401B
:1040E000FDF7FABF0846FCF7F5FC032804D8C0B278
:1040F000FDF7D2FB2946E4E720460749BDE83840F2
:104100000322FEF73CBD00BF964B0608A405002025
:104110005B4D0608706A00206B4D060838B5124DDD
:1041200004460846FFF766FB60B1104B104893F950
:1041300001104B1C0ABF0F4BC9B2597ABDE8384079
:10414000FDF7CABF0846FCF7C5FC032804D8C0B277
:1041500016F0E6FC2946E4E720460749BDE838406A
:104160000322FEF70CBD00BF964B0608A4050020F5
:10417000574D0608706A0020664D06082DE9F74F76
:10418000414BDFF81CA11A7A5B7A8AF800200546B9
:10419000012088468AF80130FFF72EFA00263B4CB2
:1041A000B1460D23394A7343414652F803B058468D
:1041B000FCF7C2FB002841D0B9F1000F01D0FDF798
:1041C000E7FE33485946FDF747FF002221462846BF
:1041D000FEF7C6FCFDF7DCFE237903F01803082B7D
:1041E00045D0102B48D02046FDF785FF274A0D23E8
:1041F00003FB0623B3F80900FBF770FD0746D8B1AF
:104200002046FBF7B6FAD7E90221009002440144A8
:104210002046FBF767FA78B9019059461D48FDF72B
:104220001BFF019AB9681346009A28460A442146A2
:10423000FEF7BAFBFDF7ACFE09F101090136B6F550
:104240000E7F04F10D04ACD10020FFF7B2F9FF237B
:104250008AF800308AF80130B9F1000F11D10E4907
:104260004246284603B0BDE8F04FFEF788BC0B4934
:104270002846FFF723FFB6E708492846FFF74EFF19
:10428000B1E703B0BDE8F08F706A00209CA5050877
:10429000864A0608864D060830480608964B0608EA
:1042A000A40500202DE9F74F074608460E4642F0C8
:1042B00097F8044620B1012825D133782A2B22D142
:1042C000A948AA4EDFF8C082FDF77AFE0025B14664
:1042D0004FF00D0A0AFB05F3404659F80310FDF7AD
:1042E000BBFE221E18BF0122314638460135FEF7BB
:1042F00037FCFDF74DFEB5F50E7F06F10D06E9D151
:1043000003B0BDE8F08F3D21304644F0E5F90028C8
:1043100000F0248103469A4613F8012D202AFAD092
:10432000AAEB060A431C994613F8012B202AFAD05F
:10433000DFF838B24FF000080D235FFA8AFA03FB6A
:1043400008F20BEB02045BF802100191084642F000
:1043500047F80199009002463046FCF7C9FA0D2350
:104360000546002853D1009A524550D1267906F0CF
:10437000E003402B00F0B8800ED8002B54D0202B47
:1043800000F08A8038467A49FEF7F9FB204603B0F0
:10439000BDE8F04FFDF7AFBE602B7ED0802BF1D192
:1043A000484642F01DF8E379A679DB0705460CD5AF
:1043B0002046FBF7A9FC0378014633B12A4648465C
:1043C00044F09FF9002840F0C380002D00F0C08029
:1043D000AE42C0F0BD800D2303FB08B3204693F826
:1043E00005A0FBF791FC3246002144F05EF9AA4596
:1043F0002BD860492A46484644F083F928B3204622
:10440000FBF782FC2A46494644F08FF91DE008F18B
:104410000108B8F50E7F92D157493246384603B0AD
:10442000BDE8F04FFEF7ABBB06F00702042A1CD133
:1044300019460A224846FCF7ABFAD4F80530834205
:1044400001469FD32046FBF777FC0D2303FB08F8BA
:104450004A485BF80810FDF7FFFD00222146384668
:1044600003B0BDE8F04FFEF77BBB4846FCF732FBDC
:10447000B4F80550B4F8071016F0050FAAB218BF2B
:104480002AB28BB218BF0BB29042FFF67BAF9842B4
:104490003FF778AF0146D5E76579394A02EBC505A4
:1044A000002695F8F4230092B2463346009AB242B1
:1044B00002D9BAF1000F03D0002B3FF463AFC4E779
:1044C000D5F8F01351F8260060B149460193FCF786
:1044D000EBF9019B30B9314620464FF0010AFBF75A
:1044E0002BFC53460136E1E76379009306F007069B
:1044F000013E009BAB42A8DD4846814610F8013BD7
:10450000202BFAD02046FBF7FFFB8246032E03D870
:10451000DFE806F0020F0F154846FCF7DBFA0AF851
:10452000050048462C2144F0D7F8013500F1010977
:10453000DFE74846FCF7CEFA2AF81500F1E700233A
:104540000A2219464846FCF723FA4AF82500E8E70C
:104550000C4932463846FEF712FB13E7314638461F
:1045600003B0BDE8F04F09E6964D06089CA5050886
:10457000E44D0608FA6C060830480608D94D0608CE
:10458000688F0508A94D0608864A06082DE9F04FF0
:10459000914689B00C461A4600218046FEF7FEFF80
:1045A000DFF8ECB006464D460027B9F1000F6CD09D
:1045B00029460622204644F04EF80028324614BF11
:1045C0000121002140460CBF4FF0010A4FF0000AC4
:1045D000FEF7E4FF0646287814F0D0FF079010B3EA
:1045E000687914F0CBFF079BEA785B790793AB7887
:1045F00095F801E04FF461714FF0190C1CFB0313A7
:104600001CFB0212297900B14079CDF804E0CDE914
:104610000232079B0093CDE904103B465A465146AF
:104620004046FDF701FD207814F0A8FF079010B375
:10463000607914F0A3FF079BE2785B790793A37876
:1046400094F801E04FF461714FF0190C1CFB031357
:104650001CFB0212217900B14079CDF804E0CDE9CC
:104660000232079B0093CDE904103B465A4651465F
:104670004046FDF791FC0137142F04F1060405F1C3
:10468000060592D109B0BDE8F08FCA46CBE700BF5E
:10469000F24D06082DE9F041064686B00846FFF7C0
:1046A000A9F80F46054638B100235D491A46012096
:1046B00006B0BDE8F04169E70846FCF70BFA13289D
:1046C000044600F3A38006264643781C8DF8175055
:1046D000FBF7C2F9534D074670B1FCF7FBF9C0B2C6
:1046E00014F062FF40B1AB19027983F858259DF8A8
:1046F000173001338DF817303846FBF7ADF9074610
:1047000068B1FCF7E7F90D2809D8062303FB045329
:1047100083F859059DF8173001338DF81730DFF80D
:104720000081B11C0DF1170241443846FCF7D6F95F
:10473000FBF792F9074668B1FCF7CCF9012809D8D4
:10474000062303FB045383F85C059DF817300133FF
:104750008DF817303846FBF77FF980B1FCF7BAF9CE
:10476000C0B214F021FF50B1062303FB04530279B9
:1047700083F85D259DF8173001338DF817309DF8CB
:104780001720042A4FF006032FD103FB0453002205
:10479000A3F85C2521F030F8062303FB04554FF401
:1047A000617695F8580514F0E9FE95F85B2595F8C3
:1047B0005A751923804695F85D0513FB076713FBAF
:1047C000026614F0DBFE437998F80520039395F810
:1047D0005C350097CDE90163134895F859352146BA
:1047E000FDF77AFC06B0BDE8F081052A05D103FB90
:1047F0000453002283F85D25CCE7062ACAD008EBD3
:104800000602002348F806309380C3E707491323C4
:104810002A46304606B0BDE8F041FEF7DFBF00BFD4
:10482000C86F0020706A0020F24D06080B4E060883
:104830002DE9F04F174689B01A460C4600218146F3
:10484000FEF7ACFE3B4EDFF8F4B007F16C03804698
:104850003D46079394F90410374A002392F9080063
:10486000884263D00133092B02F10C02F6D1079B79
:104870000C359D4204F10C04ECD109B0BDE8F08F79
:1048800029460C22204643F0E6FE0028424614BF8B
:104890000121002148460CBF4FF0010A4FF0000AE9
:1048A000FEF77CFEEA7995F9043006EB8202804639
:1048B000D2F8AC2804922A7A06EB82025146D2F84A
:1048C000AC280392AA7906EB82024846D2F8AC28BB
:1048D00002926A7906EB8202D2F8AC2801922A6829
:1048E00000925A46FDF7A0FBE27994F9043006EBFA
:1048F00082025146D2F8AC280492227A06EB820258
:104900004846D2F8AC280392A27906EB8202D2F88C
:10491000AC280292627906EB8202D2F8AC280192AE
:10492000226800925A46FDF737FBA0E7002FA7D177
:10493000BA46D9E7688F0508006F0020114E0608B7
:104940002DE9F04707468AB00846FEF753FF0446B4
:1049500038B1002354491A4601200AB0BDE8F04797
:1049600066E70DF11C080790C8E9010008464E1CD7
:10497000FCF7B0F84C4B40B21A4693F90410814250
:1049800000F08B800134092C03F10C03F5D10024D5
:1049900025463046FBF760F8064638B100230A2268
:1049A0001946FBF7F5FF01350790EDB2DFF800A1DE
:1049B0004FF000093046FBF74FF8064640B3FCF7CE
:1049C00089F83A49002251F804CB6045D3B203D0AC
:1049D0000132102AF7D100230AEB8302D2F8AC2867
:1049E000904215D1B9F1020F1FD0B9F1030F21D0B8
:1049F0005A1EB9F1010FD2B212D00B2A03D88DF88A
:104A000021300135EDB209F10109B9F1040FD1D11D
:104A1000052D15D838460AB0BDE8F047FEF7C6B8F0
:104A2000042AF0D88DF82230EBE7052BEBD88DF86F
:104A30002430E6E79A1E0D2AE5D88DF82330E0E70A
:104A400098E807001A4B84E807009DF8232003EB41
:104A500082020021D2F8AC2804929DF8242003EBB6
:104A600082020846D2F8AC2803929DF8222003EB7C
:104A70008202D2F8AC2802929DF8212003EB820337
:104A80000C4AD3F8AC380193079B00939DF9203072
:104A9000FDF782FA0AB0BDE8F0870C2303FB04247B
:104AA0008DF82000012574E7806E00201498050819
:104AB000688F0508114E06082DE9F04F8BB00C46A3
:104AC000089200211A460746FEF768FDDFF8B4B0E9
:104AD000089D099000264FF019094FF46178089B52
:104AE000002B4BD029460A22204643F0B4FD002873
:104AF000099A14BF0121002138460CBF4FF0010A6A
:104B00004FF0000AFEF74AFD2A890692EA880592CC
:104B10002A790492EA780392AA78099019FB028212
:104B200002926A7819FB028201922A780092334637
:104B30005A4651463846FDF777FA22890692E288AE
:104B4000059222790492E2780392A27819FB0282FC
:104B50000292627819FB0282019214F80A2B0092E9
:104B600033465A46514638460136FDF715FA1E2E91
:104B700005F10A05B3D10BB0BDE8F08FDDF820A038
:104B8000DBE700BF2E4E06082DE9F04380468BB0D0
:104B90000846FEF72FFE0F46044638B1002365494C
:104BA0001A4601200BB0BDE8F04385E70846FBF745
:104BB00091FF1D28054600F3B3800A264643781C62
:104BC0008DF82740FAF748FF044630B1FBF782FF23
:104BD0009DF8273001338DF827302046FAF73CFF47
:104BE000554C074668B1FBF775FF0D2809D80A2315
:104BF00003FB054383F8D4049DF8273001338DF877
:104C00002730DFF83091711C0DF1270249443846F6
:104C1000FBF764FFFAF720FF074668B1FBF75AFF7E
:104C2000222809D80A2303FB054383F8D7049DF8FB
:104C3000273001338DF827303846FAF70DFF074645
:104C400068B1FBF747FF0D2809D80A2303FB05438A
:104C500083F8D8049DF8273001338DF827309DF86C
:104C60002730062B0CD009EB0602002349F806304A
:104C7000404653601381FDF799FF0BB0BDE8F08308
:104C80000A2606FB054600233846A6F8DA34A6F8BD
:104C9000DC34FAF7E1FE074640B1FBF71BFF9DF855
:104CA0002730A6F8DA0401338DF827303846FAF7B2
:104CB000D3FE58B1FBF70EFF0A2303FB0543A3F80D
:104CC000DC049DF8273001338DF827301B4B4FF063
:104CD000FF325A600A2202FB05424FF46170B2F8BB
:104CE000DC340693B2F8DA34059392F8D83404939E
:104CF00092F8D734039392F8D614192313FB0101C9
:104D0000029192F8D51413FB0103019392F8D43465
:104D1000009300210A4A2B460846FDF73DF9ACE70F
:104D200008491D23224640460BB0BDE8F043FEF77C
:104D300055BD00BF3C800020687B0020A4050020FA
:104D40002E4E06080B4E06082DE9F04F2DED088B70
:104D5000DFF82CA195B0804691461F460C461646BA
:104D60004FF0000B94ED008AB5EE408AF1EE10FA98
:104D70007FD0D4ED019A94ED029AD4ED038AB9F173
:104D8000000F49D0D6ED00BA96ED01BAD6ED02AAD1
:104D900096ED03AAB4EE6B8AF1EE10FA6ED1F4EE42
:104DA0004B9AF1EE10FA69D1B4EE6A9AF1EE10FA6C
:104DB00064D1F4EE4A8AF1EE10FA0CBF0121002111
:104DC0003A460D46404681F00101FEF7E7FBB0EEA2
:104DD0006B0A074611A8FAF7BBFDB0EE4B0A079025
:104DE0000EA8FAF7B5FDB0EE6A0A06900BA8FAF71E
:104DF000AFFDB0EE4A0A059008A8FAF7A9FD05999B
:104E0000069A079B039002910192009352465B46DB
:104E100029464046FDF708F9B0EE480A11A8FAF70E
:104E200097FDB0EE690A05460EA8FAF791FDB0EEBF
:104E3000490A06900BA8FAF78BFDB0EE680A0590B8
:104E400008A8FAF785FD069B059A0390CDE9005363
:104E500002925B465246002140460BF1010BFDF7E2
:104E60009BF8BBF1080F04F1100406F110067FF463
:104E700079AF15B0BDEC088BBDE8F08F00219FE73E
:104E8000514E06082DE9F74FDFF898A1DFF898B1E9
:104E900007460D462846FEF7ADFC064638B100230E
:104EA00059491A46012003B0BDE8F04F4CE70522EE
:104EB00051462846FBF71CFD60B9534B00221A608F
:104EC0001A611A621A631A641A651A661A6703B0BD
:104ED000BDE8F08F4D4904222846FBF709FD044642
:104EE0002846002C44D1FAF7B7FD80460028EED0C2
:104EF00041F076FA464BC2B253F8049BB9F1000F69
:104F000007D144492A46384603B0BDE8F04FFDF7C3
:104F100036BE49464046CDE90023FBF7E9FC0134A3
:104F2000DDE9002306460028E6D1374A0346154648
:104F300000210133082B42F8101BFAD10BEBC404FB
:104F4000D4F8BCC0BCF1000F03D094F8B8E07645AB
:104F500005DB3148314D4946FDF7BEF89AE70CEBC9
:104F600006130FCB05EB061484E80F000136EEE7BD
:104F7000FBF7B0FD072804463DD82846FAF76CFD3C
:104F8000064658B3FAF7B2FA1F4B03EB041383ED4E
:104F9000000A01253046FAF75FFD064638B1FAF7F8
:104FA000A5FA194B03EB041383ED010A01353046D2
:104FB000FAF752FD064638B1FAF798FA124B03EBAE
:104FC000041383ED020A01353046FAF745FD38B97E
:104FD000384603B0BDE8F04FFDF7E8BD0546D9E718
:104FE000FAF784FA0848032D00EB041484ED030A51
:104FF0003FF455AFECE70A4907233246384603B081
:10500000BDE8F04FFEF7EABBC4720020654E06080B
:1050100074960508304806086A4E0608964B06083E
:105020000B4E0608F84A0608688F05082DE9F74F69
:1050300092460C461A4600218146FEF7AFFADFF889
:1050400070B0804656460025BAF1000F2ED031468A
:105050000422204643F0FFFA0028424614BF0121F3
:10506000002148460CBF01270027FEF797FA7388F6
:1050700001933AF82530009380462B465A4639462C
:105080004846FCF7D1FF6388019334F8043B009352
:105090005A462B46394648460135FCF77DFF042D1C
:1050A00006F10406D0D103B0BDE8F08F5746EAE719
:1050B000744E06082DE9F34105460846FEF79AFBB3
:1050C0000C46074638B1002333491A46012002B086
:1050D000BDE8F041AAE731492046FBF7E5FB03466E
:1050E00070B92D4A4FF47A704FF4FA610133042BF2
:1050F0001080518002F10402F8D102B0BDE8F081C5
:105100002046FBF7E7FC0328064641D82046FAF77D
:10511000A3FC074670B1FBF7DDFC4FF00108044625
:105120003846FAF799FC48B9284602B0BDE8F04184
:10513000FDF73CBD40F2EE248046F1E7FBF7CAFCE8
:10514000B8F1000FF0D0A4F2EE2240F2DC539A4204
:1051500003D8A0F2EE229A420AD9114940F6CA03B6
:1051600040F2EE22284602B0BDE8F041FEF736BB21
:105170000C4B0D4A03EB86030021A3F80046A3F86D
:105180000206CDE9004033460846FCF705FFB4E7C8
:10519000064903233A46E5E768810020F84A0608F5
:1051A000854E0608687B0020744E0608D84A06081B
:1051B0002DE9F04F89468FB0174600211A46064662
:1051C000FEF7ECF9DFF878A0054600240DF1240B7A
:1051D00059F824300293594602A83BF0F3FB67B319
:1051E00057F82430029A0393934218BF01212A46AC
:1051F00008BF002130460CBF4FF001084FF00008F7
:10520000FEF7CCF904A9054603A83BF0DBFB04A993
:1052100000912346524641463046FCF705FF23469F
:10522000CDF800B05246414630460134FCF7B4FE9A
:10523000202CCDD10FB0BDE8F08FB846EFE700BF0E
:10524000934E0608F0B5074689B00846FEF7D2FA35
:105250000E46054638B1002319491A46012009B007
:10526000BDE8F040A4E70846FBF734FC1F280446DD
:105270001DD83046FAF7F0FB0146204632F0E6FF33
:1052800078B10F4803AE314600EB84003BF09AFB47
:105290000C4A0096234629462846FCF77DFE09B0B5
:1052A000F0BD384609B0BDE8F040FEF735BA064912
:1052B0001F232A46384609B0BDE8F040FEF78EBAF3
:1052C00078810020934E06080B4E06082DE9F04F1A
:1052D000924685B00C461A4600218146FEF75EF9DB
:1052E000DFF874B0804655460026BAF1000F31D081
:1052F00029460422204643F0AEF90028424614BF56
:105300000121002148460CBF01270027FEF746F97E
:10531000EB780293AB7801932B8800938046334659
:105320005A4639464846FCF77FFEE3780293A37855
:10533000019334F8043B00935A46334639464846B5
:105340000136FCF729FE102E05F10405CDD105B07C
:10535000BDE8F08F5746E8E79D4E0608F0B50746D2
:1053600085B00846FEF746FA0E46054638B10023DA
:105370001C491A46012005B0BDE8F040A6E70846E2
:10538000FBF7A8FB0F28044623DC3046FAF764FB42
:105390000146204632F000FCA8B1134B04F1200274
:1053A00003EB8203294693F81326029293F8122600
:1053B0000192B3F8103600930C4A23462846FCF7B6
:1053C000EBFD05B0F0BD384605B0BDE8F040FEF796
:1053D000A3B907490F232A46384605B0BDE8F04077
:1053E000FEF7FCB9F8810020687B00209D4E06087E
:1053F0000B4E06082DE9F04F87B0144603911A466C
:1054000000210546FEF7CAF8DFF830B106464FF036
:105410000008062303FB08F7C0374FF00009039B81
:10542000DB5D0493002C00F08580E35D049A059316
:105430009A4218BF0121324608BF002128460CBFFE
:105440004FF0010A4FF0000AFEF7A8F8059B064648
:10545000CDE900935A46434651462846FCF7E4FD01
:10546000049B5A46CDE9009351464346284609F12C
:105470000109FCF791FDB9F1060F07F10107CED143
:1054800008F10108B8F1060FC3D1DFF8B0B0E42786
:10549000039BA7F1E40913F807A0002C4CD0E35DAF
:1054A00004939A45324614BF0121002128460CBFBF
:1054B0004FF001084FF00008FEF770F8049B064615
:1054C000CDE900935A46062341462846FCF7ACFD39
:1054D000CDE9009A194A0623414628460137FCF7D0
:1054E0005BFDEF2FD4D1039B93F8EF70B4B194F828
:1054F000EF804745324614BF0121002128460CBFEA
:1055000001240024FEF74AF8002300930B4ACDF84B
:105510000480072321462846FCF786FD00230093DC
:10552000064A0197072321462846FCF735FD07B0B8
:10553000BDE8F08FA24693E7A046C9E7AF4E060844
:10554000F0B5054687B00846FEF754F90B46044609
:1055500038B100231C491A46012007B0BDE8F040CD
:1055600048E71A49194F02AA184643F071F803AEEA
:10557000B8B1032C04D12846FDF718FB07B0F0BDE5
:10558000FBF7A8FA02AA46F8040B394600200134BA
:1055900043F05EF8ECE70E4832462146FCF79CFDEE
:1055A000ECE7032CE7D1DDE90346059B01931A469E
:1055B0003146E0B232F034FB019B0028EBD12846A3
:1055C000FEF7AAF8DAE700BF78810020DD40060880
:1055D000AF4E06082DE9F04F89B00C460792002126
:1055E0001A460746FDF7DAFF0026079DDFF8A0B050
:1055F0000690B2464FF019094FF46178079B43B308
:1056000029460622204643F026F80028069A14BFB1
:105610000121002138460CBF4FF0010A4FF0000A6B
:10562000FDF7BCFF6A79069019FB028205922A7980
:1056300019FB02820492EA780392AA7802926A78AD
:1056400001922A78009233465A4651463846FCF772
:10565000EBFC627919FB02820592227919FB028226
:105660000492E2780392A27802926278019214F88E
:10567000062B009233465A46514638460136FCF70F
:105680008BFC0A2E05F10605B8D109B0BDE8F08FF4
:10569000C34E06082DE9F04F80468BB00846FEF752
:1056A000A9F88946074638B1002355491A46012012
:1056B0000BB0BDE8F04F8DE7524C084694F86237C6
:1056C00094F878B694F879A60793FBF703FA0928BB
:1056D000054600F38B800626464309F101008DF84C
:1056E0002770FAF7B9F9074658B1FBF7F3F90D2817
:1056F00007D8A31983F890099DF8273001338DF856
:1057000027303846FAF7A8F9074668B1FBF7E2F9FF
:10571000834509D3062303FB054383F891099DF8CC
:10572000273001338DF827303846FAF795F90746C8
:1057300068B1FBF7CFF9504509D8062303FB0543B1
:1057400083F892099DF8273001338DF827303846C9
:10575000FAF782F9074670B1FBF7BCF9079B834261
:1057600009D3062303FB054383F893099DF82730EB
:1057700001338DF82730DFF88890311D0DF12702B5
:1057800049443846FBF7AAF99DF82730062B0BD081
:1057900009EB0602002349F8063040469380FDF7E6
:1057A00005FA0BB0BDE8F08F03FB05444FF46171BF
:1057B00094F89529192313FB0212059294F8942961
:1057C00013FB0213049394F89339039394F89239DA
:1057D000029394F89139019394F890390093002141
:1057E000094A2B460846FCF7D7FBDAE707490923A5
:1057F0003A4640460BB0BDE8F04FFDF7EFBF00BFA3
:1058000000740020706A0020C34E06080B4E060884
:105810002DE9F04F0F4689B0144600211A4606467E
:10582000FDF7BCFE0546002C00F0DB8022783B78BB
:105830009A4218BF0121024608BF002130460CBF22
:105840004FF001084FF00008FDF7A8FE23789B4AAF
:10585000054641463046FCF7E7FB3B78974A414610
:105860003046FCF799FB002C00F0BD8062787B7815
:105870009A4218BF01212A4608BF002130460CBFBA
:105880004FF001084FF00008FDF788FE63788C4A5E
:10589000054641463046FCF7C7FB7B78884A4146BF
:1058A0003046FCF779FB07F1CA030493822304F125
:1058B000CA0B05934FF002094FF0000A3B7853459D
:1058C00000F39380002C00F0F38097F8EA3094F80E
:1058D000EA209A4218BF01212A4608BF002130461B
:1058E0000CBF4FF001084FF00008FDF757FE94F889
:1058F000EA30744A054641463046FCF795FB97F876
:10590000EA30704A41463046FCF746FB07F1EC09A5
:10591000002C00F0CF8004F1EC034A4604F1FC01B6
:105920004FF001089A4633F802CB32F8020B844557
:1059300018BF4FF000088B42F5D188F001012A46CC
:10594000C9B23046FDF72AFE082105465046FAF74F
:10595000FBFE5D4A034641463046FCF765FB97F87F
:10596000EA104846FAF7F0FE574A034641463046E9
:10597000FCF712FB002C00F09F804FF0FC094FF069
:10598000010807EB090104EB0900FAF78DFF09F1A3
:105990000409002818BF4FF00008B9F58E7FF0D138
:1059A00088F001012A46C9B23046FDF7F7FD08210B
:1059B00004F1FC00FAF782F8444A034641463046B7
:1059C000FCF732FB97F8EA1007F1FC00FAF776F8DB
:1059D0003E4A03464146304609B0BDE8F04FFCF769
:1059E000DBBAA04639E7A04657E7059B3B44069340
:1059F000002C5BD0059B0698234419460793FAF7C1
:105A000053FF049B1A789BF800309A4206BFB0FA05
:105A100080F84FEA58184FF000084B4609F1100281
:105A2000F85AE15A0233884218BF4FF000089342F7
:105A3000F6D188F001012A46C9B23046FDF7AEFD25
:105A4000627804EB090105469BF81800FAF74EFE50
:105A500002909BF800300193079B00931C4A0AF1C7
:105A6000010341463046FCF7DFFA049B7A78187E42
:105A7000079307EB0901FAF739FE079B049A029096
:105A80001B7801930132069B04920AF1010A0093EC
:105A90000F4A534641463046FCF77EFA059B0933D0
:105AA0000BF1010B09F11009059307E7A046DCE7AC
:105AB000A04624E7A04652E7A04683E7DC4E06084E
:105AC000EE4E06081C4F0608344F06084B4F0608DA
:105AD000034F06082DE9F04F8FB0044602AA08468E
:105AE000AF4942F0B5FD064640B903460246AD490E
:105AF0004120FFF78DFE0FB0BDE8F08FAA49FAF7FD
:105B0000D3FE074620BBA64902AA42F0A1FDFAF740
:105B1000E1FF0828054606D9A44908233A4620464D
:105B2000FDF75CFEE7E7A24C94F87836834202DC8E
:105B300084F87856DFE7064604F5CF6731463846E5
:105B400031F03EF994F878360136B342F6DCEFE7EF
:105B500098493046FAF7A8FE0546E0B9904902AAEE
:105B600042F076FDFAF7B6FF0828064603D99249B7
:105B700008232A46D3E78E4C94F87936834202DC18
:105B800084F87966B7E72846314601353AF0F2FEE7
:105B9000082DF8D1F4E789493046FAF785FE074623
:105BA00000BB7F4902AA42F053FD0028A3D0FAF7B8
:105BB00091FF0828054603D9814908233A46AEE7F4
:105BC0007B4C94F86237834209DD014604F5CF60CF
:105BD00031F040F9294604F5CF6031F049F984F8F5
:105BE000625788E777493046FAF75EFE054618BBEC
:105BF0006F4BDFF8AC9193F8627706AE0146102246
:105C0000304642F052FDB046BD4202AA80F20E81FB
:105C10004946002042F01CFD10B96B493A460EE19E
:105C2000FAF758FF013528F8020BEDE796E80F0068
:105C3000664C84E80F005EE765493046FAF734FEAB
:105C4000054600283BD15A4B0DF1180893F862978E
:105C5000464607464F45524902AA4FF0000080F2DF
:105C6000F28042F0F5FC014610B95A494A46E6E096
:105C70000322304642F059FDB2464FF0000B304649
:105C800040F0AEFB584502D801370436E2E79AF8F7
:105C90000000FAF703FE0BF1010B0AF8010BEEE727
:105CA0004D494A46CBE041462046032231F070F888
:105CB0000135043408F10408AF42F4D11BE7474929
:105CC0003046FAF7F1FD0546002840F0AC80384F29
:105CD000334997F8788602AA42F0BAFC00283FF4CC
:105CE0000AAFFAF7F7FE461E01D4B04503DC3C4983
:105CF0004346012213E72A4902AA002042F0A8FCE9
:105D0000014600283FF4F7AE4FF00008082203A830
:105D1000CDE903888DF8148042F007FD0DF10C09E0
:105D200003A840F05DFB40451CD81D4902AA002095
:105D300042F08EFC00283FF4DEAE90F800A097F809
:105D40007996DFF8ACB04FF000084D45144902AA2F
:105D50004FF000007EDA42F07BFC024658B9214940
:105D60004A466CE099F80000FAF798FD08F101083E
:105D700009F8010BD4E7002D40D11378303B092BF3
:105D80003CD919490192FAF78FFD019A90B3104658
:105D90005946FAF789FD019A002838D013494EE098
:105DA000DD400608E8700020624F0608684F0608CC
:105DB000706A0020734F06087C4F06088A4F060859
:105DC000964F0608A84F060897500608D471002081
:105DD000D24F0608B7500608DE4F0608FC4F0608EB
:105DE00001500608D7500608AB40060814500608B4
:105DF0000D5006084FF001084FF0FF351046019294
:105E0000FAF768FE0028019A03DA214917E0A8464C
:105E1000F2E70EAB03EB4503013523F8200C94E7C2
:105E20001C494A460BE01C49324608E01B49002049
:105E300042F00EFC00283FF4F9AE19493A462046DC
:105E4000FCF79DFE57E642F003FC00287FF428AFE4
:105E5000144C31E742F0FCFB0028E1D1124C06EB78
:105E6000C6008230082203A9204430F091FF50463A
:105E7000FAF714FD37446A0087F8420704EB06106E
:105E800006A9023042F0AEFB87F85A8733E600BF1E
:105E9000495006085E50060881500608DD40060895
:105EA000B44F0608E4710020E870002070B50A4C79
:105EB0000A4E002594F8853013B12046FBF7F0FE1A
:105EC0002046FBF7C9FF01353046FBF7F7FF042DED
:105ED00004F19604EED170BDD86B0020842500201B
:105EE00038B50C46054616492046FAF7DDFC30B9B0
:105EF000FFF7DCFF1348BDE83840FCF761B81249F2
:105F00002046FAF7D1FCA8B9104A82F8ED0182F8D0
:105F1000F50182F8830282F88B0282F8190382F875
:105F2000210382F8AF0382F8B703094A82F82100FF
:105F30000848E0E72846BDE83840FDF7EDBB00BF64
:105F4000FC500608025106081D510608706A002020
:105F500084250020255106082DE9F04F89B00F4611
:105F600091460021139A98460646FDF717FB87EAEB
:105F700009096FEA0903DFF88490069304460025B7
:105F800028460CF049FC129B184230D0069BDFF8E3
:105F900070B0034014BF4FF0010A4FF0000A0493A1
:105FA00010EA070314BF4A465A462846059307924B
:105FB0000CF044FC079A039000904346514630464B
:105FC000FCF732F8049BB3FA83F1224649093046C4
:105FD000FDF7E4FA059A039B009304464346002A22
:105FE00014BF5A464A4651463046FBF7D5FF0135A5
:105FF000182DC5D109B0BDE8F08F00BF5F4E06086F
:106000004151060837B504460846019140F0E8F9C9
:106010000199054602462046FAF76AFC70B9625DAE
:106020001046FAF72BFC00B932B901352C44204652
:1060300001340378202BFAD003B030BD0020FBE7F9
:10604000F0B5032985B005460C46164614D80B4F0B
:106050003970FBF79DFF0A492846FEF72FF80949DA
:10606000224601A8FAF7E6FA01AB32460821284693
:10607000FDF7DCFAFF233B7005B0F0BDA40500205E
:10608000964B06085B4D0608F0B5032985B005461A
:106090000C46164614D80B4F7970FBF779FF0A4966
:1060A0002846FEF73BF8094922466846FAF7C2FA45
:1060B0006B46324610212846FDF7B8FAFF237B7065
:1060C00005B0F0BDA4050020964B0608574D060804
:1060D000F8B5114B93F88500D0B993F88C2012B124
:1060E00093F88D20A2B90D4E96F880748FB1187E6A
:1060F00070B90B4D0FCD06F5E0640FC495E80F00A5
:1061000084E80F00012386F83B3709F033FA38465C
:10611000F8BD0120FCE700BF706A0020687B00200A
:106120008C6A002038B50546FFF7D2FF044660B9F7
:1061300007492846FCF723FD06492846FCF71FFDC2
:10614000054B83F88C4083F88D40204638BD00BF56
:10615000FF49060848510608706A002008B5FFF795
:10616000E1FF50B1054B02229A75FBF743FD04484D
:10617000FBF72CFF0020FBF7F3FE08BD706A002040
:106180006651060810B5094C94F83C375BB9084BCA
:10619000084918680C2242F0B4FA012308B984F8BF
:1061A0003D3784F83C3794F83D0710BD687B0020EC
:1061B000002800086D5106082DE9F74F054601AA91
:1061C00008464A49DFF850B142F042FA4FF0000960
:1061D000012682464F464C46B046BAF1000F28D100
:1061E000B9F1000F2ED1424F002C7BD041482146FF
:1061F000FBF772FF97F884300BB902F07FFEF9F7D6
:1062000001FE002087F88D000EB102F013FEFFF7AB
:106210004DFE14B12046FDF7CCF9B8F1000F14D0B3
:106220002846FFF77FFF80B1FBF7E4FC0020FBF777
:1062300097FEB9F1000F0BD05046FAF74BFC84B231
:10624000002C3ED12846FDF767FA03B0BDE8F08F79
:1062500029495046FAF770FB00283CD1274950469F
:10626000FAF76AFB002839D159465046FAF764FB21
:10627000002835D122495046FAF75EFB0028E1D0CC
:10628000002FDFD1FFF77EFFB0B11E4B1E4D1C6803
:106290001E4E013C14F8011F4B1EDBB2FD2BD4D85F
:1062A0002B689C42D1D20A2903D03046FBF7D4FE9A
:1062B000F0E7FBF76DFEEDE715492846FCF75AFBC2
:1062C000C3E74FF00009094901AA002042F0C0F9D4
:1062D0000137824681E74FF00109F4E7C846F2E74B
:1062E0004E46F0E70B48FBF771FE88E7DD400608F5
:1062F000706A0020A65106087A510608BB550608A8
:10630000885106080028000804280008EE470608FF
:106310008D510608C95106088351060830B587B06B
:10632000144B0493144B0393144B0293144B01939B
:10633000144B154A00930546144B15480C46154955
:10634000FBF78AFEFBF724FEFFF71CFF58B112484B
:10635000FBF73CFE64B1114A1149124807B0BDE891
:106360003040FBF7B9BE10492846FCF703FBF1E7C4
:1063700007B030BD14520608195206082352060809
:106380002C520608E5430608DF5106087F6A002004
:10639000E95106086F5106083852060868FF0508DB
:1063A00060FF050854520608445206080121B5E76B
:1063B0002DE9F04F0A4687B000210646FDF7EEF8BA
:1063C0003B4C05903B4A2378608802EB8303D3F86B
:1063D000D4A9F9F783FC83680493374BC16893F819
:1063E0008420002A4BD0DDF8108004910027217909
:1063F0006279049B07FB012213F80290B8F1000FA9
:106400003FD018F80250059A4D4514BF01210021D4
:1064100030460CBF4FF0010B4FF0000BFDF7BEF8FC
:10642000013705907DB305F00F022D09403502922A
:10643000CDE90075214A534659463046FBF7F4FD35
:10644000B9F1000F2AD009F00F024FEA1919029290
:1064500009F14002CDE900725346184A59463046C8
:10646000FBF79AFDA279012A38BF0122BA42BEDCAD
:10647000134B0834A342A5D107B0BDE8F08F904676
:10648000B4E74546BFE7B8F1000FD9D00D4A0097F1
:10649000534659463046FBF7C7FDD1E77306E1D4B2
:1064A000084A0097534659463046FBF775FDD9E731
:1064B00054980508688F0508706A00208152060804
:1064C0003C9905089752060838B50C4B03EBC005FC
:1064D0000C4695F8EC280A4803EB8203D3F8D4194C
:1064E000FBF7BAFD95F8F23833B1611C0548BDE8F9
:1064F0003840C9B2FBF7B0BD38BD00BF688F050892
:10650000F35606084F41060873B50E461149054675
:10651000FAF7CAF918B93070012002B070BD2C78B2
:10652000602C8CBF613C413C072C10D80135012305
:106530000A2201A92846FAF72BFA019B9D4206D0B0
:106540000F2804D8013440EA04143470E4E7002032
:10655000E3E700BF034006082DE9F04F2DED028B65
:106560000A468BB000218246FDF718F86F4D814630
:1065700005F1800B00266E4B93F88440AB7AB34252
:1065800000F395801035AB45F4D140F21620F9F7B1
:10659000A5FBD0E902530CB12C461D460DF1100BA2
:1065A00015220021584642F080F800272E78002E50
:1065B00044D069780391304608F00EFA95F902301C
:1065C00002935A1C534208EE100A5341002C00F06B
:1065D000A9800399002214F802C0B44504EB02001C
:1065E00040F09C8090F90280029A424540F09480ED
:1065F00042788A4208BF012301220BF8072003F0EA
:1066000001034A4683F0010150460393FCF7C6FF9D
:10661000039B81464CB1474A18EE101ACDE900A2FF
:1066200030464246F9F7CCFA039B434A18EE101A5B
:10663000CDE900A23046029AF9F7C2FA0137152FC8
:1066400005F10305B2D16CB33A4FDFF8EC8004F1E9
:106650003F061BF8013B02930BBB2078F8B194F97D
:10666000022001321BD0617808F0B6F94A4605468F
:1066700001215046FCF792FF94F90220029B294623
:1066800081462078CDE900A7F9F79AFA2078029B95
:10669000CDE900A84FF0FF322946F9F791FA03340B
:1066A000B442D6D10BB0BDEC028BBDE8F08FE888C8
:1066B000F9F714FBD0E902230CB114461A46297AE3
:1066C0006B7A06FB013312F9038014B3E756B84521
:1066D0000CBF012300234A4614BF0121002150466C
:1066E0000293FCF75BFF029B814644B1114A31469D
:1066F000CDE900A228463A46F9F716FA029B0E4A5F
:106700003146CDE900A228464246F9F70DFA013696
:1067100031E74FF0FF37DAE700236DE703323F2A16
:106720007FF459AF4FF0FF386BE700BFCC05002076
:10673000706A002029200108991F01082DE9F04FF7
:1067400080468BB008460D463FF04AFE024678B3BD
:10675000A8492846FAF7CCF8044648BBFBF718FCD2
:10676000A548A64DA64FA74EDFF8E482FBF728FC0C
:1067700014203AF013F9E11004F007020131384611
:10678000FBF76AFC2B7F6A7F06EB8303D3F8D419EF
:1067900052B19D48FBF7A0FC0134102C05F12405F3
:1067A000E9D10BB0BDE8F08F4046FBF795FCF3E76D
:1067B0002846964905AA41F04BFF054620B90146F7
:1067C0004120FFF7C9FEECE79149FAF76DF820B9CF
:1067D00090494046FCF7D3F9E3E78F4E08270024A1
:1067E00031682846FAF760F8002808BF3446013FB0
:1067F00006F11006F4D154B988492846FAF754F83E
:1068000028B187492A464046FCF7B9F9C9E7002074
:106810007E498DF8130005AA41F01AFF0646002CA8
:1068200040D080B1FAF756F9451E09D4A37A9D42AB
:1068300006DAE2684AB1012303FA00F0104204D1FB
:1068400078493246DFE7784EFAE7E088F9F746FA0A
:10685000764A92F884301BB192F8853083F00103B8
:10686000D0E90212002B08BF0A46217A637A05FBA1
:106870000133002712F903A0039702EB030B6349CE
:1068800005AA002041F0E4FE8146A0BB684901232F
:1068900044B39BF900202046CDE900312946F9F7A1
:1068A00043F97EE768B10DF11301FFF72DFE28B122
:1068B0009DF81350284604F02DFB20B95D4932465F
:1068C000A1E7594EFAE7284603F070FB82462846B6
:1068D00008F06EF80390284608F0A6F8A34607468D
:1068E0002546CCE7CDE900319DF8130052463946E4
:1068F000F9F766F955E74649F9F7D6FF064658BB5A
:10690000ACB14D4FEDB2207972B2294603F002F8D6
:1069100000283FF446AF0288037800933146C2F363
:1069200003233846120BFBF7D7FB0136EBE7424C4B
:106930007979386872B203F04FFB00283FF431AF29
:106940000288037800933146C2F303232046120BDA
:10695000FBF7C2FB0136EBE738494846F9F7A4FFDD
:1069600010B34846FAF7B6F8064642B26CB1207941
:10697000E9B202F0CFFFC8B9CDF8009022683049E3
:106980006B1C4046FCF7FBF80BE77979386803F09D
:1069900023FB58B99DF813302A49CDF800901A0905
:1069A000403203F00F03ECE74FF0FF3606AF3946F5
:1069B0003046F9F7FDFE08A95046F9F7F9FE5645AD
:1069C00048D076B24CB18BF80060009721681E4821
:1069D00008AB6A1CFBF780FBE3E69DF81320039BE2
:1069E0001A489E701109009708AB02F00F0240315F
:1069F000F0E700BF88510608AB5206087802002075
:106A0000C1520608688F050834540608DD400608A0
:106A10002E450608D2520608CC050020E65206088C
:106A2000EA520608F9520608964B0608706A0020DA
:106A3000991F0108095306081B5306086A480608EF
:106A40003C5306085F53060887530608AA530608F6
:106A50007048060834B12168074808AB6A1CFBF788
:106A60003BFB9EE69DF813200448110908AB02F099
:106A70000F024031F3E700BFD2530608ED5306087A
:106A80002DE9F04F8BB0074640F216200391F9F73D
:106A900025F9039A044600213846FCF77FFD414A58
:106AA000D4E9025392F8844006460CB12C461D46A8
:106AB0001522002104A841F0F8FD05F13F030393DE
:106AC00095F80090B9F1000F31D095F801A0002C95
:106AD00065D0224600231178494558D128336B44AC
:106AE00092F80180012203F8182CD045324614BFD9
:106AF0000121002138460CBF4FF0010B4FF0000B75
:106B0000FCF74CFD064654B1B8F1000F07D0264BF8
:106B100000935A463B4641464846F9F795F8234BC1
:106B200000935A463B4651464846F9F78DF8039B79
:106B300003359D42C4D13CB3DFF86C90DFF86CA004
:106B4000651C0DF11008403418F8013BCBB915F85D
:106B5000013CB3B116B13046FBF738FA297815F885
:106B6000010CCDF800903B460022F9F76DF80022A9
:106B700015F8010CCDF800A03B461146F9F764F872
:106B800000260335A542DFD10BB0BDE8F08F0133FD
:106B9000152B02F103029ED14FF00008A5E7A04695
:106BA000A3E700BF706A002029200108991F01088F
:106BB0002DE9F04F80468DB008460D463FF010FCA1
:106BC000024628B9014601200DB0BDE8F04F57E755
:106BD0000390B1492846F9F78BFE039A30B9AF49C3
:106BE00040460DB0BDE8F04FFBF7C9BFAC492846A1
:106BF000F9F77EFE044600285BD1FBF7C9F9A948E6
:106C0000A94FDFF8E4B2DFF8E482FBF7D9F91720E7
:106C100039F0C4FE17F9015B002D3CD029465846D7
:106C2000FBF71AFADFF89C92DFF88CA200231A46D1
:106C3000910089B228460593049207F02BFF039038
:106C400007F0C8FF049A0178059B561CC9B11BB90F
:106C50000490FBF79DF90498039B4178DA79037857
:106C600002F0020208EB8303C1B10091D3F8D439DA
:106C70008E48002A14BF4A4652463146FBF72CFA8A
:106C80000123042E3246D3D113B98948FBF798F972
:106C900001340E2CBED10DB0BDE8F08FD3F8D4393D
:106CA0008448002A14BF4A4652463146FBF714FA7C
:106CB000E6E7002480498DF81B4007AA284641F0EA
:106CC000C7FC18B94046FCF727FDE4E70DF11B01AE
:106CD000FFF71AFC05460028F4D09DF81B603046EB
:106CE00004F018F920B975494046FBF748FFD2E790
:106CF000DFF8FC9123464FF0FF3403EB430212F818
:106D0000092096420BD0611C02D1002A08BF1C4604
:106D10000133152BF1D1631C15D16949E4E71C46F9
:106D2000654907AA002041F093FC0646002800F0C0
:106D30009E805949F9F7B8FD28BB624E624FDFF8D3
:106D4000B481044615E00025EAE7297A2868039112
:106D500007F02EFF0246E8796B79039910F0020FD5
:106D600014BF304638469B08009001334046FBF77D
:106D7000B3F901349DF81B00214607F02DFE0546AE
:106D80000028E2D187E7514902223046F9F7B0FDE9
:106D90000746002849D1B01CF9F79CFE9DF81BB0AE
:106DA0000346BA46013739465846039307F014FEA6
:106DB000039B38B94FEA1B12454900960BF00F03AD
:106DC00040323FE0027A9A42EBD1002D40D14FF0A1
:106DD000FF36BAF1FF3F9DF81B5008BF002504EBBA
:106DE000440409EB04030AF101025A7009F8045043
:106DF000FF220AAC9A709DF81B0022465146F9F713
:106E0000E7FC08AA31469DF81B00F9F7E1FC9DF864
:106E10001B20B2454FEA121120D12E4808AB02F0D8
:106E20000F024031FBF758F935E72B493046F9F7A7
:106E30003BFD50B39DF81B30284900961A0940329B
:106E400003F00F034046FBF79AFE24E74FF0FF3AAA
:106E500004EB44034B445E78013EBAE720480094BB
:106E600008AB02F00F024031FBF736F913E704EBF1
:106E700044041C4B0093A144024699F801109DF86C
:106E80001B000123F8F7E0FE05E7002DDED14FF0EF
:106E9000FF36B246A3E700BF2E450608D2520608C9
:106EA000885106080954060850FF050829540608A9
:106EB0004A5406083B540608DD40060850540608AC
:106EC00067540608A5410608964B06089054060824
:106ED000FD540608B95406086A4806089354060883
:106EE000D7540608991F010822540608688F050820
:106EF0009C2E00207B540608224BB0F5FA6F1A68CE
:106F00000346A8BF4FF4FA63B3F57A7FB8BF4FF4D6
:106F10007A73D20416D540F2DC52904215D007EEB7
:106F2000903A40F2DB529042F8EE677A1FD8DFEDDC
:106F3000166A9FED167A9FED160A77EEE67AA7EEAF
:106F4000870A7047B0F57A7F02D89FED120A704722
:106F500007EE903ADFED106A9FED107A9FED100A70
:106F6000F8EE677A77EEE67AA7EE870A7047DFEDEC
:106F70000D6A9FED0D7A9FED0D0A77EEE67AA7EE8A
:106F8000870A7047706F002000007A44D62000C046
:106F900000E082440000000000407A446610004097
:106FA0000000404200A0BB44D620004000008344C3
:106FB00010B584464FEA810E102312F4004F14BF1F
:106FC0000E2407245200013BCCF8004092B2F44456
:106FD000F3D100EB81128C01035142F821301220D1
:106FE00010BD00BF10B584464FEA810E0424130B78
:106FF00003EB430318331201013CCCF8003092B28A
:10700000F444F4D100EB01130A01845043F8214009
:10701000062010BD704700BF704700BF034B00EB58
:10702000400003EBC000407C704700BFA80900107F
:107030000023037043708370C3707047704700BFB4
:1070400000207047704700BF002070470120704744
:10705000704700BF704700BF704700BF704700BF58
:107060009FED010A704700BF00000000002070473C
:1070700003681B69184700BF03682DE9F0415F6A88
:107080001FB13B46BDE8F0411847002A164611DD06
:1070900004460D460E4400E023689B68204698474E
:1070A0000028F9D0236815F8011B1B682046984773
:1070B000AE42F1D1BDE8F08130B50A4B002193F921
:1070C00000205D78092AC8BF143A8418013125735D
:1070D0009D7885540829DA78227603F10403EED1ED
:1070E00030BD00BF74C20508C36B33B15B68426D2D
:1070F0009BB29A4205D3D01A7047D0E907239A422F
:10710000F9D2C0681044C01A704700BFD0E9091214
:107110000369914238BFC9188A1A016C39B14968AC
:10712000013B12FA81F2934204D9981A7047013B4D
:10713000981A704700207047036C13B190F86400F0
:107140007047D0E90903181AB0FA80F04009704777
:10715000C26B10B4034662B1426DC1685C69881AA3
:10716000013A205C5DF8044B08BF0A46C0B25A657C
:107170007047006A5C69411C205CDC68A14238BF32
:107180000A46C0B25DF8044B1A627047836E70B550
:1071900004460D460BB19847B8B1636AA269D5544D
:1071A000636A2169226C01338B4228BF002363622A
:1071B00032B3EFF31183502282F31288226C1168EC
:1071C000C90703D5DBB283F3118870BD516889B25A
:1071D00071B9D4E90950854218D0A6690644D66031
:1071E00018D9281A80B25060A562002184F8641072
:1071F000116841F00101DBB2116083F3118870BDA9
:10720000226ED36843F08003D36070BD012284F8FE
:107210006420D7E72569281A80B25060A162E4E7AC
:1072200070B5094C236873B10546002606E09968DD
:107230001A681E7321609047236823B15A68AA1AFE
:10724000002A1846F3DA70BD8CAF002070B5214CCF
:107250002378012B00D070BD1F4B1B68002BFAD088
:107260001E4D2B6828465B6898470028F3D01C4BBE
:107270001C4E1A68338892889A420ED21A4B1B4AC7
:107280001B7852680021217003F00203002AE2D02B
:10729000E3B9136892881A8370BD15490968002202
:1072A0004968EA622A6803FB01F12846D3689847D7
:1072B0000E4A3388526801333380002ACBD01368DA
:1072C000928859690A42E6D05A8370BD1368928841
:1072D000FAE700BF943F0020681E00206C1E0020CB
:1072E0008C3F0020923F0020B81E0020BC1E0020D2
:1072F000843F0020A64B1A6812F0040140F0EA8097
:10730000DFEDA46AA44B12F0200205D093F8D02040
:1073100012F0020240F0BC809FEDA04A93F80001F9
:1073200010F0010062D193F8011119B183F8020144
:1073300083F80101D3ED417A9FED997A9FED996A27
:1073400067EE877A93ED437AE6EE867A36EEC77A71
:10735000C3ED417A83ED427A002A40F08B80DFED65
:107360008D7A002193ED497A93ED4A5A37EEC76A38
:10737000D3ED487AA5EE067A37EE676A83ED497A4F
:10738000E5EE067AC3ED487AC3ED477A09B1C3ED5D
:10739000427A93ED4B6A93ED4D7ADFED835A93ED8C
:1073A0004E5AC3ED4B7A37EEC66AF0EE474AD6EE38
:1073B000254A7E4AF0EE477AE5EE247A127893ED7C
:1073C0004C6AC3ED4D7A37EEC67A0E2AA5EE076AEF
:1073D00083ED4C6A69D0242A27D1D3ED427A744BCD
:1073E000FDEEE77A17EE902A5A80704793F8010174
:1073F00028BB93ED417A012036EEC76A83ED437ACC
:1074000083F801010AB393F80221002A40F0878033
:1074100051B3D3ED357A77EEE65A012275EE875AED
:1074200083F80221C3ED445A7DE0372A40F0AE8054
:10743000FDEEE66A5E4B16EE902ADA80704793ED19
:10744000437A36EEC76A002ADDD193F80221002A7A
:1074500045D093F814219FED4F4A002A6BD0022AA1
:1074600002D009B1012A42D0D3ED477AF0EE466A44
:10747000012177E793F81411D3F8D420C3F8102131
:107480000120814283F8020118BFC3F8082166E792
:10749000D3ED387AB3F8E620F8EEE77AC3ED357A23
:1074A0005ABB9FED3E4A012238E764EE255AD3EDE0
:1074B000357A3F4BFDEEE55AFDEEE66A15EE902A71
:1074C000FDEEE77A1A8016EE902A5A8017EE902A7F
:1074D0009A807047304B0121D3ED316A13E70029C0
:1074E00051D093F814219FED2B4A002ABAD1F0EE27
:1074F000467A0121F0EE466A34E707EE902A9FEDC6
:107500002A6A9FED2C7AF8EEE77A86EE274AB4EEE7
:10751000C74AF1EE10FA88BFB0EE474AC3E7D3ED91
:10752000357AD3ED445A93F8142177EEE57AC3ED1A
:10753000477A002A93D1002996D093ED475A93F8C1
:10754000152175EE666A07EE902AF8EEE75A76EE98
:10755000877A9FED197AF0EEE77A67EEA57AF0EE7A
:10756000466AF4EEC77AF1EE10FAC4BF24EE077A49
:1075700087EE274AF7EE007A77EEC47A67EE867ACE
:10758000E5EE047AEEE69FED034A6DE7704700BF33
:10759000C4780020000000008CAF00209A99993E2A
:1075A000CDCC4C3FCDCC4C3E0000C842B421002095
:1075B000B82100206666663F00401C46038A2DE91C
:1075C000F047B0F80C901FFA89F919EA03092BD09B
:1075D00005460E464FF000474FF00008B9FA89F310
:1075E00027FA03F2D24391B21B3B298209EA02092E
:1075F000042B16D8DFE803F0352C231A0300B36AF6
:10760000002B37D003F1FF3A1FFA8AFAC6F8288018
:10761000746A34B123682046514698476468002C48
:10762000F8D1B9F1000FD9D1BDE8F0877068696B66
:10763000036889B29847B9F1000FCFD1F4E7B06879
:10764000A96B036889B29847B9F1000FC6D1EBE77F
:10765000F068E96B036889B29847B9F1000FBDD1B2
:10766000E2E73069296C036889B29847B9F1000FE5
:10767000B4D1D9E7E96A1FFA81FAC9E708B5254B01
:107680001B68DB040AD5B5EE400AF1EE10FA12D100
:107690009FED210A40F02EFB80B208BDDFED1F7A7E
:1076A000B4EEE70AF1EE10FA1CDA9FED1D0A40F085
:1076B00021FB80B208BDDFED197AB4EEE70AF1EEE6
:1076C00010FAE5D49FED177AB4EEC70AF1EE10FA7E
:1076D00014D870EE677A9FED147A9FED140AA7EE26
:1076E000870AE4E770EE677A9FED117A9FED110A41
:1076F000A7EE870A40F0FEFA80B208BDDFED0E7AF1
:107700009FED0E7A70EE677A9FED0D0AA7EE870A5D
:10771000CDE700BF706F00200080BB4400004042F6
:1077200000007A4400E0824466BEFFBE0060BB44B5
:1077300038DFFF3E00407A440000834466BEFF3ECF
:1077400000A0BB442DE9F04F0C4695B035490546E5
:1077500020461746FEF756FC0646002850D132490F
:107760002046FEF74FFC064600284BD12F49204605
:10777000FEF748FC0646002846D12D492046FEF774
:1077800041FC0646002841D120462A49FEF73AFC32
:107790000028064612BF0824264601240FB144F0F3
:1077A000100425493046FEF72DFC88B344F0200430
:1077B00014F480730CBF012000200793FBF71CFF1B
:1077C00014F0090F00F01E831C48FAF7FFFB00219C
:1077D0002846FEF7A3FD079B002B3BD11848FAF77C
:1077E000F5FB1848FAF7ECFB04F01803182B05D149
:1077F0001548FAF7EBFB1548FAF7E2FB01232AE0FC
:107800000124CBE70224C9E70424C7E78124C5E7A4
:107810000F493046FEF7F6FB0028C9D044F48074C7
:10782000C6E700BF3C550608435506084B550608F9
:10783000515506085A550608C05106085E550608F7
:10784000665506087E5506088A550608B25506088C
:107850008351060800230693FAF79AFB04F01003FD
:10786000B949BA480593FAF737FCB949B948FAF764
:1078700033FC04F48473082B07D1B7492846FAF780
:10788000F9FCB5492846FBF7A5FA14F080030993E3
:107890000ED1B24B93F83C21002AB14A03F59E73F6
:1078A00006BF012113460021AE4A2046FAF774FBB9
:1078B000AD492046FEF77CFDAC492046FFF7E0F8D5
:1078C000AB492046FEF748FEAA4BD3F800B0AA4BBE
:1078D0001B680493059B002B40F0D581A748FAF75D
:1078E00075FB059EA64B08939946049BDFF83CA3C5
:1078F0006BEA03034FF000080A9359F8047B002F4A
:1079000040F0C381049BDFF8289363EA0B0A089BCD
:1079100053F8042B03920893002A40F0E081994B1E
:10792000994A9A492046FCF783FF099B002B40F0B7
:107930007B82DFF80093DFF800A399F800209AF823
:107940000030DFF8F8829A4214BF01210021904AEA
:1079500020460CBF01270027FBF720FE9AF80030D5
:107960008C4A013B0646394658F823302046FAF740
:107970005BFB99F80030874A013B3946864F58F83F
:1079800023302046FAF708FBD7ED007A834AF5EE5C
:10799000407AF1EE10FA0CBF012100212046FAF7DF
:1079A000FBFA33463A467E497E4F7F4E2046FDF72E
:1079B000CBF97E4B01936FF07F4200923A683168B9
:1079C0002046FEF7C9FA7A4B019340F20222009258
:1079D000BA68B1682046FEF7BFFA059B002B40F05D
:1079E000AD817448FAF7F2FA059A73487349DFF8E3
:1079F00050C20826012710F8013B11F8018B03F152
:107A0000500EEE440EF8208C1CF801EB0EF15009DC
:107A1000E94409F8108C2FB1A3EB0E0EDEF100073C
:107A200047EB0E07013EE6D187F0010120468DF8B5
:107A30003860FBF7B3FD624A8DF8486010AB3946F9
:107A40002046FAF7F1FA5E4A0CAB39462046FAF7BF
:107A5000A3FA5C4B5C4A5D492046FDF7A9FB5C4BF1
:107A60005C4A5D492046FDF731FC5C4B564A57495C
:107A70002046FDF7BFFC5A4B5A4A5B492046FCF7AB
:107A800085FD5A4B5A4A5B492046FDF715F85A4B7B
:107A90005A4A5B492046FDF7C9FA5A4B5A4A5B4994
:107AA0002046FDF7B5FE5A4B5A4A5B492046FDF782
:107AB00091FD059B002B40F043815848FAF786FA68
:107AC000574FDFF880814FF0000B414602223846C5
:107AD00040F0C1FD002814BF01210021039A97F84E
:107AE00000A020460CBF4FF001094FF00009FBF742
:107AF00055FDBAF1020F039040F0258198F801205E
:107B00004FF0190A40F2EE231AFB0232019298F864
:107B10000020444B9A5C00925B46434A494620460B
:107B2000FAF782FA7A783F4B40F2EE211AFB021202
:107B300001923A789A5C00925B463B4A494620465D
:107B4000FAF72AFA80E000BFC25506088247060805
:107B5000D4550608A0470608964B06088CAF0020AF
:107B6000FA6C0608D9550608E6550608F0550608C9
:107B70008E430608048D00206C6F002029550608EE
:107B8000F89505080D560608806E0020D488002060
:107B9000145606081A560608C47200202356060812
:107BA000648B00205C7000208C8D0020325606080B
:107BB00039560608315506088C8A00204C110608F3
:107BC0009B4A06085A48060878810020AC820020AB
:107BD00045560608F88100202C83002040560608F0
:107BE0004B560608C86F0020A88500204F5606088F
:107BF0003C800020B483002058560608688100208D
:107C0000A083002060560608E87000204889002004
:107C10006956060800740020088C002035550608B7
:107C2000E484002048130608BB4A0608F6550608F7
:107C3000025606081C8E0020406E0020749605082F
:107C4000486E0020F47F00200BF1010BBBF1120FF6
:107C500007F1020708F102087FF437AF764B22469E
:107C600000212846FBF7E2FC230700F18280734ED7
:107C7000224631782846FEF7E3F9717822462846F5
:107C8000FEF702FAB4E06E4E2CE63B7823B30A9A74
:107C9000012303FA08F31A400CBF012100210392CB
:107CA000204632460B93FBF779FC049B63EA0B02F8
:107CB0000B9B1A4214BF012100213B465246064647
:107CC0002046FAF7B1F9039900393B46524618BFEE
:107CD00001212046FAF760F908F101080DE6039B3F
:107CE0001B784BB3049B4FF0010808FA07F813EA1E
:107CF000080F0BD06BEA030313EA080F4A46039BF5
:107D000014BF012100212046FAF78EF91BEA080F63
:107D100012D01AEA080832460CBF01210021204681
:107D2000FBF73CFCB8F100010646039B4A4618BF2E
:107D300001212046FAF730F90137E8E5414A54E6D7
:107D4000414B0393BCE698F80020404B9A5C0092AC
:107D50005B4649463E4A2046FAF766F93A783B4B7D
:107D60009A5C00925B463A4A49462046FAF714F973
:107D70006AE70027F9B2224628460137FEF760F984
:107D8000042FF7D12D4FDFF8EC803B7888F80030D6
:107D9000079B33B92F48FAF719F92F492846FCF702
:107DA0008DF9FF2388F80030F1B2224628460136CB
:107DB000FEF76AF9042EF7D1284C7B782370079BD5
:107DC000A3B92748FAF702F923492846FCF7A6F990
:107DD0002448FAF7FBF82448FAF7BAF8FF2323708F
:107DE000002015B0BDE8F04FFBF7E3BBFF23237085
:107DF000069B002BF4D01D48FAF7E8F81C48FAF768
:107E0000DFF8EDE7A10706D50C4B22461978284686
:107E1000FEF716F9E4E76207E2D5084B22465978E7
:107E20002846FEF731F9DBE7034B224618212846A6
:107E3000FBF7FCFBDCE700BF3C550608648E002026
:107E40002955060831550608355506084813060811
:107E5000CB4A06086D560608964B0608A505002075
:107E600090560608B7560608BD550608CA560608B5
:107E7000E0560608A4050020002263E4012261E424
:107E80002DE9F84F1F4DDFF88490DFF884A00646F7
:107E90000C4637274FF000082046FBF7ABFCD5F81F
:107EA00000B048B921465846F8F746FD20B9686841
:107EB0002146F8F741FD80B15846FAF749F869685C
:107EC00011B15046FAF7C8F8A96811B14846FAF757
:107ED000C3F8FAF75DF84FF00108013F05F110050E
:107EE000DAD12046FBF786FC48B9B8F1000F06D17D
:107EF000224630460449BDE8F84FFAF740BEBDE8D7
:107F0000F88F00BF94C20508F6560608F05606081A
:107F1000EA5606082DE9F0412F4C2368002B4AD081
:107F20000A2801D00D2844D12C4DFAF731F823212D
:107F3000284640F0D1FB08B1401B20602368002296
:107F40009BB902B1236025484FF48072002140F0B4
:107F5000ACFB234B1B78002B3CD0BDE8F041214803
:107F6000F9F7F6BF01220B46EAE7591E685C2028A4
:107F7000F8D002B123600022EA54DFF860801A4D85
:107F800037262F6840463946FEF73CF8014640B98F
:107F9000013E05F11005F4D114491548FAF7EAFC41
:107FA00005E0144B9D42F7D2EB6838469847002312
:107FB000C8E7FF2B0ED8A0F120025E2A0AD80BB921
:107FC000202807D05A1C2260044AD054BDE8F04152
:107FD000FAF720B8BDE8F081B8780020B877002023
:107FE000BC780020DA40060894C205080A57060843
:107FF0002657060804C60508F5F73EBA10B504462C
:108000003FF078FE81B22046BDE81040F5F734BA63
:1080100070B50468236A1B69054643B1236AD0F82A
:1080200094001B699847012824D002281FD0236A96
:10803000DA6952B95869002838D099692162BDE8D7
:108040007040C3E90522F3F73BBE216A94F828206B
:108050000E7B1433F6B22362C2B906BB2846F3F78F
:10806000B3FD28460121BDE87040F3F775BD00233C
:10807000236270BD236A143B014623622846F3F74E
:108080006BFD236ADA69002ADFD1D3E70021284695
:10809000F3F762FD002384F82830002EDED0AB68B1
:1080A000002BDBD01A689B885383D7E7236A1B7B9E
:1080B0002262002B08BF2846606270BD80690028DC
:1080C00034D003681A6A127B1ABBD3E904125B68C6
:1080D00049686AB110B4546800220A6022609A8824
:1080E0005DF8044B22F003021204120C9A808FE711
:1080F0001A891206FCD41A89D20708D400220A6011
:108100009A8822F002021204120C9A8080E79A895F
:10811000F1E78268002AD8D0116892880A83D3E9EF
:1081200004125B684968002AD4D1E1E7704700BFB8
:10813000806900B97047016830B4D1E904424B68E6
:10814000646872B15568002222602A609A8822F021
:1081500003021204120C9A800B6A1B7B9BB930BC81
:1081600056E71A891506FCD41A89D20713D40022BF
:1081700022609A8822F002021204120C9A800B6A82
:108180001B7B002BEBD08368002BE8D01A689B8800
:10819000138330BC3CE79A89E6E700BF30B504465C
:1081A000006E8389A16023F400531B041B0C8381A0
:1081B00095B06379009113F0040F21794FEA0332EF
:1081C0004FEA032303F48063ADF8083001F00103A4
:1081D00002F4005214BF4FF480550025002B4FF0DD
:1081E0000003ADF80620ADF80C3007BF00220823CD
:1081F0000C230422ADF804508D07694654BFADF836
:108200000A20ADF80A3036F013FF6279236ED007EA
:1082100000F18A8012F0080F9A8A7FD092B242F061
:1082200008029A829A8992B242F400529A81227983
:10823000D10732D5E06B002800F088800023E26D82
:108240000793CDE90B33CDE90F33CDE911334FF46B
:10825000807509936369E1680D9505920693626CD8
:1082600004924FF480634FF480350A9308910E9581
:1082700036F084FC04A9E06B36F016FDE16B236E4A
:108280000A6842F001020A609A8A92B242F0400201
:108290009A824968227989B26165920737D5206C44
:1082A00000285FD02369A26D0893A36CCDE9043246
:1082B000002240230025CDE906234FF480314FF4FE
:1082C00080630A930E91CDE90B55CDE90F55CDE9A9
:1082D000115509950D9536F051FC206C04A936F026
:1082E000E3FC226C236E506940F0800050611068FE
:1082F00040F01600106055609A8A92B242F08002F7
:1083000003F10C019A820A6842F040020A609A89DD
:1083100092B242F400529A8115B030BD22F00802A8
:108320001204120C9A827DE71D498B4223D0A1F5DD
:108330004C418B421DD001F580618B421DD1022042
:108340000121F4F7D7FA6279236E63E74FF6DF7104
:108350001980D96841F02001D960D96841F0100135
:10836000D9609AE7DA6842F0800203F10C01DA6022
:10837000C9E70120E4E70020E2E701F580618B42D4
:108380000AD001F580618B4208D001F544418B424F
:108390007FF440AF0520D3E70320D1E70420CFE7E7
:1083A0000010014030B50446006E21718389A26837
:1083B00023F400531B041B0C8381637995B013F0E5
:1083C000040F009214BF4FF480520022ADF8042035
:1083D0001A031B0203F48063ADF8083001F00103B7
:1083E00002F40052002B4FF00003ADF80620ADF868
:1083F0000C3007BF002208230C2304228D07694696
:1084000054BFADF80A20ADF80A3036F011FE62799B
:10841000236ED00700F18A8012F0080F9A8A7FD06D
:1084200092B242F008029A829A8992B242F40052C1
:108430009A812279D10732D5E06B002800F088803C
:108440000023E26D0793CDE90B33CDE90F33CDE97E
:1084500011334FF4807509936369E1680D950592B6
:108460000693626C04924FF480634FF480350A9354
:1084700008910E9536F082FB04A9E06B36F014FCEF
:10848000E16B236E0A6842F001020A609A8A92B296
:1084900042F040029A824968227989B26165920766
:1084A00037D5206C00285FD02369A26D0893A36C98
:1084B000CDE90432002240230025CDE906234FF404
:1084C00080314FF480630A930E91CDE90B55CDE9CD
:1084D0000F55CDE9115509950D9536F04FFB206CE0
:1084E00004A936F0E1FB226C236E506940F0800055
:1084F0005061106840F01600106055609A8A92B280
:1085000042F0800203F10C019A820A6842F04002B4
:108510000A609A8992B242F400529A8115B030BD35
:1085200022F008021204120C9A827DE71D498B4248
:1085300023D0A1F54C418B421DD001F580618B42C7
:108540001DD102200121F4F7D5F96279236E63E78A
:108550004FF6DF711980D96841F02001D960D968E0
:1085600041F01001D9609AE7DA6842F0800203F125
:108570000C01DA60C9E70120E4E70020E2E701F539
:1085800080618B420AD001F580618B4208D001F5F1
:1085900044418B427FF440AF0520D3E70320D1E76D
:1085A0000420CFE7001001402DE9F84FB74C94F8B4
:1085B0000031DB072DED028B074640F18180B44B83
:1085C00094F85E811E88B34DB8F1010F64D0B8F104
:1085D000020F3AD0B8F1000F46D094ED5C8AEB7BE5
:1085E00033B1AB8923B1AC4B1B78002B40F0E98051
:1085F00094F85F21424538BF42462B7A632B08D856
:10860000B8F1020F00F0FE8094F86811002940F0E4
:108610001081A24BDFEDA26A1A70D4E96030C4F871
:1086200084311B1A06FB03F307EE903AF8EEE77A63
:10863000B0EE487AA7EEA67AA97B84ED5C7A002991
:108640006FD1BDEC028BBDE8F88FB4F86231B34254
:10865000C3D2944B94ED5C8A1B68C4F874314FF01C
:10866000010884F85E81BAE7B4F86431B34220D3DC
:108670008C4BD4F874111A68EB7D03EB830303EB86
:108680008303521AB2EB830FA7DB4FF0010894ED7E
:108690005C8A84F85E81A2E7B4F86631B34280F068
:1086A0009C80B4F86031B3423CBF4FF0000884F8BE
:1086B0005E817C4B94ED5C8A1B68C4F874318EE754
:1086C00094F85E81A8F10303012B714B1E8834D905
:1086D0005B88704DF31A1433282B3FF675AFEB8887
:1086E000B34203D82A88B242BFF46EAFB6EB430F51
:1086F0003FF76AAF0323DFED6C7A674A84F85E3197
:1087000084F85F310023B0EE678AC4ED5C7A1370A1
:10871000A4F86031A4F86231A4F86431A4F8663199
:108720009CE0012A00F08E80022A8AD1BDEC028BE7
:108730000720BDE8F84F0FF0FFBA564DEA88964281
:1087400002D32988B14203D2B6EB420F40F38180B5
:108750005A88B21A1432282A00F28E8095F814C072
:108760004FF0000884F85E8184F85F81BCF1000F4F
:1087700000F0A080484B83F800C0AA88697C6B8811
:108780001FFA8CFC12FB0CF292B28A4213FB0CF320
:108790009BB2A4F8602186BF521A92B200228B428B
:1087A000A4F8623186BF5B1A9BB20023A4F866313D
:1087B000642384F869310023A4F86421C4F86C317F
:1087C00002E712F059F900284BD10223984542469E
:1087D00084F85F3138BF1A460FE7324BD4F8741172
:1087E0001A682B7E03EB830303EB8303521AB2EB6D
:1087F000830FFFF6F2AE4FF0020894ED5C8A84F826
:108800005E81ECE694F8680198B90121C4F86C71B6
:1088100084F8681107462549C3F1640307FB03F395
:1088200081FB0301DB17A3EBA153643384F86931A7
:10883000EFE6D4F86C011E493F1A8F42EBDB84F857
:108840006931E6E6BDEC028B0820BDE8F84F0FF079
:1088500073BAB8F1030F78D194ED5C8A4FF0030836
:10886000BDE62B7C83420BD301239845424684F816
:108870005F3138BF1A46C0E6B8F1030FECD0ACE662
:10888000002384F85F314246B7E600BF8CAF00207A
:10889000CC7F0020746F0020CB7F0020CA7F002097
:1088A000ACC52737B01E0020000000006BCA5F6B0C
:1088B00080969800294A29881268B6FBF1F10131A7
:1088C000082992F96C20DFF8A48028BF0821C8B2DB
:1088D0008A4288F800002ED06AB3214A92F80090AC
:1088E00009F1010202F003024A4524D04FF0FF3E95
:1088F0004FF0960B03460BE0BEF1FF3F03D1BCF1F6
:10890000000F08BF9646013202F003024A4515D017
:1089100014480BFB020C92469CF96CC06145EBD1EC
:108920005FFA8AF0F8F7B8FF0F4B98F800C01E887E
:1089300094F85E8121E7E04684461EE7BEF1FF3FE2
:108940000AD19C464FF0000817E75B88F31A1433EE
:10895000282B7FF6C4AE40E6F246E1E73C6E0020ED
:10896000786A0020D86B0020CC7F0020CB7F0020CD
:108970002DE9F843C94CA36820469847002870D0D9
:10898000B4F90E30A17D06EE903AB4F9103007EE3E
:10899000903AB4F9123007EE103AF8EEE66AF8EEC3
:1089A000E77AB8EEC77A0123092984F85430C4ED78
:1089B000126AC4ED137A84ED147A54D004F148009D
:1089C00026F000FCB64DAA8DAB6A002A40F030813B
:1089D000B44A1268520700F1F880B3F9022094ED0E
:1089E000137A07EE902AB3F90020B3F9043006EEAB
:1089F000902A06EE103AF8EEE77AF8EEE65A77EEAD
:108A0000677AD4ED126A94ED147A2B88C4ED137A48
:108A1000B8EEC66A76EEE56A37EE467AFDEEE66AAD
:108A2000FDEEE77ABDEEC77A002B79D116EE903ACB
:108A30001BB206EE903A17EE903A1BB207EE903A50
:108A400017EE103A1BB207EE103AF8EEE66AF8EEAF
:108A5000E77AB8EEC77AC4ED126AC4ED137A84EDF2
:108A6000147ABDE8F883D4ED0B5A94ED0C6A94EDBA
:108A70000D5AD4ED094A94ED084A8B4B67EEA55A7E
:108A800027EE866A67EE857A94ED0A5A1B78A6EE81
:108A9000A46AE6EE845AE6EE857AD4ED0E6AD4ED49
:108AA0000F4A94ED105AE6EE875AF0EE466AE4EE6D
:108AB000876AE5EE077AC4ED125AC4ED136AC4ED75
:108AC000147A002B7FF47EAF784B93ED055A93ED2B
:108AD000036A93ED047AD3ED014A93ED004A26EE42
:108AE000866A26EE877A66EE856A93ED025AA5EECF
:108AF000A47AE5EE856AA5EE846AD3ED064A93ED85
:108B0000075AD3ED085AA7EEA46AA7EE857AE7EED6
:108B1000A56A84ED126A84ED137AC4ED146A51E7F4
:108B200016EE903A1BB206EE903A17EE903A1BB250
:108B300007EE903A17EE103A1BB207EE103A95ED99
:108B4000025A95ED086AD5ED055AD5ED033A95ED33
:108B5000064AD5ED094AF8EEE66AF8EEE77AB8EE8D
:108B6000C77A76EEC56A37EE467A77EEE57AA6EEF4
:108B7000A35AF0EE466AE7EE845AE4EE876A95ED72
:108B8000016A95ED047AD5ED077A85ED025A35EE46
:108B9000462A75EEC72A36EEE73AA2EE236AA2EE1F
:108BA000847AE4EE837A85ED016A84ED126AC5ED7C
:108BB000055A85ED047A84ED137AC5ED086AC5ED92
:108BC000077AC4ED147ABDE8F883394EB6F89421DB
:108BD000322A73D0002A40F0CC8096F8B221002AC5
:108BE0003FF4FBAE06F5D27007C8324F4FF0000CD1
:108BF00087FB028E86F8B2C1D217A689C2EB2E126D
:108C0000921B9A8087FB0062C017C0EB221087FB83
:108C10000127C917C1EB271118805980264B012263
:108C2000A3F80EC0C3F80A20F9F71EF8AB6AD4E621
:108C3000B2F5C87F00F081801D4994ED127AD1ED24
:108C4000626AD4ED137A94ED146AF8EEE66A0026AF
:108C500076EE876A91ED637AA664B8EEC77AFDEE88
:108C6000E66A37EE277AD1ED647AC1ED626AF8EEF2
:108C7000E77ABDEEC77A77EE867A0020FDEEE77AD6
:108C8000012A188081ED637AE6645880C1ED647A28
:108C90002665988072D0013AAA8599E6981400104A
:108CA00060110010706F0020AE050020C873002016
:108CB0008CAF00201F85EB51AC6F00201A68C6F8FE
:108CC0009821B3F90420A6F89C21564ADFED567A84
:108CD000D268C6F8A02194ED127A0020002177EE28
:108CE000877AA0641980B6F89421FDEEE77A322ADB
:108CF000C6ED697A6FD096ED6A7AD4ED137AD4ED29
:108D0000146AE064B8EEC77A012A37EE277AD6ED06
:108D10006B7A5980F8EEE77ABDEEC77A77EEA67ADD
:108D20002065FDEEE77A998086ED6A7AC6ED6B7A6A
:108D300062D0013AA6F894214FE7D4ED126A94ED7F
:108D4000137AD4ED147A394EFDEEE66ABDEEC77A99
:108D5000FDEEE77A00200021A064C6ED626A19806A
:108D600086ED637AE0645980C6ED647A2065998067
:108D700091E7D6ED697AF8EEE77AACE717EE906AFC
:108D8000DFF8ACE0B4F80C80C8368EFB061916EE9E
:108D900090CAF11717EE107AC1EBE9110CF1C80C6B
:108DA000A1EB08019980C8378EFB0C614FEAEC7C7F
:108DB000CCEBE11C8EFB071EFF17C7EBEE17A3F8E9
:108DC00000C05F80174BC3F80A20D881F8F74CFF2A
:108DD000AA8DAB6A5FE794ED137AD4ED147AE06460
:108DE000BDEEC77AFDEEE77A598086ED6A7A206596
:108DF000C6ED6B7A99809CE70B2086F8B12186F846
:108E0000B0110EF099FFAB6AD6F898211A60B6F946
:108E10009C219A80034AD6F8A011D160B6F894211B
:108E200087E700BFAC6F0020000000008CAF00207F
:108E30001F85EB512DE9F84FDFF8B49099F80050F9
:108E400006461DB100242046BDE8F88FFDF79AF9CB
:108E500004460028F6D0DFF89C80D8F80070C8F8E7
:108E600000500EB11C4B1D601C4E1D491D48DFF803
:108E700088B04FF480723FF0B5FB0023D6F800A015
:108E80003360012389F80030174B1D68013D15F848
:108E9000010F431EDBB2FD2B03D8DBF80030AB42E1
:108EA00016D80D20FFF736F8002389F800301FB1DF
:108EB000094BC8F800701F604FF4807209490848D8
:108EC0003FF090FB094BC6F800A001229A73BAE765
:108ED000FFF720F8DBE700BFF86A0020B878002031
:108EE000B87700203FB1002000280008786A0020F1
:108EF000F56A0020B47700200428000838B5074C34
:108F0000074DAC4203D3074B01221A7038BDD4E998
:108F10000210A2883FF066FB1C34F2E77087060857
:108F20006C8F0608F46A0020302821D0312826D022
:108F3000322828D0332828D0342828D0352828D0E3
:108F4000202828D0212828D0102828D0112828D03F
:108F5000122828D0132828D0142812D0152826D05B
:108F6000162826D0172808BF0F2202D000207047ED
:108F70000022114B03EBC20393F8940370470122C4
:108F8000F7E70C22F5E70222F3E70322F1E70422D8
:108F9000EFE70522EDE70622EBE70722E9E70822E3
:108FA000E7E70922E5E70A22E3E70B22E1E70D22E2
:108FB000DFE70E22DDE700BF74C205080123302879
:108FC00003FA01F129D031281ED032281CD03328D1
:108FD0001AD0342813D0352811D020280FD02128BA
:108FE0000DD0102810D011280ED012280CD0132824
:108FF0000AD0142803D0152801D0162809D111F061
:10900000030018BF0120704711F0070018BF0120AE
:1090100070471728F3D00020704711F0070018BFE1
:10902000184670472DE9F04F824C94F80661012EE6
:1090300083B007D000EB800004EB8004E08903B02C
:10904000BDE8F08F7C4B1B6893F83470002F5AD02A
:109050007A4B7B4D1B7801934FF0000E2346F04670
:10906000F14640F6FF7A4FF6FF7B1BE001F4706299
:10907000B2F5006F7FD059D8B2F5806F74D0B2F5D9
:10908000C06F44D1C9B24CF0080C998283F81EC05D
:109090000EF1010E5FFA8EF2974203F1140305F10F
:1090A000020529D993F81EC09989BCF1010FDDD1C1
:1090B000514500F09980C1F30802490A02FA01F112
:1090C0008AB2002A00F08580520802F51222BEF111
:1090D000030F02F5F86289B2B2FBF1F103D8019AED
:1090E0002D2A00F089805945D2D083F81EC0D9813D
:1090F000894408F10108CBE7B8F1000F03D0B9FBB0
:10910000F8F8A4F80481022384F8063192E7B2F556
:10911000007F37D14CF0020C83F81EC093F81FC0BB
:10912000CAB294451A82B3D2D977B1E7B2F5406F8B
:1091300013D0B2F5606F06D1C9B26CF07F0C998381
:1091400083F81EC0A4E7B2F5206F1BD1C9B24CF062
:10915000200C198383F81EC09AE7C9B24CF0400C6A
:10916000598383F81EC093E7C9B24CF0040C5982AE
:1091700083F81EC08CE7C9B24CF0100CD98283F87A
:109180001EC085E7514548D0C1F30802490A02FADA
:1091900001F18AB2EAB1520802F51222BEF1030FC0
:1091A00002F5F86289B2B2FBF1F10ED8019A2D2ACC
:1091B0000BD1594529803FF46BAF894489B24CF0FB
:1091C000010CD98183F81EC093E759453FF460AF85
:1091D000F3E7BEF1030F3FF65BAF019A2D2A7FF450
:1091E00057AFA5F800B053E7BEF1030F0DD94FF00C
:1091F0000002DA819E777CE7594529803FF448AF29
:10920000894489B2D9819E7773E7019A2D2AEED1DC
:109210004FF000022A800021F4E7BEF1030F02D8CC
:10922000019A2D2A01D00021C9E74FF000022A80BF
:109230000021C4E71005001094140010B421002090
:10924000B82100202DE9F04F6F4B1B7887B0002B21
:1092500000F0D3806D4E6E48B168DFF8F8A1F8F7E2
:109260003BFF71686B48F8F737FF6B4B6B48D3E9EE
:109270000031C91A6A4B1A68B1FBF2F2F8F72CFFF9
:10928000F8F786FE6748F8F79BFE6748F8F798FE00
:109290004FF00009654B1B785FFA89F4A34222D88E
:1092A000634C644FF8F774FE2646002556F8041BFD
:1092B00038460135F8F7D0FE162DF7D1F8F768FEDD
:1092C0005C4E0125234661681B683046C91A01358A
:1092D000F8F7C2FE162D04F10404F3D107B0BDE87F
:1092E000F04FF8F755BE4FF0140808FB046820460D
:1092F000FFF798FE98F81EE04F4B1EF0010F93F811
:10930000243014BF52222D22C8251EF0020F00FB6C
:1093100005F5B5FBF3F514BF54232D231EF0040F00
:1093200007EE903A14BF56232D231EF0080F14BFEA
:109330004FF0430C4FF02D0CA9B21EF0800F4FF0F0
:109340003C0BB1FBFBF105914FF0640114BF4FF0F2
:10935000530E4FF02D0E4843671CADB2CDE902E02D
:109360000093049517EE903ACDF804C03946504664
:10937000F8F772FE98F81E30DB073AD55C232F4AC7
:109380006343D118D05891ED010A70B1DFED2C7A0A
:10939000B8EE400A20EE270A07EE900AF8EE677A48
:1093A00080EE270A3EF0A6FC00B2642290FBF2F1A8
:1093B00002FB11022348F8F74FFE142101FB076757
:1093C00001FB0464F988628A0491218B0391E18A8C
:1093D0000291A18B0191A18A009102F0030319214E
:1093E0004B431948218A9208F8F776FE09F10109E2
:1093F00050E71648F8F7ACFDDFE7154807B0BDE8C1
:10940000F04FF8F7DDBD00BF04000010100500109C
:109410002C5706083C570608240900105357060825
:10942000B43A002080570608DC57060814100010D4
:10943000BC0500108C580608E02600201806001015
:1094400000401C46555806086A5806086158060828
:109450009058060838580608002800F094810368E0
:109460002DE9F04F0C4C03F13F4505F57E0504EB6B
:109470009524012594F8104404F01F066409032C78
:1094800005FA06F500F09C81042C00F07D81022C89
:1094900000F07F8102E000BF74C205088088B0FA46
:1094A00080FCCCF11F0CCCF3CC0603EB86060CF051
:1094B000070C346A4FEA8C0C0F2502FA0CF205FAFD
:1094C0000CFC24EA0C043462346A01F003052243E4
:1094D00032626A1E012AC1F38107C1F30018C1F389
:1094E000411E40F21181C2070ED51A6822F0030214
:1094F0001A601A682A431A60DA6822F00302DA60F6
:10950000DA684EEA0202DA6087070FD51A6822F09D
:109510000C021A601A6842EA85021A60DA6822F0C0
:109520000C02DA60DA6842EA8E02DA6046070FD58A
:109530001A6822F030021A601A6842EA05121A60AC
:10954000DA6822F03002DA60DA6842EA0E12DA6093
:1095500004070FD51A6822F0C0021A601A6842EA9E
:1095600085121A60DA6822F0C002DA60DA6842EA2C
:109570008E12DA60C1060FD51A6822F440721A60A2
:109580001A6842EA05221A60DA6822F44072DA6048
:10959000DA6842EA0E22DA6082060FD51A6822F4EF
:1095A00040621A601A6842EA85221A60DA6822F478
:1095B0004062DA60DA6842EA8E22DA6047060FD546
:1095C0001A6822F440521A601A6842EA05321A6098
:1095D000DA6822F44052DA60DA6842EA0E32DA607F
:1095E00006060FD51A6822F440421A601A6842EA49
:1095F00085321A60DA6822F44042DA60DA6842EAB8
:109600008E32DA60C4050FD51A6822F440321A602F
:109610001A6842EA05421A60DA6822F44032DA60D7
:10962000DA6842EA0E42DA6081050FD51A6822F440
:1096300040221A601A6842EA85421A60DA6822F407
:109640004022DA60DA6842EA8E42DA6042050FD5DB
:109650001A6822F440121A601A6842EA05521A6027
:10966000DA6822F44012DA60DA6842EA0E52DA600E
:1096700007050FD51A6822F440021A601A6842EAF8
:1096800085521A60DA6822F44002DA60DA6842EA47
:109690008E52DA60C6040FD51A6822F040721A6042
:1096A0001A6842EA05621A60DA6822F04072DA60EB
:1096B000DA6842EA0E62DA6084040FD51A6822F092
:1096C00040621A601A6842EA85621A60DA6822F01B
:1096D0004062DA60DA6842EA8E62DA6041040FD5ED
:1096E0001A6822F040521A601A6842EA05721A603B
:1096F000DA6822F04052DA60DA6842EA0E72DA6022
:1097000002044BD4BDE8F08F00210A4601264FF039
:10971000030906FA02FC3CEA00042DD11C6809FA90
:1097200001FA24EA0A041C60D3F800B005FA01F437
:1097300044EA0B041C609C6824EA0A049C60D3F889
:1097400008B007FA01F444EA0B049C605C6824EA60
:109750000C045C60D3F804C008FA02F444EA0C0478
:109760005C60DC6824EA0A04DC60D3F80CC00EFA02
:1097700001F444EA0C04DC600132102A01F1020118
:10978000C7D1BDE8F08F7047104C266B3543256379
:1097900084E60E4C666C354365647FE61A6822F0F9
:1097A00040421A601A6842EA85751D60DA6822F044
:1097B0004042DA60DA6842EA8E72DA60BDE8F08F21
:1097C000024C266C3543256468E600BF0038024031
:1097D00010B5437B82680446581C6073D154627B89
:1097E000237B934206D82AB12368D4E90101984724
:1097F0000023637310BD00BF427B42B110B5036804
:109800000446D0E9010198470023637310BD7047F7
:1098100003685A6A32B1904200D0FEE71A6A002A01
:10982000FCD170471A6A002AFCD17047134B1B68A1
:10983000B0EB930F14D2B0EBD30F13D2B0EB131FD6
:1098400012D2B0EB531F11D2B0EB931F10D2B0EB7A
:10985000D31F0FD2B0EB132F0ED24FF4807070478E
:10986000022070470420704708207047102070477E
:10987000202070474020704780207047E818002063
:1098800010B1036882885A83704700BF10B1036823
:1098900082881A83704700BF013902292CD81B4BDC
:1098A0004FF02C0C0CFB01FC10B403F52D74634439
:1098B000644493F8B42204604FF0010C022A80F84B
:1098C00088C003F52D7419D0C9B2114A0901525844
:1098D000C3F8B82272B1022283F8B42200F1100159
:1098E0004FF480724C30A281C3E9B31060465DF83A
:1098F000044B70470020FAE70020704793F8C1221C
:109900006244604683F8C122F1E700BF8CAF0020BB
:10991000AC260020D3B2012B23D870B502EB420253
:10992000114C4FEA820E4FF0000C22460EF1080552
:10993000634604E00133152B11D012F81CCF6045AB
:10994000F8D192F801C08C45F4D15659002EF1D0CF
:10995000C3EBC3030EEB83030433E01870BD002098
:1099600070BD0020704700BF8CC6050810B40468A5
:10997000EFF3118C102383F312880268536AB3B19A
:10998000984214D08B680A461BB1D3691432002B5D
:10999000FBD1236ACBB19C683CB9934215D01C68BB
:1099A0008CB15B689C68002CF7D01433F3E7136A22
:1099B000002BE7D121625FFA8CFC8CF311885DF8F3
:1099C000044BF2F77DB9C3E900015FFA8CFC8CF31C
:1099D00011885DF8044B704730B593B00446089287
:1099E0008DF80710002201210DF10705CDE9025283
:1099F000CDE9062204918DF8142009938DF82810E2
:109A000000238DF83C100B920E92109202A90022B6
:109A1000CDE90C23FFF7AAFF23685A6A3AB19442B2
:109A200000D0FEE71A6A002AFCD113B030BD1A6AD2
:109A3000002AFAD01A6A002AF9D1F6E730B505688B
:109A40008C462978012997B032D0022904D11C46CE
:109A50006B6A23B1984202D0002017B030BD2B6A48
:109A6000002BF9D16CF07F019FED237B8DF817104F
